:100000000C94DE170C9417180C9417180C941718EE
:100010000C9448440C9448440C9448440C94484430
:100020000C9417180C9417180C9417180C94171894
:100030000C9417180C94962B0C9417180C941718F2
:100040000C9417180C94FD270C949FD20C9417183D
:100050000C94698F0C945F8F0C9417180C941718DC
:100060000C9417180C9417180C9417180C94171854
:100070000C9417180C9417180C9417180C94171844
:100080000C94B1830C9417180C9417184E414E49D8
:100090004E495459494E46CDCCCC3D0AD7233C1746
:1000A000B7D13877CC2B329595E6241FB14F0A0093
:1000B0000020410000C84200401C4620BCBE4CCA83
:1000C0001B0E5AAEC59D7400407A10F35A00A07200
:1000D0004E18090010A5D4E80000E8764817000083
:1000E000E40B54020000CA9A3B000000E1F5050051
:1000F0000080969800000040420F000000A086019A
:10010000000000102700000000E803000000006469
:1001100000000000000A00000000000100000000D4
:10012000002C76D888DC674F0823DFC1DFAE59E1A9
:10013000B1B796E5E3E453C63AE651997696E8E618
:10014000C28426EB898C9B62ED407C6FFCEFBC9CEB
:100150009F40F2BAA56FA5F490055A2AF75C936BFD
:100160006CF9676DC11BFCE0E40D47FEF520E6B5B8
:1001700000D0ED902E0300943577050080841E0892
:100180000000204E0A000000C80C333333330F98B0
:100190006E12831141EF8D2114893BE65516CFFE77
:1001A000E6DB18D1844B381BF77C1D901DA4BBE403
:1001B00024203284725E228100C9F124ECA1E53D45
:1001C000275045544700504C41005072696E7420CE
:1001D00041626F72746564004D3235005061757311
:1001E000696E672E2E2E004D323400454550524F19
:1001F0004D2056657273696F6E204572726F720082
:10020000454550524F4D20496E64657820457272C5
:100210006F7200454550524F4D2043524320457266
:10022000726F72003F0049676E6F726500526573AE
:10023000657400496E697469616C697A6520454529
:1002400050524F4D0000FE0003FF8007C7C007015A
:10025000E00000E00000F00000700400700E00708C
:100260001F00703F80F00E00E00F01E007C7C003E1
:10027000FF8000FE0000FE0003FF8007C7C00F01E3
:10028000E00E00E03F80F01F00700E007004007070
:100290000000700000F00000E00701E007C7C003A5
:1002A000FF8000FE000E000E000E000E000E000E7D
:1002B000000E000E007FC03F801F000E00040004EF
:1002C000000E001F003F807FC00E000E000E000ECB
:1002D000000E000E000E000E00FFFFFF7F80FFC02B
:1002E000FFC0FFC07F807F80FFC0FFC0FFC03F0016
:1002F0001E000C0050726F6265205A204F666673B4
:1003000065740020082046616374002008204D6158
:1003100078002008204D696E004F6666004F6E0021
:100320004175746F74656D700045207374657073EA
:100330002F6D6D005A2053746570732F6D6D0059C9
:100340002053746570732F6D6D0058205374657061
:10035000732F6D6D00416476616E63656420536533
:100360007474696E67730054656D7065726174753D
:1003700072650053746570732F6D6D00436F6E6608
:10038000696775726174696F6E003F004E657874BD
:1003900020436F726E657200446F6E65004E657823
:1003A0007400486F6D696E672058595A0053746F16
:1003B00072652053657474696E6773004C6F616475
:1003C0002053657474696E677300426564205472CB
:1003D000616D6D696E670050726F6265205A204FC3
:1003E0006666736574004661646520486569676880
:1003F00074004F6666004F6E00426564204C65765F
:10040000656C696E67004C6576656C2042656400BA
:100410004732394E00473239004175746F20486FBA
:100420006D65004D6F74696F6E0053572D4D6F648D
:10043000650053746F77004465706C6F7900536585
:100440006C662D5465737400526573657400436F58
:100450006E66696775726174696F6E005265737458
:100460006F72652044656661756C7473004C6F61D2
:10047000642053657474696E67730053746F72659A
:100480002053657474696E6773004F6666004F6E23
:100490000052756E6F75742053656E736F720042F3
:1004A0004C546F7563680050726F6265205A204F1C
:1004B000666673657400416476616E63656420539B
:1004C000657474696E6773004D61696E003F004228
:1004D00061636B0053746F70004D3232004174746D
:1004E000616368204D65646961004D32310050726E
:1004F000696E742066726F6D204D6564696100528B
:10050000656C65617365204D6564696100436F6E5C
:1005100066696775726174696F6E0054656D7065A8
:10052000726174757265004D6F74696F6E0052650B
:1005300073756D65205072696E740054756E650038
:1005400053746F70205072696E74005061757365DA
:10055000205072696E7400496E666F205363726535
:10056000656E000A4D3234004D3233202573003F52
:10057000005374617274205072696E740043616E2E
:1005800063656C005072696E740043616E6E6F74C7
:1005900020656E746572207375626469723A20001A
:1005A00002202E2E000152656672657368004D614F
:1005B000696E002100486F74656E6420746F6F204F
:1005C000636F6C64004261636B0050726F636565BA
:1005D00064004D6F74696F6E0044697361626C658D
:1005E000205374657070657273004D383400426535
:1005F00064204C6576656C696E67004175746F2088
:10060000486F6D6500473238004D61696E00507269
:1006100065686561742024204265640050726568D5
:10062000656174202420456E640054656D706572A8
:10063000617475726500C601C101436F6F6C646FB0
:10064000776E005072656865617420240046616EA3
:1006500020537065656400426564004E6F7A7A6C61
:1006600065004D61696E0050726F6265205A204FBF
:10067000666673657400466C6F770046616E205342
:100680007065656400426564004E6F7A7A6C65003F
:100690005370656564004D61696E00486F6D696EE9
:1006A00067204661696C6564006F70656E00545226
:1006B00049474745524544003A200066696C616DE0
:1006C000656E74007A5F6D696E00795F6D696E00AA
:1006D000785F6D696E005265706F7274696E672025
:1006E000656E6473746F70207374617475730A003F
:1006F00020746F6F206C6F6E6720657874727573ED
:10070000696F6E2070726576656E7465640A00208C
:10071000636F6C6420657874727573696F6E207096
:10072000726576656E7465640A00486F6D65202594
:100730007325732573204669727374005761726E56
:10074000696E673A20486F6D696E672042756D70FB
:100750002044697669736F72203C20310A000202DE
:10076000040000E0C0000000C000000000000068BD
:10077000430000634300007A430000A0400000A053
:100780004000000040FFFDFCFAF8F6F4F2F0EEEC59
:10079000EAE9E7E5E3E1E0DEDCDAD9D7D5D4D2D087
:1007A000CFCDCBCAC8C7C5C3C2C0BFBDBCBAB9B71D
:1007B000B6B4B3B2B0AFADACAAA9A8A6A5A4A2A185
:1007C000A09E9D9C9A99989795949392908F8E8DC8
:1007D0008B8A8988878684838281807F7E7D7B7AED
:1007E000797877767574737271706F6E6D6C6B6AF1
:1007F000696867666564636261605F5E5D5C5B5AE1
:100800005958585756555453525150504F4E4D4CBD
:100810004B4A4A4948474646454443424241403F85
:100820003E3E3D3C3B3B3A3938383736353534333C
:1008300032323130302F2E2E2D2C2B2B2A292928E5
:10084000272726252524232322212120201F1E1E81
:100850001D1C1C1B1B1A1919181817161615151410
:10086000131312121111100F0F0E0E0D0D0C0C0B95
:100870000A0A090908080707060605050404030310
:1008800002020100000000000100000001000080E1
:1008900000555555000000400033333300AAAA2A02
:1008A000004992240000002000C7711C009999198A
:1008B00000D1451700555515003BB11300244912CE
:1008C0000011111100000010000F0F0F00E3380E8F
:1008D0000043790D00CCCC0C00C3300C00E8A20B17
:1008E0000064210B00AAAA0A00703D0A009DD809E5
:1008F00000427B090092240900DCD30800888808A4
:10090000001042080000000800F0C10700878707B8
:100910000075500700711C07003EEB0600A1BC06E5
:10092000006990060066660600703E0600611806C3
:100930000017F4050074D105005BB00500B2900506
:1009400000627205005555050078390500B81E058E
:1009500000050505004EEC040087D40400A1BD0489
:100960000090A7040049920400C17D0400EE6904D0
:1009700000C7560400444404005C3204000821040B
:100980000041100400000004003FF00300F8E00301
:100990000026D20300C3C30300CCB503003AA8036A
:1009A000000A9B0300388E0300C08103009F75037B
:1009B00000D0690300505E03001D53030034480358
:1009C00000913D03003333030016290300381F0351
:1009D0000097150300300C0300030303000BFA0219
:1009E0000049F10200BAE802005CE002002DD802E2
:1009F000002DD0020059C80200B0C0020031B90277
:100A000000DAB10200AAAA0200A0A30200BC9C0264
:100A100000FA9502005C8F0200DF880200828202E9
:100A200000457C02002776020027700200436A021C
:100A3000007C640200D05E02003F590200C85302ED
:100A400000000061430000614300007A430000E0C1
:100A5000C0000000C00000000053657474696E6738
:100A6000732053746F726564000000FA430000FA4B
:100A7000430000A0400000C8410000A0420000A0C8
:100A8000420000C8430080C043F4010000F40100AC
:100A900000640000008813000024F4D43050C38E9A
:100AA00020C2A24017828B7011127A910D816CD9ED
:100AB0000AA861E108C7586607615143061E4B5DED
:100AC00005C145A7041A411104093D980371393144
:100AD000034036DB0265339102D4305402802E1D70
:100AE00002632CEE01752AC501B028A001102781F0
:100AF000018F2564012B244B01E0223401AC211F1E
:100B0000018D200D01801FFC00841EED00971DDF6C
:100B100000B81CD200E61BC600201BBC00641AB241
:100B200000B219A8000A19A0006A189900D11791FB
:100B30000040178B00B516840031167E00B315797E
:100B4000003A157300C7146F0058146A00EE13665C
:100B5000008813630025135E00C7125B006C1257F8
:100B60000015125400C111510070114F0021114B9A
:100B700000D61049008D1047004610440002104274
:100B800000C00F4000800F3E00420F3C00060F3BAC
:100B900000CB0E3800930E37005C0E3500270E3464
:100BA00000F30D3200C10D3100900D3000600D2EAC
:100BB00000320D2D00050D2C00D90C2B00AE0C2998
:100BC00000850C29005C0C2700350C27000E0C2634
:100BD00000E80B2400C40B2400A00B23007D0B2392
:100BE000005A0B2100390B2100180B2000F80A1FB6
:100BF00000D90A1E00BB0A1E009D0A1D00800A1DA6
:100C000000630A1C00470A1B002C0A1B00110A1A69
:100C100000F7091A00DD091900C4091900AB091908
:100C200000920917007B091800630917004C091688
:100C30000036091600200916000A091500F50815E6
:100C400000E0081400CC081400B8081400A408142C
:100C500000900813007D0812006B0813005808125A
:100C60000046081200340811002308110012081170
:100C70000001081100F0071000E0071000D0071075
:100C800000C0071000B0070F00A107100091070E69
:100C90000083070F0074070F0065070E0057070E4B
:100CA0000049070E003B070D002E070E0020070D20
:100CB0000013070D0006070D00F9060C00ED060DE8
:100CC00000E0060C00D4060C00C8060C00BC060CA4
:100CD00000B0060C00A4060B0099060C008D060B54
:100CE0000082060B0077060B006C060B0061060AFB
:100CF0000057060B004C060A0042060A0038060A96
:100D0000002E060A0024060A001A060A0010060928
:100D10000007060A00FD050900F4050900EB0509B6
:100D200000E2050900D9050900D0050900C7050939
:100D300000BE050900B5050800AD050800A50509B8
:100D4000009C050800940508008C0508008405082F
:100D5000007C050800740508006C0507006505089F
:100D6000005D050700560508004E0507004705070A
:100D7000004005080038050700310507002A05076F
:100D800000230507001C050600160507000F0507D0
:100D9000000805060002050700FB040600F504072D
:100DA00000EE040600E8040600E2040700DB040687
:100DB00000D5040600CF040600C9040600C30406DB
:100DC00000BD040600B7040600B1040500AC04062B
:100DD00000A6040600A00405009B04060095040577
:100DE00000900406008A04050085040500800406BE
:100DF000007A04050075040500700405006B040505
:100E00000066040500610405005C04050057040544
:100E100000520405004D0405004804050043040584
:100E2000003E0404003A04050035040500300404C3
:100E3000002C04050027040400230405001E0404FC
:100E4000001A04040016040500110404000D040433
:100E500000090405000404040000040400FC030469
:100E600000F8030400F4030400F0030400EC03049E
:100E700000E8030400E4030400E0030400DC0304CE
:100E800000D8030400D4030400D0030400CC0304FE
:100E900000C8030300C503030024F404D9201BC4C5
:100EA0000C5C0E9804C4095F0265077101F405F932
:100EB00000FB04B30048048700C1036900580355D0
:100EC0000003034500BE023A008402310053022AA7
:100ED000002902250004022000E4011C00C80119B9
:100EE00000AF011700980114008401130071011074
:100EF000006101100051010E0043010D0036010B8D
:100F0000002B010B0020010B00150109000C010949
:100F10000003010800FB000800F3000800EB0007D5
:100F200000E4000600DE000600D8000600D200063D
:100F300000CC000500C7000500C2000500BD00048C
:100F400000B9000400B5000400B1000400AD0004C5
:100F500000A9000400A5000300A20003009F0004F4
:100F6000009B00030098000300950002009300031B
:100F700000900003008D0002008B00030088000237
:100F8000008600020084000300810002007F00024E
:100F9000007D0002007B0002007900020077000162
:100FA000007600020074000200720001007100026D
:100FB000006F0002006D0001006C0002006A000179
:100FC0000069000200670001006600010065000181
:100FD0000064000200620001006100010060000185
:100FE000005F0002005D0001005C0001005B000189
:100FF000005A00010059000100580001005700018B
:10100000005600010055000100540001005300008B
:101010000053000100520001005100010050000186
:10102000004F0001004E0000004E0001004D000185
:10103000004C0001004B0000004B0001004A000181
:10104000004900010048000000480001004700017D
:101050000046000000460001004500000045000178
:101060000044000100430000004300010042000072
:101070000042000100410000004100010040000169
:10108000003F0000003F0001003E0000003E000164
:10109000003D0000003D0001003C0000003C00005D
:1010A000003C0001003B0000003B0001003A000052
:1010B000003A00010039000000390001003800004A
:1010C0000038000000380001003700000037000140
:1010D0000036000000360000003600010035000038
:1010E000003500000035000100340000003400002D
:1010F0000034000100330000003300000033000121
:101100000032000000320000003200010031000017
:10111000003100000031000100300000003000000C
:1011200000300001002F0000002F0000002F000001
:10113000002F0001002E0000002E0000002E0001F4
:10114000002D0000002D0000002D0000002D0001EA
:10115000002C0000002C0000002C0000002C0001DE
:10116000002B0000002B0000002B0000002B0001D2
:10117000002A0000002A0000002A0000002A0001C6
:1011800000290000002900000029000000290000BB
:1011900000290001002800000028000000280000AD
:1011A00000280000002800010027000000270000A0
:1011B0000027000000270000002700010026000093
:1011C0000026000000260000002600000026000186
:1011D000002500000025000000250000002500007B
:1011E000002500000025000100240000002400006C
:1011F000002400000024000000240001002300005F
:101200000023000000230000002300000023000052
:101210000023000000230001002200000022000043
:101220000022000000220000002200000022000135
:10123000002100000021000000210000002100002A
:10124000002100000021000000210001002000001A
:10125000002000000020000000200000002000000E
:10126000002000000020000000200001001F0000FE
:10127000001F0000001F0000001F0000001F0000F2
:10128000001F0000001F0001001E0000001E0000E3
:10129000001E0000001E0000003930000033250051
:1012A0000087190000B00F0000DB080000BD04003B
:1012B00000740200003F01000020436F756E74202F
:1012C000583A00426564004531004500626564009B
:1012D0002C2073797374656D2073746F70706564FE
:1012E00021204865617465725F49443A2000457267
:1012F000723A204D415854454D50004D4158544587
:101300004D50207472696767657265640048656155
:1013100074696E67204661696C6564004865617434
:10132000696E67206661696C6564004572723A2077
:101330004D494E54454D50004D494E54454D502059
:1013400074726967676572656400544845524D411F
:101350004C2052554E4157415900546865726D6199
:101360006C2052756E6177617900202F0020424019
:101370003A0020403A007C3C3E5E2B3D3F2F5B5DB7
:101380003B2C2A225C00434F4D4D554E494341545E
:10139000494F4E0044525952554E004552524F52F9
:1013A0005300494E464F004543484F0053544F5059
:1013B0005045442E20005072696E7465722073741B
:1013C0006F707065642064756520746F206572723B
:1013D0006F72732E2046697820746865206572727A
:1013E0006F7220616E6420757365204D3939392024
:1013F000746F20726573746172742E202854656D49
:1014000070657261747572652069732072657365A9
:10141000742E20536574206974206166746572208F
:1014200072657374617274696E67290A004E6F2069
:10143000436865636B73756D2077697468206C69A8
:101440006E65206E756D6265722C204C6173742020
:101450004C696E653A20004E6F20436865636B737C
:10146000756D2077697468206C696E65206E756D86
:101470006265722C204C617374204C696E653A2051
:1014800000636865636B73756D206D69736D61745E
:1014900063682C204C617374204C696E653A20009F
:1014A0004C696E65204E756D626572206973206EA1
:1014B0006F74204C617374204C696E65204E756D9D
:1014C0006265722B312C204C617374204C696E65FF
:1014D0003A20004D3131300053657269616C2073E0
:1014E0007461747573206D69736D617463680A004B
:1014F00053442072656164206572726F720A002124
:1015000021204B494C4C20636175736564206279DE
:1015100020746F6F206D75636820696E61637469F4
:1015200076652074696D65202D2063757272656E15
:101530007420636F6D6D616E643A20004D3235002A
:101540004D6564696120496E7365727465640062FB
:101550007573793A2070617573656420666F7220C7
:10156000696E7075740A00627573793A20706175DE
:1015700073656420666F7220757365720A00627508
:1015800073793A2070726F63657373696E670A00CE
:10159000506C6561736520526573657400505249E3
:1015A0004E5445522048414C5445440025533A205E
:1015B0002553004B494C4C45442E20005072696E17
:1015C0007465722068616C7465642E206B696C6C44
:1015D00028292063616C6C6564210A0053544F50C4
:1015E0005045442E20005072696E746572207374E9
:1015F0006F707065642064756520746F2065727209
:101600006F72732E20466978207468652065727247
:101610006F7220616E6420757365204D39393920F1
:10162000746F20726573746172742E202854656D16
:101630007065726174757265206973207265736577
:10164000742E20536574206974206166746572205D
:1016500072657374617274696E67290A00656368E4
:101660006F3A004572726F723A0042696C696E653A
:101670006172204C6576656C696E6720477269649B
:101680003A0A0021212053544F502063616C6C654D
:10169000642062656361757365206F6620424C54F7
:1016A0006F756368206572726F72202D207265738A
:1016B000746172742077697468204D3939390A0071
:1016C00021212053544F502063616C6C656420626B
:1016D000656361757365206F6620424C546F756356
:1016E00068206572726F72202D207265737461724A
:1016F000742077697468204D3939390A004F46469D
:101700000A00466164652048656967687420004284
:101710006564204C6576656C696E6720004661697A
:101720006C656420746F20656E61626C6520426533
:1017300064204C6576656C696E670A00496E766157
:101740006C6964206D6573682E0A0050726F62695F
:101750006E6720506F696E740025532025692F2510
:1017600069002E0A002F0050726F62696E67206D4B
:1017700065736820706F696E742000202844525988
:1017800052554E2900473239204175746F20426509
:1017900064204C6576656C696E67003F20284C2C90
:1017A000522C462C4229206F7574206F6620626F80
:1017B000756E64732E0A003F2856296572626F7336
:1017C00065206C6576656C20696D706C61757369F8
:1017D000626C652028302D34292E0A004261642075
:1017E0005A2076616C75650A004E6F2062696C69DB
:1017F0006E65617220677269640A004732384C3046
:101800000020204D3230312058004D617820416356
:1018100063656C65726174696F6E2028756E69749A
:10182000732F7332290020204D3230332058004D61
:101830006178206665656472617465732028756ED1
:101840006974732F73290020520020204D323034E8
:10185000205000416363656C65726174696F6E202E
:1018600028756E6974732F7332292028503C70726A
:10187000696E742D616363656C3E20523C726574C1
:10188000726163742D616363656C3E20543C7472B5
:101890006176656C2D616363656C3E2900204A00AA
:1018A00020540020530020204D323035204200418A
:1018B0006476616E6365642028423C6D696E5F7377
:1018C00065676D656E745F74696D655F75733E20E5
:1018D000533C6D696E5F66656564726174653E2038
:1018E000543C6D696E5F74726176656C5F666565A8
:1018F00064726174653E204A3C6A756E635F64651C
:10190000763E290020440020490020204D3330310C
:10191000205000486F74656E642050494400204494
:101920000020490020204D333034205000426564AF
:1019300020504944002E0A00206E6F7420646973A1
:1019400061626C65642E20536861726564207769FA
:10195000746800203B204C6576656C696E672000DA
:1019600020204D3432302053004175746F20426581
:1019700064204C6576656C696E67002046002042E5
:101980000020480020204D3134352053004D617433
:10199000657269616C206865617475702070617230
:1019A000616D657465727300203B2053656E736FC3
:1019B00072200020440020204D3431322053004654
:1019C000696C616D656E742072756E6F75742073CD
:1019D000656E736F7200204A00202047323920570D
:1019E00020490020204D3134392043203B20556EC2
:1019F00069747320696E2043656C736975730A009E
:101A000054656D706572617475726520556E697488
:101A100073002020473231203B004C696E656172B3
:101A200020556E6974730020496E76616C6964207C
:101A300065787472756465722000536C6565702EEC
:101A40002E2E005A2050726F6265205061737420F0
:101A50004265640A005A2050726F626520506173BB
:101A6000742042656400205A3A200020593A200030
:101A700042656420583A20004D65736820706F6994
:101A80006E74206F7574206F662072616E67650AD0
:101A900000436C69636B20746F20526573756D65CC
:101AA0002E2E2E00616C736F20656E61626C656412
:101AB000290A004E6F204D6F76652E004E6F206D07
:101AC000656469610A00456E642066696C65206C16
:101AD0006973740A00426567696E2066696C6520E7
:101AE0006C6973740A00286E6F2066696C65290042
:101AF0004E6F74205344207072696E74696E670A69
:101B0000005344207072696E74696E672062797444
:101B100065200043757272656E742066696C653A63
:101B200020002E0A0044656C6574696F6E20666142
:101B3000696C65642C2046696C653A200046696CC6
:101B4000652064656C657465643A002569730025D9
:101B5000696D20256973002569682025696D202538
:101B6000697300256964202569682025696D202531
:101B70006973002569792025696420256968202515
:101B8000696D20256973005072696E742074696DE7
:101B9000653A20006F6B006F666600A713A2139B67
:101BA000139413861344454255473A004D31313260
:101BB0002053687574646F776E004D313133205354
:101BC000004D656761205A65726F20322E30204FBC
:101BD00046462E00434F4E4649475F4558504F52A8
:101BE00054004D4541545041434B00434F4F4C45E9
:101BF000525F54454D50455241545552450043485B
:101C0000414D4245525F54454D5045524154555205
:101C10004500424142595354455050494E470041B6
:101C2000524353004D4F54494F4E5F4D4F4445531F
:101C300000544845524D414C5F50524F5445435417
:101C4000494F4E00455854454E4445445F4D32304F
:101C5000004C4F4E475F46494C454E414D45004173
:101C600055544F5245504F52545F53445F53544163
:101C70005455530053445F57524954450052455000
:101C8000454154005344434152440050524F4D503B
:101C9000545F535550504F525400484F53545F4176
:101CA0004354494F4E5F434F4D4D414E44530045C1
:101CB0004D455247454E43595F504152534552009E
:101CC000434153455F4C494748545F425249474856
:101CD000544E45535300544F47474C455F4C49477A
:101CE00048545300534F4654574152455F504F5745
:101CF0004552004255494C445F50455243454E546D
:101D0000004C4556454C494E475F44415441005AAA
:101D10005F50524F42450052554E4F555400415569
:101D2000544F4C4556454C005052494E545F4A4F13
:101D3000420050524F4752455353004155544F5261
:101D400045504F52545F54454D50004155544F52E9
:101D500045504F52545F504F5300564F4C554D45D0
:101D60005452494300454550524F4D0042494E415F
:101D700052595F46494C455F5452414E5346455275
:101D80000053455249414C5F584F4E5F584F4646AD
:101D9000004649524D574152455F4E414D453A4DDF
:101DA00061726C696E20322E302E392E332D6B61AC
:101DB00064312028446563203237203230323120AC
:101DC00031333A34353A30342920534F5552434554
:101DD0005F434F44455F55524C3A6769746875627A
:101DE0002E636F6D2F6B61642F4D61726C696E2075
:101DF00050524F544F434F4C5F56455253494F4EEC
:101E00003A312E30204D414348494E455F54595098
:101E1000453A4D656761205A65726F20322E302039
:101E200045585452554445525F434F554E543A31EC
:101E300020555549443A64626663636435352D65BF
:101E40006262612D343631352D616264372D31394E
:101E5000366161343338663330340A002F2F004D39
:101E600031343520533C696E6465783E206F75745B
:101E7000206F662072616E67652028302D31290A37
:101E8000003F4A206F7574206F662072616E67652F
:101E90002028302E303120746F20302E33290A0054
:101EA00020580020204D61783A2000200020204D4D
:101EB000696E3A2000203B200020204D3231312035
:101EC000530046523A0020466C6F773A2000206F4C
:101ED0007574206F662072616E67650A00536572C3
:101EE000766F20003A200020536572766F200050F4
:101EF000726F6265204F6666736574205A00507277
:101F00006F6265204F6666736574205A006469735A
:101F100000656E0043290A0061626C656420286DCB
:101F2000696E2074656D702000436F6C6420657865
:101F30007472756465732061726520004F464600B7
:101F40004F4E006D6D00203B2044697374616E63D9
:101F500065200046696C616D656E742072756E6FE8
:101F6000757420004D34323120696E636F72726572
:101F7000637420706172616D657465722075736140
:101F800067650A004D65736820706F696E74206F15
:101F90007574206F662072616E67650A0045455052
:101FA000524F4D204F4B0A00290A0020746F200029
:101FB0003F5A206F7574206F662072616E676520CE
:101FC0002800290A0020746F20003F59206F757483
:101FD000206F662072616E676520282D00290A0037
:101FE00020746F20003F58206F7574206F66207238
:101FF000616E676520282D004D383400446F6E6592
:10200000207072696E74696E672066696C650A007B
:102010004D3737004D333100496E76616C6964206D
:1020200065787472756465720A004361703A0020C5
:10203000286D6D2900203B0020204D383531205877
:10204000005A2D50726F6265204F6666736574008A
:10205000436F6F6C696E672E2E2E00486561746940
:102060006E672E2E2E0045312025530020573A0052
:1020700020573A0042656420436F6F6C696E672E8B
:102080002E2E004265642048656174696E672E2EAD
:102090002E0023646566696E652044454641554CB3
:1020A000545F00626564004B6420004B6920004B64
:1020B000702000504944204175746F74756E65201E
:1020C00066696E6973686564212050757420746850
:1020D00065206C617374204B702C204B6920616EFD
:1020E00064204B6420636F6E7374616E747320663A
:1020F000726F6D2062656C6F7720696E746F20431C
:102100006F6E66696775726174696F6E2E680A001A
:10211000504944204175746F74756E65206661691D
:102120006C6564212074696D656F75740A0050498F
:1021300044204175746F74756E65206661696C65C5
:1021400064212054656D70657261747572652074C8
:102150006F6F20686967680A0050494420437963BB
:102160006C65730025532025692F256900204B6479
:102170003A2000204B693A2000204B703A20002082
:10218000436C617373696320504944200A00204EF8
:102190006F206F76657273686F6F740A00205475D4
:1021A0003A2000204B753A2000206D61783A2000DB
:1021B000206D696E3A200020643A20002062696137
:1021C000733A20005761697420666F7220686561F8
:1021D000742075702E2E2E00504944204175746F66
:1021E00074756E652073746172740A0050494420DE
:1021F0004175746F74756E65206661696C656421E4
:102200002054656D706572617475726520746F6FAE
:1022100020686967680A00504944204175746F74EA
:10222000756E6500504944204175746F74756E6514
:10223000206661696C656421204261642068656183
:102240007465722069640A004572723A207574667A
:102250003820666F6E74206E6F7420696E697469C1
:10226000616C697A65642E004572723A20757466F5
:102270003820666F6E74206E6F7420696E697469A1
:10228000616C697A65642E004572723A20757466D5
:102290003820666F6E74206E6F7420696E69746981
:1022A000616C697A65642E0042656400456E636CFA
:1022B0006F73757265002568753A25303268750050
:1022C00025303268753A253032687500253032681D
:1022D000752725303268750020202020202020001E
:1022E0002020202000657272001FE02010201020A6
:1022F00010102010202010201030300840048003DF
:10230000001FE03FF03FF03FF01FE01FE03FF03FD5
:10231000F03FF00FC0078003003FFFF0380070303F
:10232000FC3020FC102078102030102C00D02E31F2
:10233000D02F7BD02F7BD02E31D02C00D02030104E
:1023400020781020FC1030FC303800703FFFF03F48
:10235000FFF03800703186302387102787902F8751
:10236000D02F03D02030102078102078102030108B
:102370002F03D02F87D027879023871031863038BE
:1023800000703FFFF01FFFF81FFFF8041040020825
:102390002002082004104008208010410010410055
:1023A0000820800410400000001FFFF81FFFF80005
:1023B0001DC43F0000000C86198000000D0E19801E
:1023C00000000F0B198000000D9F198000000DD335
:1023D000998000001CFBFF000000000000000000CE
:1023E0000000000000F380001F80007700001980CB
:1023F000005B1CF6131DAE5B35AB0635FB5B3DA7E2
:102400000CBD9B4B30EB19B19BE39D8E9F9D8E00C5
:1024100001E00000000001200000000001E00000D9
:1024200000000C0F00FE07022503BB017FFE08FE23
:1024300008FE05080806000040F0C8888898781053
:10244000050808060000C0F88888888888F805050F
:10245000050600012030F83020050808060000209D
:1024600070F820202020E00509090600FF2070A850
:10247000A8B888887020070505070001D86C366C5D
:10248000D80509090600FFF8A88888888888A8F870
:10249000050A0A0600FE205050505088A8A88870EF
:1024A00003030306000340A040FFFFFFFFFFFFFF01
:1024B000FFFFFFFFFFFFFFFFFFFFFFFFFFFFFF002B
:1024C00000000605FF01070706020080808080806B
:1024D0000080030303060105A0A0A0050606060070
:1024E0000050F85050F8500509090600FF2070A868
:1024F000A07028A87020050707060000C8C8102093
:1025000040989805070706000040A0A040A89068E2
:102510000103030602058080800309090601FF20EC
:1025200040408080804040200309090601FF804030
:102530004020202040408005070706000020A870AA
:102540002070A8200505050600012020F8202002A3
:1025500003030601FFC04080050101060003F802E5
:102560000202060100C0C00507070600000810109F
:1025700020404080050707060000708898A8C8889A
:102580007003070706010040C040404040E00507D7
:1025900007060000708808102040F80507070600AD
:1025A00000F8081030088870050707060000103092
:1025B0005090F81010050707060000F880F0080892
:1025C0008870050707060000304080F08888700595
:1025D0000707060000F8081010202020050707064E
:1025E00000007088887088887005070706000070F2
:1025F000888878081060020505060100C0C000C088
:10260000C00206060601FFC0C000C04080030505E9
:102610000601012040804020050303060002F80067
:10262000F8030505060101804020408005070706E4
:1026300000007088102020002005070706000070A9
:1026400088B8A8B88070050707060000708888F869
:10265000888888050707060000F04848704848F059
:1026600005070706000070888080808870050707CE
:10267000060000F04848484848F0050707060000F3
:10268000F88080F08080F8050707060000F8808059
:10269000F080808005070706000070888080988899
:1026A00070050707060000888888F888888803076F
:1026B00007060100E04040404040E00507070600F3
:1026C0000038101010109060050707060000889071
:1026D000A0C0A09088050707060000808080808049
:1026E00080F805070706000088D8A888888888052C
:1026F00007070600008888C8A89888880507070685
:10270000000070888888888870050707060000F038
:102710008888F08080800507070600007088888818
:10272000A89068050707060000F08888F0A0908848
:102730000507070600007088807008887005070785
:10274000060000F8202020202020050707060000B2
:102750008888888888887005070706000088888828
:102760008850502005070706000088888888A8A898
:102770005005070706000088885020508888050704
:102780000706000088885020202020050707060043
:1027900000F80810204080F80309090601FFE080D6
:1027A000808080808080E005070706000080404030
:1027B000201010080309090601FFE0202020202036
:1027C0002020E005030306000520508805010106CE
:1027D00000FEF803030306010580402005050506F9
:1027E000000070087888780507070600008080F0F0
:1027F000888888F0050505060000708080887005CF
:102800000707060000080878888888780505050607
:1028100000007088F080700507070600003048400F
:10282000E04040400507070600FE70888888780869
:10283000700507070600008080F0888888880307F5
:10284000070601004000C0404040E00409090601BD
:10285000FE100030101010109060050707060000F1
:1028600080808890E09088030707060100C0404000
:10287000404040E0050505060000D0A8A8A8A8052E
:102880000505060000B0C888888805050506000013
:1028900070888888700507070600FEF0888888F031
:1028A00080800507070600FE788888887808080574
:1028B0000505060000B0C8808080050505060000FB
:1028C00078807008F00507070600002020F8202017
:1028D0002018050505060000888888986805050504
:1028E00006000088888850200505050600008888B5
:1028F000A8A8500505050600008850205088050747
:10290000070600FE888888502040800505050600DF
:1029100000F8102040F80309090601FF204040405C
:1029200080404040200109090602FF8080808080AD
:10293000808080800309090601FF804040402040DC
:1029400040408005030306000248A890FF43616EE3
:102950006E6F74206F70656E20737562646972208B
:102960000053442063617264206F6B0A006F7065CE
:102970006E526F6F74206661696C65640A00766FD1
:102980006C756D652E696E6974206661696C65642D
:102990000A004E6F20534420636172640A002E0ABD
:1029A000006F70656E206661696C65642C204669F5
:1029B0006C653A200046696C652073656C656374CC
:1029C00065640A002053697A653A200046696C659F
:1029D000206F70656E65643A2000454E4420535563
:1029E00042524F5554494E450A002220706F7300E1
:1029F0002220706172656E743A2200535542524F24
:102A00005554494E452043414C4C207461726765D2
:102A1000743A220053756263616C6C204F76657264
:102A2000666C6F77004578636565646564206D61E9
:102A30007820535542524F5554494E452064657095
:102A400074683A00667265736800646F696E670047
:102A50002066696C653A20004E6F772000577269D6
:102A600074696E6720746F2066696C653A20006D2A
:102A700061726C696E66772E6F726700322E302E2F
:102A8000392E332D6B616431001FFFFFFFFFFFFF05
:102A9000600000000001FF400000000000FF800017
:102AA000000000007F83CF00000C303F87FF8000D4
:102AB0000C301F867980000C000F8C30C7838C305F
:102AC000E78C30CFC7CC31F38C30DCECEC33B98CF5
:102AD00030D86C6C33198C30D06C0C33198C30D8E6
:102AE0006C0C33198C30DC6C0E3B198C30CF7C07AE
:102AF0009F198C30C77C038F194000000000000232
:102B0000600000000000061FFFFFFFFFFFF87001DC
:102B10002C0190012701B0012201C0011D01F0012B
:102B200018011002130130020E0160020901900227
:102B30000401C002FF000003FA004003F500800317
:102B4000F000D003EB002004E6007004E100E00494
:102B5000DC004005D700C005D2004006CD00D006FD
:102B6000C8008007C3003008BE00F008B900C009E3
:102B7000B400B00AAF00B00BAA00D00CA500000E44
:102B8000A000500F9B00C01096005012910000143E
:102B90008C00C0158700B0178200B0197D00D01BD3
:102BA0007800001E730040206E0090226900F0241F
:102BB000640040275F0090295A00E02B5500102E3A
:102BC000500020304B0010324600E0334100903579
:102BD0003C001037370070383200A0392D00B03A71
:102BE0002800A03B2300603C1E00103D1900903DD2
:102BF0001400103E0F00703E0A00C03E0500003F6A
:102C00000000403FFBFF803FF6FFC03FF1FF202068
:102C1000506C616E6E65724275666665724279745B
:102C200065733A20002046726565204D656D6F72B0
:102C3000793A200020436F6D70696C65643A2044D6
:102C4000656320323720323032310A00204C617304
:102C50007420557064617465643A20323032312DCD
:102C600030392D3033207C20417574686F723A20E2
:102C7000286B61642C20416E796375626963204D15
:102C8000656761205A65726F20322E302041424CB8
:102C900020323456290A004D61726C696E20322E42
:102CA000302E392E332D6B6164310A0020536F664C
:102CB00074776172652052657365740A00205761EC
:102CC000746368646F672052657365740A002042FC
:102CD000726F776E206F75742052657365740A0089
:102CE0002045787465726E616C2052657365740A54
:102CF00000506F77657255700A0073746172740AC0
:102D0000004732385859004D313030310065727209
:102D10006F722077726974696E6720746F206669BC
:102D20006C650A00446F6E6520736176696E67207A
:102D300066696C652E0A004D323900456E64737405
:102D40006F707300255320256320256320256320A1
:102D5000256300205A3A0020593A0020583A00656D
:102D60006E6473746F7073206869743A2000000099
:102D700000010200090A0000000004030807000027
:102D80000000000000000000000000000000004DF6
:102D90006F76652025736D6D004D6F766520302E42
:102DA000316D6D004D6F766520316D6D004D6F7624
:102DB000652031306D6D004D6F7665204178697307
:102DC000004D6F7665204578747275646572004DAC
:102DD0006F7665205A004D6F76652059004D6F76ED
:102DE000652058005072696E742066726F6D204DB8
:102DF0006564696100FFFFFF205A3A200020593ABC
:102E0000200042656420583A20004D656761205AD1
:102E100065726F20322E302052656164792E005029
:102E200072696E74696E672E2E2E005072696E7410
:102E30002050617573656400204500205A002059B8
:102E40000020204D39322058005374657073207073
:102E5000657220756E6974003B2000220A00556E71
:102E60006B6E6F776E20636F6D6D616E643A2022BA
:102E7000006F6B00DB0FC93F45BCDA3F8FB30240E8
:102E8000FCF0274056946140FE4B9B4084A5D840FF
:102E9000E0231841346A5641E859974164DBD54133
:102EA0006E271742B4B75542CE1A9742C8AED542E4
:102EB000B5885A43D40684BFA65FA7BF7443E0BF5A
:102EC00010B11AC01C2C58C0E8F697C0B849D6C03B
:102ED0004E4E17C124D355C1802497C1A0B5D5C18A
:102EE000121A17C244AE55C2781797C26CACD5C23D
:102EF00067885AC320746F6F206C6F6E6720657887
:102F000074727573696F6E2070726576656E746524
:102F1000640A0020636F6C6420657874727573694D
:102F20006F6E2070726576656E7465640A006F6BF3
:102F30000A00526573656E643A200020453A00200D
:102F40005A3A0020593A00583A0000002200250061
:102F500028002B0000002100240027002A00020284
:102F6000020202020202040404040404040403032F
:102F70000303030303030101010101010101010234
:102F80000408102040800102040810204080010243
:102F9000040810204080804020100804020145727F
:102FA000726F722077726974696E6720746F204542
:102FB0004550524F4D210A0043DF4FE611241FBEFA
:102FC000CFEFD0E4DEBFCDBF84B78093851514BEAC
:102FD0000FB6F894A8958091600088618093600096
:102FE000109260000FBE12E0A0E0B1E0ECECF8EE51
:102FF00001E00BBF02C007900D92A839B107D9F7C5
:1030000025E1A8E9B2E001C01D92A538B207E1F7B9
:1030100017E1CDEDD7E104C02197FE010E94B4F184
:10302000CC3DD107C9F70E9409E00C945AF40C94E6
:103030000000A0E1B0E0EFE1F8E10C94DDF18C01DB
:10304000DC01ED91FC910280F381E02DBE016F5F08
:103050007F4F0995882309F45DC08981807C91F5B3
:103060006F81637070E0762F6627770F770F888502
:10307000B4E08B9FC0011124682B792B8985829540
:10308000869586958370682B6F5F7F4F90E080E018
:103090002A852370220F3B8537FB332730F9232BFA
:1030A0003E813F70230F3327331F2750310904C05F
:1030B000660F771F881F991F2A95D2F76096E4E064
:1030C0000C94F9F1803419F568856695669570E081
:1030D00090E080E0CB01772766272A85622B09855F
:1030E00010E0102F0027012E000C220B330B602B59
:1030F000712B822B932B6F5F7F4F8F4F9F4F4AE037
:10310000660F771F881F991F4A95D1F7D7CF8BE09D
:10311000F801848360E070E0CB01D0CF0895FC011A
:10312000828108954F925F926F927F928F929F92C9
:10313000AF92BF92CF92DF92EF92FF92CF93DF9345
:10314000CDB7DEB728970FB6F894DEBF0FBECDBF60
:1031500060913F07709140076115710511F18091F1
:103160003B0790913C07A0913D07B0913E078983B2
:103170009A83AB83BC83072E000C880B990B0E94AB
:10318000EFEA29813A814B815C810E9406F24B0172
:103190005C0120E030E040E251EC0E94E9EA87FF68
:1031A00007C081E080933701C12CD12C760113C078
:1031B00020E030E040E251E4C501B4010E946AF32E
:1031C000181604F581E080933701C12CD12C9FE7BC
:1031D000E92E93E4F92EC701B60128960FB6F894AC
:1031E000DEBF0FBECDBFDF91CF91FF90EF90DF909C
:1031F000CF90BF90AF909F908F907F906F905F9097
:103200004F9008958091460790914707A0914807F5
:10321000B09149078D839E83AF83B8878091370132
:10322000882391F01092A0041092A1041092A2049D
:103230001092A30410929C0410929D0410929E047C
:1032400010929F04109237012091A0043091A104A4
:103250004091A2045091A304C501B4010E9407F259
:103260002B013C0120E030E0A9010E946AF3C12C4F
:10327000D12C760187FD14C02D813E814F81588568
:1032800060E070E08FE793E40E947EF26B017C01C6
:10329000A30192010E94E9EA181614F47301620175
:1032A000C092A004D092A104E092A204F092A304E0
:1032B00020914207309143074091440750914507C0
:1032C000C501B4010E944EEB4B015C018092940455
:1032D00090929504A0929604B0929704A70196014B
:1032E0006D817E818F8198850E944EEB6B017C0100
:1032F000C0929804D0929904E0929A04F0929B04B0
:1033000040909C0450909D0460909E0470909F0497
:1033100029813A814B815C81609190047091910484
:1033200080919204909193040E9406F220914A07A2
:1033300030914B0740914C0750914D070E944EEB46
:10334000A30192010E9406F220ED3CEC4CE45DE307
:103350000E944EEBA30192010E9407F29B01AC0177
:1033600020939C0430939D0440939E0450939F04AB
:1033700089819A81AB81BC81809390049093910460
:10338000A0939204B0939304C501B4010E9407F284
:10339000A70196010E9407F26B017C0120E030E05A
:1033A0004FE753E40E94E9EA181634F4C12CD12CFB
:1033B0008FE7E82E83E4F82E20E030E0A901C70172
:1033C000B6010E946AF387FF06CFEECE60913B07FD
:1033D00070913C0780913D0790913E070895FC0154
:1033E00090E1AFE7B4E001900D929A95E1F708956E
:1033F000EF92FF920F931F93E0929403F092950344
:103400000093960310939703B62F172F022FF32ED6
:10341000242F582FB0939C0310939D0350939E0329
:103420006FEFFF27B01B1F09520B30F4509510951A
:10343000B195160B560B66276093B504A6E0BA9FAC
:103440000092A904712DEE271A9F700DE11D5A9F5D
:10345000E00D7093AA04E093AB04AFE0BA9F009232
:10346000AD04712DEE271A9F700DE11D5A9FE00DDE
:103470007093AE04E093AF04AAE0BA9F0092B10447
:10348000712DEE271A9F700DE11D5A9FE00D70936C
:10349000B204E093B3041F910F91FF90EF90089551
:1034A000A5E0B0E0E6E5FAE10C94D6F16F367105DF
:1034B0008105910578F4FB01EE0FFF1FEE0FFF1F52
:1034C000EB57F74F65917591859194912596EBE0B7
:1034D0000C94F2F1F62EE72E282FE5E8F7E000270E
:1034E000BB275F2D8E2D922F992341F4982F852F86
:1034F000B85F992319F4982F8827B85F903138F472
:1035000082959295582F5F70807F952BBC5F903489
:1035100028F4880F991F880F991FBE5F903818F400
:10352000880F991FB395880F991FE90FF01F5491C9
:1035300081E09927B85079F1C0F0B0FF02C0550F73
:10354000881FB1FF04C0550F881F550F881FB2FF99
:1035500006C082955295152F1F70507F812BB3FFA7
:103560001AC0982F852F552716C0B195B0FF02C0FD
:1035700085955795B1FF04C08595579585955795C5
:10358000B2FF05C08295507F5295582B8F70B3FFC4
:1035900002C0582F8827BB247727AA27B2E0F59EC0
:1035A000B0187109A00BB00BE59E7019A109B00B02
:1035B000259FA019B109F89E7019A109B00BE89ECA
:1035C000A019B109289FB019F99EA019B109E99E67
:1035D000B0195B9DA12C99244427662733278B9D26
:1035E000A00C911C401F601F301F9B9D900C411D23
:1035F000601F301F579FA00C911C401F601F301F81
:10360000879F900C411D601F301F979F400D611DCB
:10361000301F5A9F900C411D601F301F8A9F400D24
:10362000611D301F9A9F600D311D5B9F400D611D14
:10363000301F8B9F600D311D9B9F300DB1E0AA277D
:103640007727BB24F49EB0187109A00BB00BE49E41
:103650007019A109B00B249FA019B109F69E701929
:10366000A109B00BE69EA019B109269FB019F39EDF
:10367000A019B109E39EB019BF187E09A20B20F072
:10368000B1E04B0F601F301F1124762F642F90E0A4
:10369000832F1CCFFC017081472F50E0062E02C003
:1036A000559547950A94E2F740FF14C040911704DE
:1036B00050E0062E02C0559547950A94E2F740FF68
:1036C00009C021E030E001C0220F6A95EAF7209599
:1036D0002723208308958F929F92AF92BF92CF921B
:1036E000DF92EF92FF92FC01C080D180E280F380F4
:1036F00020E030E048EC52E4C701B6010E944EEBF6
:103700004B015C0120E030E0A901C701B6010E9435
:10371000E9EA20E030E040EA50E487FF04C020E01E
:1037200030E040EA50ECC501B4010E9407F22DECF4
:103730003CEC4CEC5DE30E944EEB0E94E6F29B01F8
:103740008BE237FF05C022273327261B370B8DE27C
:103750008093A202C90168EE73E00E94A1F1CB013F
:10376000EAE0F0E0BF010E94A1F1805D8093A30236
:10377000C90164E670E00E94A1F1CB01BF010E9483
:10378000A1F1805D8093A402C901BF010E94A1F153
:103790009C01CB01BF010E94A1F1805D8093A50235
:1037A0008EE28093A602205D2093A70282EA92E037
:1037B000FF90EF90DF90CF90BF90AF909F908F9051
:1037C00008954F925F926F927F928F929F92AF92E5
:1037D000BF92CF92DF92EF92FF92FC01C080D18026
:1037E000E280F38020E030E04AE754E4C701B6010C
:1037F0000E944EEB4B015C0120E030E040E251ECD6
:10380000C701B6010E94E9EA181654F420E030E03E
:1038100048EC52E4C701B6010E946AF387FD8AC0F2
:1038200020E030E0A901C701B6010E94E9EA87FF64
:1038300072C060E070E080EA90ECA50194010E9403
:1038400007F22DEC3CEC4CEC5DE30E944EEB0E9449
:10385000E6F26B017C01F7FC63C020E137E240E057
:1038600050E00E9439F1CA01B9012AE030E040E09D
:1038700050E00E9439F1605D6093A202C701B60179
:1038800028EE33E040E050E00E9439F19AE0892EC2
:10389000912CA12CB12CCA01B901A50194010E945F
:1038A00039F1605D6093A302C701B60124E630E000
:1038B00040E050E00E9439F1CA01B901A50194012C
:1038C0000E9439F1605D6093A4028EE28093A502AC
:1038D000C701B601A50194010E9439F16B01CA012B
:1038E000B901A50194010E9439F1605D6093A602BF
:1038F000F0E3CF0EC092A70282EA92E0FF90EF9031
:10390000DF90CF90BF90AF909F908F907F906F90FF
:103910005F904F90089560E070E080EA90E48DCF72
:10392000F094E094D094C094C11CD11CE11CF11C13
:103930006DE2A2CF20E030E0A901C701B6010E94EC
:10394000E9EA87FF6BC060E070E080EA90ECA501D7
:1039500094010E9407F22DEC3CEC4CEC5DE30E94DC
:103960004EEB0E94E6F24B015C0120E030E0A90141
:10397000C701B6010E94E9EA87FD0BC020E030E0F4
:1039800040E251E4C701B6010E946AF360E287FD9C
:1039900013C0B7FC48C0C501B40128EE33E040E0D5
:1039A00050E00E9439F1CA01B9012AE030E040E05C
:1039B00050E00E9439F1605D6093A302C501B4013B
:1039C00024E630E040E050E00E9439F18AE0482EE1
:1039D000512C612C712CCA01B901A30192010E94E2
:1039E00039F1605D6093A4028EE28093A502C50167
:1039F000B401A30192010E9439F16B01CA01B9011E
:103A0000A30192010E9439F1605D6093A60280E3F8
:103A1000C80EC092A70283EA92E070CF60E070E027
:103A200080EA90E494CFB094A09490948094811C08
:103A3000911CA11CB11C6DE2BFCF282F81E324365D
:103A400009F080E28093A40290E22A3040F03AE04C
:103A5000822F632F0E9474F10E9474F1905D909305
:103A6000A502822F6AE00E9474F1905D9093A602F5
:103A700085E28093A70284EA92E0089560912C0188
:103A800070912D01072E000C880B990B0E94EFEA14
:103A90002AE037ED43E25CE30E944EEB6093740151
:103AA0007093750180937601909377010895CF9379
:103AB000DF93EC01CB01BA010E94EFEA23E333E389
:103AC00043E250E40E944EEB20E030E040E05FE350
:103AD0000E9407F20E94EBF26883DF91CF91089574
:103AE0000E94EFEA23E333E343E250E40E944EEB0B
:103AF00020E030E040E05FE30E9407F20E94EBF23A
:103B000024E6629FC001112481589F4F6FEF70E03F
:103B10000E94A1F1862F91CF80917F07811104C06F
:103B2000809133078093B20708958091CA14882347
:103B3000C1F081508093CA14E4E0F3E1882351F08E
:103B40008150990B2BE1289FF001299FF00D112442
:103B5000E454FC4E8BE1A9EEB2E101900D928A95FE
:103B6000E1F72091CA14211105C08091D41480641A
:103B70008093D41481E090E0A0E0B0E0211103C074
:103B800080E090E0DC018093750790937607A09326
:103B90007707B09378071092700781E080937207DF
:103BA00083E080936F010895CF93DF93EC01CB0105
:103BB000BA010E94EFEA688379838A839B83DF914D
:103BC000CF910895CF93DF93EC01CB01BA010E940E
:103BD000EFEA2DEC3CEC4CEC5DE30E944EEB68838D
:103BE00079838A839B83DF91CF910895CF93DF936D
:103BF000EC01CB01BA010E94EFEA2AE037ED43E283
:103C00005CE30E944EEB688379838A839B83DF9118
:103C1000CF910895CF92DF92EF92FF92CF93DF93EF
:103C200000D000D0CDB7DEB70E94EFEA2AE037ED32
:103C300043E25CE30E944EEB6B017C0120E030E04C
:103C4000A9010E94E9EA2DEB37E346E055E387FF3F
:103C500004C02DEB37E346E055EBC701B6010E94E7
:103C600007F269837A838B839C83CE010196A9DD59
:103C70000F900F900F900F90DF91CF91FF90EF90EA
:103C8000DF90CF900895CF93DF93EC01CB01BA0181
:103C90000E94EFEA0E94E6F279836883DF91CF9178
:103CA00008958F929F92AF92BF92CF92DF92EF9240
:103CB000FF92FC01C080D180E280F38020E030E000
:103CC000A901C701B6010E94E9EA87FD99C06DEB21
:103CD00077E386E095E3A70196010E9407F29F77BC
:103CE00020E030E048EC52E40E944EEB20E030E06F
:103CF00040EA50E40E9407F22DEC3CEC4CEC5DE312
:103D00000E944EEB0E94E6F26B017C0180E2809300
:103D1000A10260E2F0E1CF16F7E2DF06E104F10470
:103D20008CF0C701B60120E137E240E050E00E948C
:103D300039F1CA01B9012AE030E040E050E00E94C8
:103D400039F1605D6093A20260E288EEC81683E0FC
:103D5000D806E104F1048CF0C701B60128EE33E087
:103D600040E050E00E9439F1CA01B9012AE030E098
:103D700040E050E00E9439F1605D6093A30260E290
:103D8000E4E6CE16D104E104F1048CF0C701B601DB
:103D900024E630E040E050E00E9439F1CA01B90168
:103DA0002AE030E040E050E00E9439F1605D60932D
:103DB000A4028AE0882E912CA12CB12CC701B60157
:103DC000A50194010E9439F16B01CA01B901A50155
:103DD00094010E9439F1605D6093A5028EE28093A8
:103DE000A602F0E3CF0EC092A70281EA92E0FF9014
:103DF000EF90DF90CF90BF90AF909F908F900895FD
:103E00006DEB77E386E095EB66CFA4E0B0E0EBE006
:103E1000FFE10C94DFF10E94EFEA2DEC3CEC4CEC5E
:103E20005DE30E944EEB69837A838B839C83CE0192
:103E3000019637DF2496E2E00C94FBF1CF93DF93F9
:103E4000EC018D810E949F8F60E08B810E9406D1E2
:103E5000DF91CF910895CF92DF92EF92FF920F936F
:103E60001F93CF938C01C62F69017A01E7DF0E946F
:103E70007FD28C2F80640E94938F8F2D0E94938F0E
:103E80008E2D0E94938F8D2D0E94938F8C2D0E94DA
:103E9000938F87E8C11101C085E90E94938FCC30D0
:103EA00011F40E94988FC0E00E94988FF8018683D9
:103EB00087FF04C0CF3F11F0CF5FF6CFCF911F91A6
:103EC0000F91FF90EF90DF90CF90089561E0FC019B
:103ED00083810E9406D18FEF0C94938F0F931F93D1
:103EE000CF938C01ABDF0E947FD2C82F882369F06B
:103EF0008DEF0E94938F0E947FD2C82FC801E6DF0A
:103F00008C2FCF911F910F91089582E1F801848346
:103F1000F5CFB0E0A0E0EFE8FFE10C94D5F1EC01C3
:103F20006A017B014801590120E030E0A90167E303
:103F300092DFA501980167E1CE018DDF81111DC0DF
:103F40008F81833039F089E0CC0CDD1CEE1CFF1C26
:103F50008A95D1F7A701960169E1CE017CDF11E0D6
:103F6000882319F010E087E08C83CE01AFDF812F2A
:103F7000CDB7DEB7ECE00C94F1F189E08C8310E072
:103F8000F4CFCF93DF93EC016EBDFA01CA019E5FBF
:103F90000DB407FEFDCF20812EBD0DB407FEFDCF71
:103FA00021812EBD3296E817F90791F70DB407FE6F
:103FB000FDCF8FEF0E94938F8FEF0E94938F0E940F
:103FC000988F8E838F71853041F083E18C83CE0191
:103FD0007DDF80E0DF91CF91089581E0FBCF0F93EB
:103FE0001F93CF93DF93EC018B0128DF0E947FD2D8
:103FF00081110BC085E18C8310E0CE0167DF812F3A
:10400000DF91CF911F910F910895A8016CEFCE0120
:10401000B8DF182F882371F3F0CF0F931F93CF933E
:10402000DF93EC0189018F81833039F089E0440FFF
:10403000551F661F771F8A95D1F79A01AB0168E17A
:10404000CE0109DF811127C0A8016EEFCE0199DFF3
:10405000182F8823A9F00E947FD2182F8823C1F03F
:1040600020E030E0A9016DE0CE01F5DE882321F0EB
:1040700086E18C8310E004C00E94988F8111F8CFF4
:10408000CE0124DF812FDF91CF911F910F910895F1
:1040900087E18C83F5CF86E0ECCF1F93CF93DF933E
:1040A000EC01CCDE20E030E0A9016CE0CE01D3DEF3
:1040B00011E0882319F010E083E08C83CE0106DF45
:1040C000812FDF91CF911F9108951F93CF93DF939D
:1040D000EC018F81833039F089E0440F551F661F52
:1040E000771F8A95D1F79A01AB0162E1CE01B3DE69
:1040F00011E0882319F010E085E08C83CE01E6DE24
:10410000812FDF91CF911F9108958F929F92AF924F
:10411000BF92EF92FF920F931F93CF93DF938C0187
:10412000EB017A010E94EBD14B015C012CE2820E83
:1041300021E0921EA11CB11C0E94988FF801868379
:104140008F3F69F40E94EBD1681979098A099B09AC
:1041500097FDF2CF81E1F8018483C0E021C08E3F5A
:1041600069F5F1E0EF1AF1088FEF8EBDFE012FEF38
:104170000DB407FEFDCF8EB581932EBDCF018C1BF4
:104180009D0B8E159F05A0F30DB407FEFDCF8EB5D8
:10419000CE0DDF1D88830E94988F0E94988FC1E00A
:1041A000C80194DE8C2FDF91CF911F910F91FF906A
:1041B000EF90BF90AF909F908F9008958FE0CBCFFE
:1041C0000F931F93CF93DF93EC018B0137DE40E019
:1041D00052E0B801CE0199DFDF91CF911F910F918D
:1041E00008950F931F93CF93DF93EC0189018F8183
:1041F000833039F089E0440F551F661F771F8A9579
:10420000D1F79A01AB0161E1CE0125DE882351F09F
:1042100084E08C83CE015ADE80E0DF91CF911F9144
:104220000F91089540E052E0B801CE016EDFF5CF66
:10423000B0E0A0E0EEE1F1E20C94D5F1EC01162F34
:104240001F821C824B830E94EBD16B017C0120ED0D
:10425000C20E27E0D21EE11CF11CA89561E08B8103
:104260000E9406D18B810E94D4B6249A2C9A279A58
:104270002698259A81E00E949F8F85E08D830E9479
:104280009F8F0AE08FEF0E94938F0150D9F7A89576
:1042900020E030E0A90160E0CE01DDDD8E838130D9
:1042A00079F00E94EBD16C197D098E099F0997FD69
:1042B000EFCF81E08C83CE0109DE1A8280E065C0F9
:1042C000A8952AEA31E040E050E068E0CE01C3DD85
:1042D000853031F581E08F83A8958F81812C912CD9
:1042E0005401823029F4812C912CA12C80E4B82E29
:1042F00020E030E0A90167E3CE01ADDDA501940126
:1043000069E2CE01A8DD8E838823F1F00E94EBD113
:104310006C197D098E099F0997FDEACF8AE0CACF03
:1043200004E00E94988F8E830150D9F78A3A11F4E5
:1043300082E0D1CF0E94EBD16C197D098E099F09D3
:1043400097FDBFCF82E0B6CF8F818230B9F420E0F5
:1043500030E0A9016AE3CE017EDD882311F088E018
:10436000A9CF0E94988F807C803C11F483E08F83DA
:104370000E94988F0E94988F0E94988FCE01A6DD90
:1043800081E08A83173030F41D83CDB7DEB7ECE0CF
:104390000C94F1F188E18C8391CF0F931F93CF930D
:1043A000DF93EC018B0120E030E0A90169E053DDEF
:1043B000882351F080E18C83CE0188DD80E0DF919D
:1043C000CF911F910F91089540E150E0B801CE01C7
:1043D0009CDEF5CFCF93C82FCB010E94918488EB50
:1043E00096E00E94918489EA96E0CC2311F08EEA4F
:1043F00096E00E9491848AE00E947084CF91089593
:10440000EF92FF920F931F93CF937B018A01C2E437
:104410008F3F09F0C4E580E20E9470848C2F0E94D7
:1044200070848AE30E947084F701608171818281C7
:10443000938142E00E94F3B68AE693E10E94918460
:10444000F801608171818281938142E00E94F3B61C
:1044500062E070E080E090E00E9462D1CF911F9115
:104460000F91FF90EF9008950C94F7D14091920333
:1044700021E042276CE070E00C94A8B640919203D2
:1044800021E0422764E070E00C94A8B640919203CA
:1044900021E0422761E070E00C94A8B640919203BD
:1044A00021E0422761E070E00C94A8B640919203AD
:1044B00021E0422768E070E00C94A8B64091920396
:1044C00021E042276CE070E00C94A8B641E061E086
:1044D00070E00C94A8B64091920321E042270C941E
:1044E000A8B66CE070E00C9495D161E070E00C949B
:1044F00095D161E070E00C9495D16CE070E00C9483
:1045000095D164E070E00C9495D19091B90281E06E
:1045100089270C94097A61E083E397E00C94957AFB
:1045200020E030E0A901BC018AE791E00C94C2C709
:1045300080E090E0A0E8B0E4809382019093830152
:10454000A0938401B09385018FE192E0E9DF80E0E0
:1045500090E0A0EFB1E480937A0190937B01A09367
:104560007C01B0937D0180937E0190937F01A093A5
:104570008001B0938101E091F403EE0FFF0BE15055
:10458000FE4F808191818330910539F1843091050E
:10459000C9F1029761F480E090E0A3E4B3E4809372
:1045A0007A0190937B01A0937C01B0937D0187E019
:1045B00092E0B6DF10928201109283011092840182
:1045C000109285018FE192E0ABDF8091F4038F5F61
:1045D0008430ECF48093F403089580E090E0A3E449
:1045E000B3E480937A0190937B01A0937C01B09314
:1045F0007D0180937E0190937F01A0938001B09311
:104600008101D5CF80E090E0A3E4B3E4F2CF109233
:10461000F4030895A4E0B0E0E0E1F3E20C94DFF1EC
:1046200084EF91E0A0E0B0E089839A83AB83BC8300
:10463000BE016F5F7F4F88E70E9438832496E2E0D7
:104640000C94FBF1B0E0A0E0E8E2F3E20C94DFF1BF
:1046500020E24F8158856E818D810E94B9CCE2E0C5
:104660000C94FBF180913307909134070C942CD279
:10467000609133078FEF0C9436D280913307682F07
:104680000C9436D26FEF809133070C9436D26EE1E2
:1046900073E582E00C94C7CE62E273E581E00C948E
:1046A000C7CE66E273E580E00C94C7CE6AE273E59C
:1046B00083E00C94C7CE109270070C9416D84FE389
:1046C00050E069ED74E081EF96E00C9440F4809145
:1046D0006A1390916B13891B8F7011F40C94E97B12
:1046E00081E0089580916F01882341F06091EC038F
:1046F0007091ED0341E081E00C9459CC08950F9343
:104700001F93CF93DF93FC012381222331F080E0BC
:10471000DF91CF911F910F9108958B01EC01FB0167
:104720008789803139F582E08B831D8A1E8A1F8A32
:10473000188E808D918DB0E0A0E025E0880F991F44
:10474000AA1FBB1F2A95D1F7898B9A8BAB8BBC8B89
:104750001A8F098F81E08983188619861A861B862D
:104760001C821D821E821F82188A1C861D861E8640
:104770001F86CECF803259F683E08B83428D538DD6
:10478000648D758D4D8B5E8B6F8B788F9E012F5E48
:104790003F4FC8010E9474D98111DACFB8CFCF93AF
:1047A000DF93EC010E94DDD91B82DF91CF91089548
:1047B000CF93DF93EC01462F41706C857D858E850C
:1047C0009F850E9486D6882351F0888920E2829FA7
:1047D000C001112480569F4EDF91CF91089590E043
:1047E00080E0FACFCF93DF93EB01FC01238121110D
:1047F00004C080E0DF91CF9108952250223028F448
:104800008FE28883198281E0F5CF60E0D1DF0097E5
:1048100081F3DC0160E080E09EE22D91203299F08E
:10482000883031F49E01260F311DF90190836F5FAE
:104830009E01260F311DAD0141505109FA01408101
:10484000F90140836F5F8F5F8B3039F7FE01E60F10
:10485000F11D1082D8CFACE0B0E0E1E3F4E20C94BB
:10486000D0F15C01DC0159968D909C90F40181851A
:104870009285A385B4859C01AD012F5F3F4F4F4FBB
:104880005F4F29873A874B875C87D50114964D90F7
:104890005D906D907C9017974114510461047104F0
:1048A00009F459C0BFEF4B1A5B0A6B0A7B0A312C23
:1048B000730162011D821E821F821886F4018185A8
:1048C0009285A385B4852D813E814F815885281717
:1048D00039074A075B0708F056C089859A85AB857A
:1048E000BC858C159D05AE05BF0550F482E0C82E31
:1048F000D12CE12CF12C92E0492E512C612C712C01
:104900009E012F5F3F4FB701A601C4010E94F8D856
:104910008823C9F189819A81AB81BC81892B8A2B3B
:104920008B2B01F1260137019FEF491A590A690AB9
:10493000790A2D813E814F8158852F5F3F4F4F4F20
:104940005F4F2D833E834F8358873FEFC31AD30AAF
:10495000E30AF30AB3CF408051806280738033242E
:104960003394A6CFC414D504E604F70411F70FEF6F
:104970001FEF2FEF3FE0B701A601C4010E947ED8D0
:10498000782E811106C0712C872D2C96E1E10C94B4
:10499000ECF1F5014481558166817781411551051E
:1049A0006105710539F097018601C4010E947ED826
:1049B000882349F3D5011496CD92DD92ED92FC92B5
:1049C0001797332051F0D701C6010196A11DB11DE3
:1049D000F40180839183A283B383F501858996894D
:1049E000A789B08D892B8A2B8B2B71F6C58AD68A25
:1049F000E78AF08E818180688183C6CF40E050E0F5
:104A0000BA010C9426DA4F925F926F927F92AF9226
:104A1000BF92CF92DF92EF92FF920F931F93CF93AB
:104A2000DF931F92CDB7DEB78C017B015A01C22EF6
:104A3000DB0159968D919C91F801928F818FCB016A
:104A4000DDDF712CF70180859185A285B3854189D1
:104A500052896389748984179507A607B70708F0F8
:104A600052C055E0B695A795979587955A95D1F779
:104A7000F82FFF70DF2ED70113968C91823010F43F
:104A800080E0DAC041E050E0BE016F5F7F4FC701B8
:104A90000E9421DB0197A1F7F70180859185A2850E
:104AA000B3854F96A11DB11D80879187A287B387DB
:104AB000F0E2DF9EB001112460567F4E6115710552
:104AC000F9F2DB018C91882341F0853E09F04BC05F
:104AD000772029F077247394B5CF71100EC08091A0
:104AE000A0129091A112A091A212B091A312F8016C
:104AF00084879587A687B787D08ADB018C9181113F
:104B0000E9CF772473948C2D8274823409F0B8CF66
:104B1000772009F4A1C0F801D08861E0C80148DE1F
:104B2000009709F4ADCF20E2DC011D922A95E9F748
:104B30002BE0F501DC0101900D922A95E1F721E2CD
:104B400038E2FC01318B208B40E058E057874687E4
:104B5000338B228B318F208F578B468B0E943DD613
:104B6000811109C08DCF4BE050E0C5010E94F0F3E8
:104B7000892B09F067CFF0E2DF9ED00111249D015F
:104B800020563F4EF9018385817121F08C2D827171
:104B900009F000C1F801818D928D4091A0125091D1
:104BA000A1126091A2127091A31244875587668763
:104BB0007787D08AFD01E056FF4E44885588712CD6
:104BC000612C320155244424D80155964D925D92B2
:104BD0006D927C925897428D538D70E060E044292D
:104BE00055296629772955964D935D936D937C934E
:104BF0005897D9011B962C91287109F0BDC0848D5E
:104C0000958DA68DB78DF801818B928BA38BB48B7C
:104C100081E083838C2D8F70F8018183148215824B
:104C200016821782108611861286138681E0C4FED2
:104C300003C0C8010E94ABDA0F90DF91CF911F91A2
:104C40000F91FF90EF90DF90CF90BF90AF907F904B
:104C50006F905F904F900895D70113968C911397A2
:104C6000823009F40DCF51968D919D910D90BC919C
:104C7000A02D803E9F4FAF41B10508F001CFC70185
:104C8000EADD882309F4FCCE0E943DD6882309F48E
:104C9000F7CED7015996ED91FC915A9714964D9005
:104CA0005D906D907C901797B2E04B1A51086108A7
:104CB0007108858504C0440C551C661C771C8A95B8
:104CC000D2F786859785A089B189480E591E6A1E3C
:104CD0007B1E81E08093A4124092A0125092A112F8
:104CE0006092A2127092A312E0EAF0E180E092E0FA
:104CF000DF019C011D9221503040E1F7DD24D39467
:104D0000D7015996ED91FC918481D816C0F4809119
:104D1000A5129091A612DC01ED91FC910288F38915
:104D2000E02D20EA30E1B301A2014D0D511D611DBE
:104D3000711D0995882309F4A3CED394E1CF25856D
:104D400080E092E0A0E0B0E004C0880F991FAA1FA5
:104D5000BB1F2A95D2F7F70141895289638974896B
:104D6000840F951FA61FB71F818B928BA38BB48BCB
:104D700080EA90E1D12CD7CE203161F498012F5EEA
:104D80003F4F0E9474D9882329F084E0D8011396FC
:104D90008C9340CFD80113961C9272CEFC012381D4
:104DA0002111FDCC0895A1E4B0E0E9EDF6E20C9408
:104DB000CFF14C015B017A01222E19821C821C8EDC
:104DC0001F8E6115710569F410E0CE014C96E6DF87
:104DD000CE010196E3DF812FCF5BDF4FE2E10C9440
:104DE000EBF1FC0183818111EFCFFA0180818F32D9
:104DF00051F18B01CE0101966C012C0180E2382E1D
:104E0000360122963FAE229721963FAE21973FAEC4
:104E10003EAE3DAE3CAE3BAE3AAE39AE38AE3FAA4A
:104E2000970190E047E0D9018D91882309F446C0AD
:104E30008F3209F443C08E3201F54A3029F298E0EE
:104E40004AE09D01F0CFFB0183818250823098F0CF
:104E5000618D728DCE014C9652DC882309F4B4CF5B
:104E60008E01045E1F4FC7017C010196F70120816E
:104E70002F32D1F3BFCF8B01F6CFE6E7F3E12491D8
:104E8000222321F031968213FACF9ECF491708F4DE
:104E90009BCF813208F498CF8F3709F495CF3FE943
:104EA000380F3A3108F420EEE7E3F0E0EC0FFD1F95
:104EB000E90FF11D820F80839F5FC3CF8FA98032DE
:104EC00009F482CF7901F90180812F5F3F4F8F3242
:104ED000C9F38823C1F021E0AE01495C5F4FB801FE
:104EE000C60191DD882309F46FCF0A151B0511F067
:104EF000C80155DCCE014C964C145D0409F0C30189
:104F000086016C017ECF222DAE01495C5F4FB80156
:104F1000C40179DD182F59CFEF92FF921F93CF93E1
:104F2000DF93CDB7DEB728970FB6F894DEBF0FBE7C
:104F3000CDBF182F85EBE82E82E1F82EF7016085B2
:104F40007185072E000C880B990B0E94EFEA6D8388
:104F50007E838F839887F70184819581A681B781AD
:104F600089839A83AB83BC83AE014B5F5F4FBE01E5
:104F70006F5F7F4F80E044DA97E3E92E97E0F92EE8
:104F8000F70160857185072E000C880B990B0E9434
:104F9000EFEA6D837E838F839887F7018481958103
:104FA000A681B78189839A83AB83BC83AE014B5FB3
:104FB0005F4FBE016F5F7F4F8FEF22DA87E11802EC
:104FC000F0011124EB54FD4E628570E082E793E11D
:104FD0000E940F8EF701628570E08DE693E10E94DA
:104FE0000F8E28960FB6F894DEBF0FBECDBFDF91AF
:104FF000CF911F91FF90EF9008950F930FB70F93EC
:1050000000916E000B7F00936E0078940F930BB7A6
:105010000F930CB70F921F922F933F934F935F9371
:105020006F937F938F939F93AF93BF93EF93FF9370
:1050300011240E942B66FF91EF91BF91AF919F9138
:105040008F917F916F915F914F913F912F911F9021
:105050000F900CBF0F910BBF0F910460F894009359
:105060006E000F910FBF0F911895CF93DF931092A1
:10507000A603C5EBD2E1198618860E94F7D11A86DD
:105080005D98C7E3D7E0198618860E94846A1A865D
:105090005C98DF91CF910895B0E0A0E0E2E5F8E2FE
:1050A0000C94D5F1B0E4A0E06A2F70E0AB014B0F97
:1050B000511D55954795411111C0E0E1FBE2659105
:1050C0007491072E000C880B990B0E94EFEACDB764
:1050D000DEB7ECE00C94F1F1B42FE8CFA41711F097
:1050E000B41303C0ECE0FCE2EACF9A01215031098D
:1050F000220F331F220F331FF901E25FF44DE590B9
:10510000F490F901EE5EF44DC591D4918E159F0592
:105110001CF3A42FC817D9070CF4C6CFF901E05F20
:10512000F44D05911491F901EC5EF44DC590D490C5
:10513000BC016E197F09072E000C880B990B0E9489
:10514000EFEA4B015C01B601601B710B072E000CEE
:10515000880B990B0E94EFEA9B01AC01C501B401D9
:105160000E944EEB4B015C01BE016E197F09072EB8
:10517000000C880B990B0E94EFEA9B01AC01C50162
:10518000B4010E947EF26B017C01B801012E000C7B
:10519000880B990B0E94EFEA9B01AC01C701B60195
:1051A0000E9407F294CFEF92FF920F931F93CF9339
:1051B000C82F7B018A0180913207833090F00E94D2
:1051C000FE8AC7010E94918480ED92E10E94918441
:1051D000CF3FF1F48CEC92E10E9491848AE00E942E
:1051E000708443DFA89580918F04811123C081E0F2
:1051F00080938F0482E08093320737DF63EC72E1A3
:10520000CF3F11F067EC72E140E0C8010E94C18E0F
:10521000C7FDE4CF8AEC92E10E9491846C2F0C2EA2
:10522000000C770B880B990B0E94A9B48AE00E94AE
:105230007084D4CFCF911F910F91FF90EF9008957C
:10524000B0E0A0E0E6E2F9E20C94D1F1EC016B01F0
:105250004A01B22EFA014080518062807380A3011E
:1052600092016D817E818F8198850E94E9EA882371
:10527000A1F04D825E826F827886AA24A39420E0FA
:1052800030E0A901F40160817181828193810E94E3
:105290006AF318160CF0A12CAC828C818230A1F03C
:1052A000833009F44FC08130D1F52D813E814F818B
:1052B0005885F60160817181828193810E94E9EABB
:1052C00087FD2DC082E08C83B7010F2C000C880B6A
:1052D000990B0E94EFEA9B01AC016D817E818F8169
:1052E00098850E9406F29B01AC01F60160817181F4
:1052F000828193810E946AF387FD16C00E94EBD1E0
:105300006B017C019801A8EEB3E00E9465F1C60E26
:10531000D71EE81EF91EC882D982EA82FB82CDB769
:10532000DEB7E0E10C94EDF10E94EBD10881198128
:105330002A813B81601B710B820B930B97FDEFCF92
:1053400083E08C834AE453E16AE573E18B2D2BDF24
:10535000E6CF4EEE52E16BEF72E125CFCF93DF93B4
:10536000A8958091B7129091B8120E9421B66093CF
:10537000B9127093BA128093BB129093BC128091B1
:10538000390790913A0788DE60933B0770933C079A
:1053900080933D0790933E07C091B712D091B81209
:1053A0008091680190916901C817D90714F480E0D1
:1053B000D0DF8091BD129091BE12181619066CF4C0
:1053C00080916601909167018C179D0734F44BE240
:1053D00053E168E373E180E0E6DE20913907309124
:1053E0003A078091E8069091E9062817390714F4E6
:1053F0008FEFAFDF80913F07909140071816190695
:105400008CF42091390730913A0780916401909192
:1054100065018217930734F44BE253E168E373E1CB
:105420008FEFC1DEDF91CF910895A4E0B0E0EBE112
:10543000FAE20C94D5F180913207811106C0A8954B
:105440002496ECE00C94F1F128C18091A404811120
:10545000F7CF81E08093A4048091A703811107C056
:105460001092A4042496ECE00C94F1F116C176DFBE
:105470001092A7030E94EBD14B015C010E94C4B4BF
:105480006B017C0160916C0170916D01072E000C25
:10549000880B990B0E94EFEA9B01AC01C701B60192
:1054A0000E946AF318160CF4E7C06091BD12709167
:1054B000BE12072E000C880B990B0E94EFEA69833D
:1054C0007A838B839C8334E0E32EF12C08E210E096
:1054D00020E0AE014F5F5F4F69EB72E18FE193E136
:1054E000AFDEC090B912D090BA12E090BB12F0902B
:1054F000BC1260916A0170916B01072E000C880B41
:10550000990B0E94EFEA9B01AC01C701B6010E9412
:105510006AF31816CCF460916C0170916D01072E3E
:10552000000C880B990B0E94EFEA9B01AC01C701AC
:10553000B6010E94E9EA87FF07C00E94CDB40E942D
:10554000E6F27595679501C060E06093BF128091A7
:10555000B1129091B212A091B312B091B41200970F
:10556000A105B105C1F0A5019401281B390B4A0B17
:105570005B0BDA01C901B7FD0EC00E94C4B40E94E2
:10558000E6F22091AF123091B012621773070CF45B
:105590007DC00E94F7D10E94E61920E030E04AEF7A
:1055A00052E40E946AF318160CF463C08091A203BF
:1055B0009091A303A091A403B091A5030097A10526
:1055C000B105A1F0881A990AAA0ABB0AB7FC0EC055
:1055D0000E94E6190E94E6F22091A0033091A103F7
:1055E000621773070CF44BC00E94846A60913F07F6
:1055F00070914007072E000C880B990B0E94EFEA70
:1056000069837A838B839C8392E0E92EF12C04E1F9
:1056100010E02FEFAE014F5F5F4F6BE377E088E262
:1056200093E10EDE80903B0790903C07A0903D07F1
:10563000B0903E0720E030E040EA50E4C501B401FC
:105640000E946AF387FD11C020E030E04AEF52E487
:10565000C501B4010E94E9EA18163CF00E949218B4
:105660000E94E6F27595679501C060E0609341077E
:10567000F7CE8FEF6EDE9ACF80E06BDE16CF4DE077
:1056800053E16CE173E18FEF8EDDB0CF4DE053E17C
:105690006CE173E180E087DD7ECFCF92DF92EF9205
:1056A000FF92CF93DF93EC01C880D980EA80FB8022
:1056B00089EB92E10E949184C701B6010E9456765F
:1056C000CC80DD80EE80FF8083E49FE20E949184A5
:1056D000C701B6010E945676C884D984EA84FB8447
:1056E0008FE39FE20E949184C701B6010E94567623
:1056F0008AE00E947084DF91CF91FF90EF90DF905D
:10570000CF900895BC0120917004309171044091B4
:105710007004509171042417350731F481E0261785
:10572000370709F080E008959A01F1CF0F930FB782
:105730000F9300916E000F930B7F00936E0000910A
:105740006F000D7F00936F000F930BB70F930CB793
:105750000F921F922F933F934F935F936F937F937B
:105760008F939F93AF93BF93EF93FF931124E1D453
:10577000FF91EF91BF91AF919F918F917F916F9129
:105780005F914F913F912F911F900F900CBF0F9100
:105790000BBF0F910260F89400936F000F9100937C
:1057A0006E000F910FBF0F91189500C000C080913F
:1057B000EC0680FF1FC0459A8FEF809329048091EB
:1057C000EC0681FF1AC0479A8FEF80932A048091DC
:1057D000EC0682FF15C02A988FEF80932B048091EE
:1057E000EC0683FF10C028988FEF80932C0400C034
:1057F00000C00895459881E0E0CF479881E0E5CF6B
:105800002A9A81E0EACF289A81E0EFCF8091930332
:10581000982F977F90939303982F937081E011F0C6
:1058200080E008955E9A08955E9880919303886061
:10583000809393030895E82FF0E021E030E0082EF4
:1058400002C0220F331F0A94E2F720953095909101
:105850009303922390939303E550FE4F208192236C
:1058600021E019F020E0822F0895813079F038F09E
:105870008230C9F7159A909182079B7F04C05E9A87
:10588000909182079E7F90938207EDCF5E9A9091D0
:1058900082079D7FF8CF80E0CEDF81E0CCDF82E021
:1058A000CADFB4CF813079F070F0823071F021E03E
:1058B00030E001C0220F8A95EAF780919303822B92
:1058C0008093930308955E98F2CF1598F0CFB0E0DF
:1058D000A0E0EDE6FCE20C94D7F1C4E7DDE00AE9D4
:1058E00017E084E8A82E8DE0B82EC12CD12C7601CB
:1058F000C39469917991899199910E94EDEA2889DF
:1059000039894A895B890E944EEB0E94EBF2F801CB
:1059100061937193819391938F01C616D706E80620
:10592000F90610F46B017C01AC16BD0611F76FEFA0
:105930007FEFCB01A70196010E9417F12093AA07E0
:105940003093AB074093AC075093AD07CDB7DEB7AC
:10595000EAE00C94F3F10F931F93CF93DF9308E8E1
:105960001DE0C3EBD7E0F8012191319141915191B4
:105970008F0160E070E080E89FE30E947EF269930F
:10598000799389939993F7E0C33CDF0761F70E940D
:10599000E5C79DDFDF91CF911F910F910895DBCF78
:1059A000DACFD9CFD8CF90916A1380916B13981327
:1059B00006C08091BC0D9091BD0D892B21F080E037
:1059C0000E94B08FF0CF089590916A1380916B136D
:1059D000981307C08091BC0D9091BD0D892B09F4DF
:1059E0005ACF80E00E94B08FEFCFCF92DF92EF923C
:1059F000FF92CF93DF932091B902222319F1EC019A
:105A000008960E94BA776B017C0120E030E0A90182
:105A10000E94E9EA20E030E0A901882349F0CE01A4
:105A20000E943278A70196010E944EEB9B01AC01C7
:105A3000688579858A859B850E9406F268877987C3
:105A40008A879B87DF91CF91FF90EF90DF90CF9077
:105A50000895CF92DF92EF92FF92CF93DF93209140
:105A6000B902222319F1EC0108960E94BA776B0162
:105A70007C0120E030E0A9010E94E9EA20E030E06A
:105A8000A901882349F0CE010E943278A70196012E
:105A90000E944EEB9B01AC01688579858A859B85C8
:105AA0000E9407F2688779878A879B87DF91CF9169
:105AB000FF90EF90DF90CF900895AEE1B0E0E3E685
:105AC000FDE20C94D1F19E8F8D8F5B018A01FC0168
:105AD000EA5BFF4F2081318142815381298B3A8BD0
:105AE0004B8B5C8BCA01B9010E94EDEA6B017C0112
:105AF000D5012D913D914D915C910E944EEB0E94FC
:105B00006BF22B013C01F8012081318142815381EC
:105B1000C701B6010E944EEB0E946BF24B015C0183
:105B2000C301B2010E94EBF26D8B7E8B8F8B988F3D
:105B3000683771058105910540F428E730E040E0C1
:105B400050E02D8B3E8B4F8B588FC501B4010E94C6
:105B5000EBF2698F7A8F8B8F9C8F68377105810587
:105B6000910540F488E790E0A0E0B0E0898F9A8F3B
:105B7000AB8FBC8FED8DFE8DEE5AFF4F20813181B2
:105B80004281538129873A874B875C87CA01B901D3
:105B90000E94EFEA2B013C016D897E898F89988DE7
:105BA0000E94EDEA6D837E838F83988720E030E04A
:105BB000A901C301B2010E94E9EA882309F4BBC12B
:105BC000A7019601C701B6010E944EEB4B015C0193
:105BD0002D813E814F815885CA01B9010E944EEB4B
:105BE0009B01AC01C501B4010E9406F24B015C01AE
:105BF000A3019201C301B2010E9407F29B01AC0113
:105C0000C501B4010E947EF20E946BF20E94EBF289
:105C100069837A838B839C8369857A858B859C8550
:105C200090958095709561957F4F8F4F9F4F0E9403
:105C3000EFEA4B015C01698D7A8D8B8D9C8D0E9402
:105C4000EDEA69877A878B879C8720E030E0A9019D
:105C5000C501B4010E94E9EA882309F470C12985CD
:105C60003A854B855C85CA01B9010E944EEB6D8770
:105C70007E878F87988BA7019601C701B6010E9486
:105C80004EEB9B01AC016D857E858F8598890E94C6
:105C900006F26B017C01A5019401C501B4010E94CB
:105CA00007F29B01AC01C701B6010E947EF20E947F
:105CB00017F3AD8DBE8D95962D913D914D915C91D3
:105CC00098972D873E874F87588B69017A012981E4
:105CD0003A814B815C81C21AD30AE40AF50A0E9418
:105CE000EBF2C61AD70AE80AF90AF7FE8CC02D8132
:105CF0003E814F815885CA01B9010E944EEB6B016C
:105D00007C0120E030E0A901C301B2010E94E9EA70
:105D1000882309F418C16D857E858F8598890E9436
:105D2000EDEA9B01AC010E9407F2A30192010E94DF
:105D30004EEB4B015C0129853A854B855C85CA0198
:105D4000B9010E944EEB9B01AC01C501B4010E9458
:105D500007F2A70196010E9406F24B015C0120E0C8
:105D600030E040E850E4C301B2010E944EEB9B01D9
:105D7000AC01C501B4010E947EF20E946BF24B019E
:105D80005C0120E030E0A9010E946AF387FF03C0B4
:105D9000812C912C5401C501B4010E94EBF269835E
:105DA0007A838B839C832D853E854F855889261762
:105DB00037074807590720F429833A834B835C83CC
:105DC00069817A818B819C810E94EDEA4B015C01A3
:105DD000A3019201C301B2010E9407F29B01AC0131
:105DE000C501B4010E944EEBA70196010E9407F283
:105DF0000E94A3F30E94EBF2698B7A8B8B8B9C8BB6
:105E0000C12CD12C760169897A898B899C892D894D
:105E10003E894F89588D621B730B840B950B0E9432
:105E2000EDEAA30192010E947EF220E034E244EF09
:105E300059E40E944EEB0E94EBF24B015C01698930
:105E40007A898B899C89298D3A8D4B8D5C8D621B5B
:105E5000730B840B950B0E94EDEAA30192010E9443
:105E60007EF220E034E244EF59E40E944EEB0E94BF
:105E7000EBF26D837E838F839887C501B4010E9406
:105E8000501A2B013C016D817E818F8198850E9483
:105E9000501A29813A814B815C81AD8DBE8D9996D6
:105EA0002D933D934D935C939C9789019A010C0D22
:105EB0001D1D2E1D3F1DFD0105A716A727A730ABF1
:105EC000E65BFF4F2D893E894F89588D20833183B2
:105ED00042835383D5968D929D92AD92BC92D89772
:105EE0002D813E814F815885D9962D933D934D93B9
:105EF0005C93DC973D974082518262827382349634
:105F0000608371838283938329893A894B895C8971
:105F1000D1962D933D934D935C93D4973D96298DC7
:105F20003A8D4B8D5C8D20833183428353836E96F3
:105F3000E0E10C94EDF160E070E0CB0165CE60E053
:105F400070E0CB01B4CE60E070E0CB0116CF909151
:105F50006F0081E091FD02C080E0089590916F0094
:105F60009D7F90936F000895EFE6F0E0808182605E
:105F700080830895CF93C82FEADF94E0C99F9001F2
:105F80001124F901ED58FB4F21583B4FD9014D9198
:105F90005D916D917C91408351836283738391E025
:105FA000909372048111E0DFCF910895CF93DF9336
:105FB0008091EB06811105C08091ED06882309F4DC
:105FC0004EC080910404329B4DC0816080930404D4
:105FD00080910404339B48C08260809304048091C4
:105FE0000404349B43C0846080930404C091630420
:105FF000C0FF0FC08091EC0680FF0BC080910404AD
:1060000080FF07C08091310781608093310780E075
:10601000B1DFC1FF0FC08091EC0681FF0BC0809102
:10602000040481FF07C080913107826080933107AB
:1060300081E0A0DFC2FF13C08091EC0682FF0FC099
:106040008091ED06882359F08091040482FF07C0F7
:106050008091310784608093310782E08BDFDF918C
:10606000CF9108958E7FB2CF8D7FB7CF8B7FBCCF7E
:106070006EDF1092AE071092AF071092B007109229
:10608000B107811171CF08950F931F9380916A1307
:1060900090916B13891B8F7009F449C0909167131D
:1060A000992361F0833040F48FEF890F29F08093BA
:1060B000671390E080E038C01092671380916B13F3
:1060C0002BE5829FC00111248D53984FFC01208144
:1060D00020FDEFCF4091AE075091AF076091B00720
:1060E0007091B107E95AFF4F0081118122813381FC
:1060F000401B510B620B730B4093AE075093AF07DD
:106100006093B0077093B10720916B132F5F2F70CE
:106110002093681330916B1320916913321304C0DC
:1061200020916813209369131F910F910895A0DFA8
:10613000C0CFA3E1B0E0EFE9F0E30C94CFF18FEF33
:106140009FEF90938900809388002AE02983312C67
:10615000212C789480916C0490916D04A0916E0430
:10616000B0916F04892B8A2B8B2B09F0C2C18091CF
:1061700072048823D1F08091700490917104109280
:106180007204892B91F01092710410927004109295
:10619000630490916A1380916B13981731F080918A
:1061A0006B138F5F8F7080936B138091700490914D
:1061B0007104892B09F49DC14091680450916904D0
:1061C00060916A0470916B048091640490916504FD
:1061D000A0916604B091670400915A0410E030E089
:1061E00020E0841B950BA60BB70B081719072A078D
:1061F0003B0710F4D901C8018A8B840F951FA61F95
:10620000B71F8093680490936904A0936A04B093C5
:106210006B04E1E0C0903104D0903204E09033048C
:10622000F09034048091410490914204A091430481
:10623000B0914404C80ED91EEA1EFB1EC092410450
:10624000D0924204E0924304F0924404F7FC33C03D
:1062500040912904042E000C550B660B770B80919E
:106260007F0490918004A0918104B0918204840FF6
:10627000951FA61FB71F80937F0490938004A0935F
:106280008104B093820480912D0490912E04A091FA
:106290002F04B0913004B701A601481B590B6A0BBB
:1062A0007B0BDB01CA018093410490934204A093CD
:1062B0004304B093440400913504109136042091B6
:1062C0003704309138048091450490914604A091A0
:1062D0004704B0914804080F191F2A1F3B1F009361
:1062E000450410934604209347043093480437FD37
:1062F00033C040912A04042E000C550B660B770B1B
:106300008091830490918404A0918504B0918604C7
:10631000840F951FA61FB71F809383049093840456
:10632000A0938504B093860480912D0490912E044F
:10633000A0912F04B091300428013901481A590A5C
:106340006A0A7B0AD301C2018093450490934604F4
:10635000A0934704B09348044091390450913A0403
:1063600060913B0470913C048091490490914A04EF
:10637000A0914B04B0914C04480F591F6A1F7B1F1A
:106380004093490450934A0460934B0470934C0427
:1063900077FD33C080902B04082C000C9908AA08C4
:1063A000BB088091870490918804A0918904B091E2
:1063B0008A04880D991DAA1DBB1D809387049093A4
:1063C0008804A0938904B0938A0480912D0490914D
:1063D0002E04A0912F04B09130043A014B01681AA9
:1063E000790A8A0A9B0AD401C301809349049093D5
:1063F0004A04A0934B04B0934C0480903D049090C9
:106400003E04A0903F04B090400480914D049091D0
:106410004E04A0914F04B0915004880D991DAA1DFF
:10642000BB1D80934D0490934E04A0934F04B093F2
:106430005004B7FD33C040902C04042C000C5508C8
:106440006608770880908B0490908C04A0908D044F
:10645000B0908E04840C951CA61CB71C80928B04F3
:1064600090928C04A0928D04B0928E0480902D04A2
:1064700090902E04A0902F04B09030042C013D0188
:10648000481859086A087B085301420180924D045C
:1064900090924E04A0924F04B0925004E11104C0B7
:1064A000E0918400F0918500F7FE5F9A37FF469AED
:1064B00077FF2B9AB7FF299AE0918400F09185002D
:1064C000E0918400F0918500F7FE5F9837FF4698D1
:1064D00077FF2B98B7FF29985A88552021F0809193
:1064E0008400909185002A8921502A8BE0E02111B7
:1064F00091CE80916C0490916D04A0916E04B09146
:106500006F04892B8A2B8B2B09F004C740907004F1
:10651000509071045B8A4A8A4114510409F456C7A9
:106520008091680490916904A0916A04B0916B0411
:106530004091640450916504609166047091670411
:1065400084179507A607B70708F49DC0809132010C
:10655000882309F44FC0F20185899689A789B08DF7
:10656000892B8A2B8B2B81F4818D928DA38DB48DF9
:10657000892B8A2B8B2B41F4858D968DA78DB0A10D
:10658000892B8A2B8B2BB1F1AA89BB8991966D91AE
:106590007D918D919C919497809098039090990310
:1065A000A0909A03B0909B03AB5BBF4F2C9123FF4D
:1065B00007C090958095709561957F4F8F4F9F4F45
:1065C0000E94EFEA2091BF073091C0074091C107B8
:1065D0005091C2070E944EEB9B01AC01C501B40172
:1065E0000E9406F2609398037093990380939A0334
:1065F00090939B03109271041092700410926304A4
:1066000090916A1380916B13981709F4DFC68091FB
:106610006B138F5F8F7080936B13A0EDCA2EA7E072
:10662000DA2EE12CF12C8091700490917104892B69
:1066300009F068C629DD9093710480937004892B5A
:1066400009F460C640907004509071045B8A4A8AD5
:10665000D2018C9183FF08C5C20145960E94EF19B3
:1066600010927104109270041092630490916A1356
:1066700080916B139817F1F280916B138F5F8F707D
:1066800080936B13D7CF40915F0450916004609169
:10669000610470916204481759076A077B0708F480
:1066A0000FC240915B0450915C0460915D04709155
:1066B0005E04EA89FB8985A996A9A7A9B0AD481708
:1066C00059076A077B0708F0D0C1411551056105DC
:1066D000710509F066C080909C0390909D03A09086
:1066E0009E03B0909F0389E992E1A1E0FC0105912E
:1066F000159125913491081519052A053B0558F483
:10670000B694A79497948794AA0F0496E5EBF2E1C8
:10671000E817F90759F7A0935A04F0E28F1691048D
:10672000A104B10428F4E0E28E2E912CA12CB12C0E
:1067300020E2821A9108A108B108811438E093067A
:10674000A104B10408F49AC1A4E09A9EC0011124E6
:106750008756914FFC01329625913491B82DEE2742
:10676000B39F8001B29F010D1E1F06940E1F1E1FB6
:10677000112430E020E0FC01C590D490F12CE12CF4
:10678000C01AD10AE20AF30A4C0D5D1D6E1D7F1D71
:1067900040935B0450935C0460935D0470935E04CB
:1067A00042CF00E01A81942F852E862FBC81AD81C7
:1067B000FE81EF81388529854B80E0919403E99F24
:1067C000A12DFF2730919503399FA00DF11D109049
:1067D0009603199EF00DE89DA00DF11D389DF00D5A
:1067E000E89FF00D4A2EBF2F4A9EE12D3327222726
:1067F0004F9EE00D311D201FBA9FE00D311D201F5F
:10680000BF9F300D211D432EB22F4A9E112D3327DD
:1068100022274F9E100D311D201FBA9F100D311DD4
:10682000201FBF9F300D211D432EB22FEE279091C8
:106830009C0380909D0380919E030090B504002AE4
:1068400009F483C03091B104349DE119900B800AA2
:10685000800B2091B204249DE0199109800A800BDD
:106860001091B304149D90198108800B3B9FE0198F
:106870009109800A800B2B9F90198108800B1B9F28
:10688000801881094A9E112D332722274F9E100D13
:10689000311D201FBA9F100D311D201FBF9F300DCD
:1068A000211D432EB22F3091AD04349DE10D901F78
:1068B000801E801F2091AE04249DE00D911D801E3E
:1068C000801F1091AF04149D900D811C801F3B9F71
:1068D000E00D911D801E801F2B9F900D811C801F3D
:1068E0001B9F800C811D4A9E112D332722274F9E0E
:1068F000100D311D201FBA9F100D311D201FBF9F8D
:10690000300D211D432EB22F3091A904349DE11981
:10691000900B800A800B2091AA04249DE019910914
:10692000800A800B1091AB04149D90198108800B94
:106930003B9FE0199109800A800B2B9F90198108D9
:10694000800B1B9F8018810982C03091B104349D57
:10695000E10D901F801E801F2091B204249DE00D48
:10696000911D801E801F1091B304149D900D811CF9
:10697000801F3B9FE00D911D801E801F2B9F900D5F
:10698000811C801F1B9F800C811D4A9E112D332767
:1069900022274F9E100D311D201FBA9F100D311D53
:1069A000201FBF9F300D211D432EB22F3091AD040B
:1069B000349DE119900B800A800B2091AE04249D38
:1069C000E0199109800A800B1091AF04149D901971
:1069D0008108800B3B9FE0199109800A800B2B9F57
:1069E00090198108800B1B9F801881094A9E112DE8
:1069F000332722274F9E100D311D201FBA9F100DE7
:106A0000311D201FBF9F300D211D432EB22F30910D
:106A1000A904349DE10D901F801E801F2091AA04BF
:106A2000249DE00D911D801E801F1091AB04149DCC
:106A3000900D811C801F3B9FE00D911D801E801FCB
:106A40002B9F900D811C801F1B9F800C811D11248A
:106A50004B821A83BC83AD83FE83EF8338872987FB
:106A6000982C892EB12CA82E3ECEAA89BB89D1960E
:106A70008D909D90AD90BC90D49735CED501C4013A
:106A8000B695A795979587958C7F8756954FFC016E
:106A9000C590D490FC01329625913491E82DE77091
:106AA0008E2EE29FC001E39F900D112433E0969556
:106AB00087953A95E1F7C81AD90AF12CE12C64CEF2
:106AC00040915604509157046091580470915904B4
:106AD000481759076A077B0708F030C280905104B5
:106AE00090905204A0905304B090540480915504A7
:106AF000EA89FB8981117CC0EF5BFF4FE080F18068
:106B000002811381EA89FB89E25BFF4F2081318199
:106B100042815381AA89BB89D1966D917D918D91D6
:106B20009C91D4970E94F819B1E0B0935504EA897A
:106B3000FB8941A952A963A974A989E992E1A1E05D
:106B4000FC0105911591259134910417150726072D
:106B5000370758F47695679557954795AA0F049689
:106B6000E5EBF2E1E817F90759F7A0935A04403230
:106B700051056105710520F440E250E060E070E0ED
:106B800040525109610971094115F8E05F0761053B
:106B9000710508F4B3C124E0529FC0011124875647
:106BA000914FFC01329625913491AA27439FF00121
:106BB000429FE10DFA1F0694EA1FFA1F1124AF014C
:106BC00070E060E0FC01C590D490F12CE12CC41A77
:106BD000D50AE60AF70A8C0C9D1CAE1CBF1C8092DD
:106BE000510490925204A0925304B09254041BCDCD
:106BF00081AD92ADA3ADB4AD88169906AA06BB06C9
:106C000008F072C181149104A104B10449F44091C7
:106C10009C0350919D0360919E0370919F038DCFC3
:106C2000A0E0FA85982D492D8A2DEB857C856D8510
:106C3000BE855F853889298950919403599F612DBC
:106C4000BB2730919503399F600DB11D10909603BD
:106C5000199EB00D549F600DB11D349FB00D589F0B
:106C6000B00DE62F7B2FE69F512D33272227EB9F78
:106C7000500D311D2A1F769F500D311D2A1F7B9FFD
:106C8000300D211DE32F722FE69FF12D3327222790
:106C9000EB9FF00D311D2A1F769FF00D311D2A1F2D
:106CA0007B9F300D211DE32F722F552790919C0360
:106CB00040919D0380919E030090B5040A2A09F437
:106CC00083C03091B1043E9F51199A0B4A0B8A0B35
:106CD0002091B2042E9F501991094A0B8A0BF09112
:106CE000B304FE9F901941098A0B379F50199109EF
:106CF0004A0B8A0B279F901941098A0BF79F40196D
:106D00008109E69FF12D33272227EB9FF00D311DDE
:106D10002A1F769FF00D311D2A1F7B9F300D211DEC
:106D2000E32F722F3091AD043E9F510D9A1F4A1FE1
:106D30008A1F2091AE042E9F500D911D4A1F8A1F5D
:106D4000F091AF04FE9F900D411D8A1F379F500D9B
:106D5000911D4A1F8A1F279F900D411D8A1FF79F73
:106D6000400D811DE69FF12D33272227EB9FF00D6B
:106D7000311D2A1F769FF00D311D2A1F7B9F300D7C
:106D8000211DE32F722F3091A9043E9F51199A0BB8
:106D90004A0B8A0B2091AA042E9F501991094A0B85
:106DA0008A0BF091AB04FE9F901941098A0B379F23
:106DB000501991094A0B8A0B279F901941098A0B98
:106DC000F79F4019810982C03091B1043E9F510D57
:106DD0009A1F4A1F8A1F2091B2042E9F500D911DA9
:106DE0004A1F8A1FF091B304FE9F900D411D8A1F18
:106DF000379F500D911D4A1F8A1F279F900D411DDF
:106E00008A1FF79F400D811DE69FF12D3327222712
:106E1000EB9FF00D311D2A1F769FF00D311D2A1FAB
:106E20007B9F300D211DE32F722F3091AD043E9FCB
:106E300051199A0B4A0B8A0B2091AE042E9F5019C0
:106E400091094A0B8A0BF091AF04FE9F90194109FA
:106E50008A0B379F501991094A0B8A0B279F90196B
:106E600041098A0BF79F40198109E69FF12D3327CD
:106E70002227EB9FF00D311D2A1F769FF00D311D4B
:106E80002A1F7B9F300D211DE32F722F3091A90403
:106E90003E9F510D9A1F4A1F8A1F2091AA042E9FC0
:106EA000500D911D4A1F8A1FF091AB04FE9F900D5B
:106EB000411D8A1F379F500D911D4A1F8A1F279F12
:106EC000900D411D8A1FF79F400D811D1124FA87E7
:106ED000EB877C876D87BE875F87388B298B542F24
:106EE000492F70E0682F29CE2A893B89225B3F4FCA
:106EF000D9014D915D916D917C911FCEDB01CA014D
:106F0000B695A795979587958C7F8756954FFC01E9
:106F1000C590D490FC013296259134914770429FE0
:106F2000C001439F900D1124A3E096958795AA95E3
:106F3000E1F7C81AD90AF12CE12C4DCE809133012A
:106F400090913401A0913501B0913601B7FF61C035
:106F5000EA89FB89EA5BFF4FC080D180E280F38041
:106F600089E992E121E0FC01459155916591749187
:106F70004C155D056E057F0558F4F694E794D7949B
:106F8000C794220F049645EB52E14817590759F769
:106F900020935A0450E2C516D104E104F10428F408
:106FA00070E2C72ED12CE12CF12C60E2C61AD10878
:106FB000E108F108C11478E0D706E104F10408F40F
:106FC00031C0A4E0DA9EC00111248756914FFC0124
:106FD000329625913491BC2D6627B39FA001B29FB4
:106FE000410D561F0694461F561F112470E060E0A5
:106FF000FC0185919491B0E0A0E0841B950BA60B59
:10700000B70B8093330190933401A0933501B09373
:107010003601C0903301D0903401E0903501F090FA
:10702000360101CBD701C601B695A79597958795EF
:107030008C7F8756954FFC0125913491FC01329647
:1070400045915491EC2DE770E49FC001E59F900DB0
:10705000112463E0969587956A95E1F7281B390B13
:10706000C901B0E0A0E0CDCFEA89FB898588968888
:10707000A788B08C81E081149104A104B10409F4C3
:1070800080E0AA89BB895996CD90DD90ED90FC9067
:107090005C97C114D104E104F10409F08260EA892B
:1070A000FB89458D568D678D70A141155105610590
:1070B000710509F08460809363041092510410926A
:1070C0005204109253041092540410925B041092D4
:1070D0005C0410925D0410925E04EA89FB8985A12C
:1070E00096A1A7A1B0A58093640490936504A09392
:1070F0006604B0936704442455243201481A590A9F
:107100006A0A7B0A4092410450924204609243040E
:1071100070924404409245045092460460924704A1
:10712000709248044092490450924A0460924B0481
:1071300070924C0441A052A063A074A0440C551C52
:10714000661C771C880C991CAA1CBB1C80923104FD
:1071500090923204A0923304B0923404CC0CDD1C23
:10716000EE1CFF1CC0923504D0923604E092370426
:10717000F0923804440F551F661F771F409339045F
:1071800050933A0460933B0470933C0440923D0456
:1071900050923E0460923F0470924004880F991F01
:1071A000AA1FBB1F80932D0490932E04A0932F043D
:1071B000B0933004109268041092690410926A042B
:1071C00010926B0481A592A5A3A5B4A580935F043A
:1071D00090936004A0936104B093620485A596A582
:1071E000A7A5B0A98093560490935704A093580480
:1071F000B0935904EB5BFF4F80819091EC068917A7
:1072000021F08093EC060E94D52B0E94D62F4424B7
:107210004A94542C320140923301509234016092CE
:10722000350170923601EA89FB89FD96E080F18094
:1072300002811381AA89BB89D1962D913D914D91EF
:107240005C91D4976D01BAE4CB0ED11CF60160813C
:107250007181828193810E94F81910925504D601A0
:107260004D915D916D917C9189E992E1A1E0FC01E4
:1072700005911591259134910417150726073707B5
:1072800058F47695679557954795AA0F0496E5EBC0
:10729000F2E1E817F90759F7A0935A044032510573
:1072A0006105710520F440E250E060E070E040527A
:1072B0005109610971094115F8E05F076105710520
:1072C00008F462C024E0529FC00111248756914FF8
:1072D000FC01329625913491AA27439FF001429FE9
:1072E000E10DFA1F0694EA1FFA1F1124AF0170E0A6
:1072F00060E0FC01C590D490F12CE12CC41AD50AB1
:10730000E60AF70AC0926C04D0926D04E0926E0413
:10731000F0926F0480916C0490916D04A0916E04C2
:10732000B0916F04AC01BD01009731E0A307B10536
:1073300020F04FEF5FEF60E070E0841B950BA60B31
:10734000B70B80936C0490936D04A0936E04B0937C
:107350006F04F89480918400909185004096A981F3
:10736000A150A983AA2381F1240E351E28163906BF
:1073700010F40C94A93030928900209288007894FF
:107380006396E2E10C94EBF1DB01CA01B695A79597
:10739000979587958C7F8756954FFC01C590D49023
:1073A000FC013296259134914770429FC001439F62
:1073B000900D112433E0969587953A95E1F7C81A18
:1073C000D90AF12CE12C9ECF1C01D5CF80EDC82E1F
:1073D00087E0D82EE12CF12C2DC9CF93DF9380913B
:1073E0006A1390916B13891B80958F7019F40E941A
:1073F000B08FF5CF80916A138F5F8F70A0916A1361
:107400009BE5A99FD0011124FD01ED53F84FEF0139
:1074100019929A95E9F798E09083A852B84F90E1B5
:10742000ECE6F3E101900D929A95E1F720916A1351
:1074300090916B13291303C094E690936713809384
:107440006A130E94B42FDF91CF910895FC0120812F
:107450003181428153816091940D7091950D80919D
:10746000960D9091970D0E944EEB0E946FF36093E2
:1074700078137093791380937A1390937B13909180
:107480006A1380916B13981709F0A7CF0E94D32C31
:107490000E94A72F409178135091791360917A132D
:1074A00070917B1340938B0450938C0460938D04F4
:1074B00070938E0481110C94B42F08954F925F92B3
:1074C0006F927F928F929F92AF92BF92CF92DF92F4
:1074D000EF92FF92CF93DF93EC012091940D3091C6
:1074E000950D4091960D5091970D6C857D858E85FB
:1074F0009F850E944EEB0E946FF36B017C012091EF
:10750000900D3091910D4091920D5091930D6885A1
:1075100079858A859B850E944EEB0E946FF34B0113
:107520005C0120918C0D30918D0D40918E0D50910C
:107530008F0D6C817D818E819F810E944EEB0E9418
:107540006FF32B013C012091880D3091890D409102
:107550008A0D50918B0D688179818A819B810E946F
:107560004EEB0E946FF360936C1370936D138093D6
:107570006E1390936F134092701350927113609238
:107580007213709273138092741390927513A09279
:107590007613B0927713C0927813D0927913E09259
:1075A0007A13F0927B1390916A1380916B13981762
:1075B00081F013DFDF91CF91FF90EF90DF90CF90BC
:1075C000BF90AF909F908F907F906F905F904F9003
:1075D00008950E94D32C0E94A72FC82F8CE693E118
:1075E0000E94EF19CC2331F30E94B42FE3CFCF9246
:1075F000DF92EF92FF92CF93DF93C82F0E94A72FC5
:1076000094E0C99FE0011124FE01E158FB4FC080C6
:10761000D180E280F38081110E94B42FCD54D84FE5
:10762000C701B6010E94EFEA288139814A815B8156
:107630000E944EEBDF91CF91FF90EF90DF90CF90C3
:1076400008958F929F92AF92BF92CF92DF92EF9266
:10765000FF921F93CF93DF93CDB7DEB760970FB63E
:10766000F894DEBF0FBECDBF182F80E0C0DF4B0106
:107670005C018092050490920604A0920704B092E7
:10768000080481E0B4DF6B017C01C0920904D09250
:107690000A04E0920B04F0920C0482E0A8DF6093ED
:1076A0000D0470930E0480930F04909310041D86B4
:1076B0001E861F86188A89829A82AB82BC82CD82FE
:1076C000DE82EF82F88669877A878B879C8783E0E2
:1076D0008EDF6D877E878F87988BCE0101960E9403
:1076E000F52C1E3FD9F480E1FE013196AAE7B1E006
:1076F00001900D928A95E1F760960FB6F894DEBF7F
:107700000FBECDBFDF91CF911F91FF90EF90DF9023
:10771000CF90BF90AF909F908F90089584E0189F76
:10772000F0011124DF01A658BE4F81E090E08C0FDC
:107730009D1FE80FF91F40815181628173814D9334
:107740005D936D937C931397D7CFCF92DF92EF9297
:10775000FF92CF93DF93C82F0E94A72F94E0C99F79
:10776000E0011124FE01ED58FB4FC080D180E28082
:10777000F38081110E94B42FCD54D84FC701B601B8
:107780000E94EFEA288139814A815B810E944EEB99
:10779000DF91CF91FF90EF90DF90CF900895A1E01F
:1077A000B0E0E5EDFBE30C94DFF1898360E0CE010E
:1077B00001960E944A1B61E0CE0101960E944A1B7D
:1077C00062E0CE0101960E944A1B89812196E2E087
:1077D0000C94FBF1A2E1B0E0E0EFFBE30C94DBF1F1
:1077E000DEDF8823C1F1EDB6FEB646E952E082FF46
:1077F00002C04DE852E026E932E081FF02C02FE8E6
:1078000032E080FD25C086E992E05F934F933F937D
:107810002F939F938F938AE297E09F938F938E018C
:107820000F5F1F4F1F930F930E9482EA0E94018BEC
:10783000C8010E948284C8010E944EC60FB6F89407
:10784000DEBF0FBECDBF81E06296E6E00C94F7F19B
:1078500081E992E0DACF80E0F7CFA0E2B0E0E3E3A5
:10786000FCE30C94CFF180911201882309F4BEC08F
:1078700080911704082F10E080FF3CC0C0901401D5
:10788000D0901501E0901601F09017012091A90207
:107890003091AA024091AB025091AC02C701B601EF
:1078A0000E946AF3181644F4C092A902D092AA0268
:1078B000E092AB02F092AC02C0902001D090210186
:1078C000E0902201F09023012091A9023091AA02B8
:1078D0004091AB025091AC02C701B6010E94E9EAA7
:1078E00087FF08C0C092A902D092AA02E092AB0220
:1078F000F092AC0201FF3CC0C0901801D090190179
:10790000E0901A01F0901B012091AD023091AE027F
:107910004091AF025091B002C701B6010E946AF3D4
:10792000181644F4C092AD02D092AE02E092AF02BB
:10793000F092B002C0902401D0902501E090260181
:10794000F09027012091AD023091AE024091AF023C
:107950005091B002C701B6010E94E9EA87FF08C052
:10796000C092AD02D092AE02E092AF02F092B002AD
:1079700002FF3CC0C0901C01D0901D01E0901E0190
:10798000F0901F012091B1023091B2024091B302F8
:107990005091B402C701B6010E946AF3181644F46C
:1079A000C092B102D092B202E092B302F092B4025D
:1079B000C0902801D0902901E0902A01F0902B017D
:1079C0002091B1023091B2024091B3025091B402C1
:1079D000C701B6010E94E9EA87FF08C0C092B10260
:1079E000D092B202E092B302F092B4028091730D91
:1079F00083FD61C02091860130918701409188010B
:107A0000509189016091B5027091B6028091B702E0
:107A10009091B8020E94E9EA882309F44CC00E94C0
:107A2000A1B7182F882331F00E94018B8FE097E0D7
:107A30000E949184209186013091870140918801B4
:107A4000509189016091B5027091B6028091B702A0
:107A50009091B8020E9406F29F77209174013091B4
:107A6000750140917601509177010E944EEB20E024
:107A700030E046E154E40E946AF31816D4F40E9400
:107A8000018B80EF96E00E9491848091B5029091E5
:107A9000B602A091B702B091B8028093860190938C
:107AA0008701A0938801B093890185EB92E0CEDC39
:107AB00002C01111EACF2AE037ED43E25CE36091A6
:107AC0000C0170910D0180910E0190910F010E94A7
:107AD0004EEB6B017C016091100170911101072E3A
:107AE000000C880B990B0E94EFEA9B01AC01C701C7
:107AF000B6010E944EEB698B7A8B8B8B9C8B8091AD
:107B0000B902882309F18090BA029090BB02A0903C
:107B1000BC02B090BD02C090B102D090B202E09021
:107B2000B302F090B40220E030E0A901C501B40135
:107B30000E94E9EA8823F9F0A7019601C501B40182
:107B40000E946AF31816BCF020E030E0A901BE01E3
:107B50006F5E7F4F89EA92E00E94C2C780E1E9EA46
:107B6000F2E0AAE7B1E001900D928A95E1F7A096C4
:107B7000E2E10C94EBF120917A0130917B0140918C
:107B80007C0150917D016091A9027091AA028091BF
:107B9000AB029091AC020E9406F24B015C01209175
:107BA0007E0130917F01409180015091810160916F
:107BB000AD027091AE028091AF029091B0020E942E
:107BC00006F26D8B7E8B8F8B988F20918201309186
:107BD00083014091840150918501C701B6010E9443
:107BE00006F26D8F7E8F8F8F98A320918601309142
:107BF000870140918801509189016091B50270918F
:107C0000B6028091B7029091B8020E9406F2698F85
:107C10007A8F8B8F9C8F20E030E0A901C501B401E1
:107C20000E94E9EA81110CC020E030E0A9016D89D1
:107C30007E898F89988D0E94E9EA882309F484CF90
:107C4000A5019401C501B4010E944EEB6B017C01BA
:107C50002D893E894F89588DCA01B9010E944EEB8A
:107C60009B01AC01C701B6010E9407F26B017C01C8
:107C70002D8D3E8D4F8D58A1CA01B9010E944EEB4A
:107C80009B01AC01C701B6010E9407F26B017C01A8
:107C9000298D3A8D4B8D5C8DCA01B9010E944EEB46
:107CA0009B01AC01C701B6010E9407F26B017C0188
:107CB0000E94A3F32B013C012CEC3CEB4CE85BE273
:107CC000C701B6010E94E9EA87FF06C0498C5A8CB9
:107CD0006B8C7C8CE89477F82DEB37E346E855E322
:107CE000C301B2010E94E9EA87FD38CF2DEC3CECDC
:107CF0004CE45EE3C301B2010E944EEB0E94EBF242
:107D00001B01672B19F422242394312CB10190E03C
:107D100080E00E94EDEA9B01AC0160E070E080E849
:107D20009FE30E947EF26B017C01AC019B01C301C9
:107D3000B2010E944EEB2B013C01A7019601C50147
:107D4000B4010E944EEB4B015C01A70196016D89C5
:107D50007E898F89988D0E944EEB6D8B7E8B8F8BE9
:107D6000988FA70196016D8D7E8D8F8D98A10E94B1
:107D70004EEB6D8F7E8F8F8F98A3A7019601698D33
:107D80007A8D8B8D9C8D0E944EEB698F7A8F8B8FB5
:107D90009C8F80E1EAE7F1E08E010F5F1F4FD80171
:107DA00001900D928A95E1F70E94EBD16B017C0165
:107DB00028ECC20ED11CE11CF11C81E0281A31080C
:107DC00009F454C00E94EBD19B01AC012C193D0970
:107DD0004E095F0957FD4DC06B017C0128ECC20EB6
:107DE000D11CE11CF11C80E00E94B08FA501940120
:107DF00069817A818B819C810E9407F269837A83F1
:107E00008B839C832D893E894F89588D6D817E811E
:107E10008F8198850E9407F26D837E838F83988778
:107E20002D8D3E8D4F8D58A169857A858B859C85DA
:107E30000E9407F269877A878B879C87298D3A8D04
:107E40004B8D5C8D6D857E858F8598890E9407F2AC
:107E50006D877E878F87988BA3019201BE016F5E2D
:107E60007F4FC8010E94C2C78111A7CFA301920111
:107E70006ECE0E94152ABACF8091130490911404FB
:107E8000A0911504B091160480930C0190930D01FC
:107E9000A0930E01B0930F018091110490911204F0
:107EA0009093110180931001089580910C0190919D
:107EB0000D01A0910E01B0910F01809313049093D6
:107EC0001404A0931504B0931604809110019091AE
:107ED0001101909312048093110484E690E0909332
:107EE0001101809310010895ACE0B0E0EAE7FFE3F0
:107EF0000C94D1F12B013C0129873A874B875C8791
:107F000047015801D601CD90DD90ED90FC9020E026
:107F100030E0A901C701B6010E94E9EA811171C0F0
:107F20008091700190917101A0917201B0917301E3
:107F300089839A83AB83BC8320E030E0A901C70129
:107F4000B6010E94E9EA811106C0C12CD12C80E85B
:107F5000E82E80E4F82ECD82DE82EF82F886A5013D
:107F600094016091820170918301809184019091CC
:107F700085010E94E9EA87FF0CC0809282019092FD
:107F80008301A0928401B0928501CE0105960E94E2
:107F9000902240927A0150927B0160927C01709213
:107FA0007D0189859A85AB85BC8580937E01909300
:107FB0007F01A0938001B0938101CE0101960E94C0
:107FC0009022A501940160918201709183018091BA
:107FD0008401909185010E946AF3181664F48092DE
:107FE000820190928301A0928401B0928501CE011A
:107FF00005960E9490220E94D32C2C96E0E10C94CE
:10800000EDF1D701C60194CFCF92DF92EF92FF92AC
:108010000F931F936B01FC01E080F18002811381BB
:10802000EAE7F1E0248135814681578160817181E1
:108030008281938159DF1F910F91FF90EF90DF9024
:10804000CF9008950C94E5C70F931F93CF93DF93C0
:10805000EC018B010E947A8E882331F081E0DF9160
:10806000CF911F910F910895B801CE01CDDF80917E
:108070003107C82FC47082FD0AC01092310782E018
:10808000E0DAE0DF81E0CC2351F380E0E8CF0E942A
:10809000398E882391F3E2CFCF930E94A72FC82F68
:1080A00080916B1380936A13809369138093681394
:1080B00084E6809367130E94383080ED93E09093BC
:1080C000BD0D8093BC0DC1110E94B42F81E080933F
:1080D00072040E94D32C8EEFB4DAB4DFCF910895EE
:1080E000ACE0B0E0E6E7F0E40C94DFF10E9460B7AA
:1080F0000E94A72F9CE0EFE7F4E0DE0111960190CB
:108100000D929A95E1F781110E94B42FCE0101964C
:108110000E944D2B2C96E2E00C94FBF1B0E0A0E025
:10812000E4E9F0E40C94D1F140907A0150907B01A5
:1081300060907C0170907D0180907E0190907F0125
:10814000A0908001B0908101C0908201D090830105
:10815000E0908401F09085010E94672C60912C01D1
:1081600070912D01072E000C880B990B0E94EFEAED
:108170002AE037ED43E25CE30E944EEB609374012A
:1081800070937501809376019093770104E111E07B
:10819000D0E0C0E0CE01835B954F0E94B477F80138
:1081A00061937193819391938F01CE018F5B954F72
:1081B0000E94B477F801608771878287938724963D
:1081C000CC30D10539F760E085E294E00E94957AE1
:1081D0000E94627B0E94AB2CA301920160917A0104
:1081E00070917B0180917C0190917D010E94E9EA70
:1081F00081111BC0A501940160917E0170917F01E6
:1082000080918001909181010E94E9EA81110DC065
:108210002091820130918301409184015091850128
:10822000C701B6010E94E9EA81115ADFCDB7DEB776
:10823000E0E10C94EDF1A4E0B0E0E1E2F1E40C94B3
:10824000DFF184EF91E0A0E0B0E089839A83AB8313
:10825000BC83BE016F5F7F4F8CE30E94388386ED45
:1082600096E00E94918486B160ED76E082FB8827DB
:1082700080F90E94EA2186B16AEC76E083FB8827C8
:1082800080F90E94EA2186B164EC76E082958170E3
:108290000E94EA2180B16BEB76E082FB882780F9AF
:1082A0000E94EA21349907C00E946C832496E2E080
:1082B0000C94FBF106C00E9455832496E2E00C94D6
:1082C000FBF18091EB06811103C08091ED068111D5
:1082D0000C94D62F0895ACE0B0E0E1E7F1E40C9403
:1082E000DFF1A4E7BDE090E080E0FC01E757F54F47
:1082F00045915591659174914D935D936D937D93E7
:10830000FC01E758F54F4591559165917491509650
:108310004D935D936D937C935397FC01E759F54F13
:10832000459155916591749190964D935D936D93A0
:108330007C939397049680319105B9F680E29EE490
:10834000A0E0B0E08093840D9093850DA093860DFE
:10835000B093870D80E090E0AAEFB3E48093A80D7E
:108360009093A90DA093AA0DB093AB0D8093AC0D83
:108370009093AD0DA093AE0DB093AF0D8093B00D63
:108380009093B10DA093B20DB093B30D1092B40DB4
:108390001092B50D1092B60D1092B70D1092B80D47
:1083A0001092B90D1092BA0D1092BB0D8AE097EDA4
:1083B000A3EABDE38093960790939707A09398074D
:1083C000B0939907109232010E94716A80E090E0A8
:1083D000A0EEB0E480932E0190932F01A093300182
:1083E000B093310180E090E0A0E2B1E480932504F5
:1083F00090932604A0932704B09328040E944B7AFC
:108400008CE0EAE8F1E0DE01119601900D928A9588
:10841000E1F789819A81AB81BC8180935913909354
:108420005A13A0935B13B0935C138D819E81AF812F
:10843000B88580935D1390935E13A0935F13B09300
:10844000601389859A85AB85BC8580936113909371
:108450006213A0936313B09364138EEB90E0909338
:108460004F0780934E078CE390E0909351078093E1
:108470005007109253071092520786EE90E09093A7
:1084800055078093540786E490E0909357078093B4
:10849000560710925907109258078FE892ECADE8F2
:1084A000B1E48093C0129093C112A093C212B09312
:1084B000C3128CE998EFA5E4BEE38093C4129093B5
:1084C000C512A093C612B093C71281E49CEBABEC2B
:1084D000B3E48093C8129093C912A093CA12B093C8
:1084E000CB1280E090E0AFEAB3E480934207909330
:1084F0004307A0934407B093450785E996E2A5E2B8
:10850000B1E48093460790934707A0934807B09340
:10851000490780EA9CE6ACE2B5E480934A07909371
:108520004B07A0934C07B0934D071092EB061092A7
:10853000EA06C7DEF3DD2C96E2E00C94FBF1CBCE2D
:10854000A4E0B0E0E6EAF2E40C94D0F19091ED06FC
:10855000981709F455C0382E80E090E0A0E2B1E40D
:1085600089839A83AB83BC83C0906113D0906213DC
:10857000E0906313F090641320E030E0A901C7019C
:10858000B6010E94E9EA87FF0CC0A701960160E0EE
:1085900070E080E291E40E9406F269837A838B8323
:1085A0009C83CE0101960E9476C840907A0150903B
:1085B0007B0160907C0170907D0180907E019090A5
:1085C0007F01A0908001B09081013320F1F00E94E2
:1085D0007A8E19821A821B821C82E0908201F090AE
:1085E00083010091840110918501CE0101966C01F7
:1085F000A5019401C301B20177DC3092ED0661DE82
:1086000080E02496E1E10C94ECF10E94398EE1CFF8
:10861000B0E0A0E0EEE0F3E40C94D1F1C82FE82E36
:10862000F12CF701EB50F24DD491823071F481E0DE
:1086300087DF811105C00E947A8E882309F4E2C089
:10864000CDB7DEB7E0E10C94EDF16D2FDD0F770BC8
:10865000880B990B0E94EFEA2B013C01C701880FA0
:10866000991F880F991F8758984F0E94B4774B0124
:108670005C01A3019201C501B4010E944EEB4B01C4
:108680005C016701CC0CDD1CCC0CDD1CC6018359E0
:10869000984F0E94B477A30192010E944EEB20E014
:1086A00030E040EC5FE30E944EEBAB01BC0100E028
:1086B00010E098018C2F0E94ACCBC23009F0CCC0E6
:1086C0000E94398E20E030E0A901C501B4010E946A
:1086D000E9EA882329F100E010E020E830E4B50160
:1086E000A40170588C2F0E94ACCBC23009F467C033
:1086F000A5019401C501B4010E9407F24B015C0180
:10870000C23009F062C000E010E020E030E4B501C2
:10871000A4018C2F0E94ACCBC23011F40E94398E80
:1087200081E090E00C2E01C0880F0A94EAF7909146
:108730008207982B9093820790911704892B80933E
:108740001704C6018F59984F0E94B477F601E65876
:10875000FE4F6083718382839383C230D1F4209172
:1087600061133091621340916313509164136091CF
:1087700082017091830180918401909185010E9412
:1087800006F2609382017093830180938401909339
:10879000850158DCF601E755FD4FD601A658BE4FBE
:1087A0008D919D910D90BC91A02D80839183A2838A
:1087B000B383C23009F044CF80E0C2DE41CF0E94D3
:1087C0007A8E882309F494CF3BCFF701E25AF84F11
:1087D0006491611107C00E94018B8CE397E00E94B5
:1087E00091846AE070E090E080E00E94EDEA9B01F5
:1087F000AC0161E070E088E492E40E947EF28B01BB
:108800009C0185CF81E897E00E94B47720E030E0BA
:10881000A9010E94E9EA882309F417CF6D2FDD0F23
:10882000770B880B990B0E94EFEA2B013C0181E842
:1088300097E00E94B4774B015C0120E030E040EA11
:1088400050E40E946AF387FF14CF812C912C90EAA8
:10885000A92E90E4B92E0DCF20E030E0A901C5018A
:10886000B4010E94E9EA882309F45ACF00E010E03D
:10887000980135CF80913107882319F01092310784
:10888000089540E070E060E08BE996E00E94C18EC0
:108890001F920F920FB60F9211240BB60F922F93C7
:1088A0003F934F935F936F937F938F939F93AF9378
:1088B000BF93EF93FF930E94D62FFF91EF91BF914B
:1088C000AF919F918F917F916F915F914F913F9168
:1088D0002F910F900BBE0F900FBE0F901F90189509
:1088E0000F931F9380919207813019F50E94EBD16D
:1088F0000091FC031091FD032091FE033091FF03D2
:10890000601B710B820B930B28EE33E040E050E0CC
:108910000E9417F16091F8037091F9038091FA03B6
:108920009091FB03620F731F841F951F1F910F917E
:108930000895609100047091010480910204909167
:108940000304D6CF109292071092FC031092FD03FD
:108950001092FE031092FF03109200041092010483
:1089600010920204109203041092F8031092F9037B
:108970001092FA031092FB030895809192078130C0
:10898000E1F08230C1F4ACDF6093F8037093F90337
:108990008093FA039093FB0381E0809392070E94F7
:1089A000EBD16093FC037093FD038093FE039093DF
:1089B000FF0381E00895C6DFEFCF80E008950E94B5
:1089C000C4C80E94FC7B882351F08091D41482FD9E
:1089D00006C087EE91E09093F0068093EF06CDCF2E
:1089E00080919207813079F482E0809392070E940F
:1089F000EBD1609300047093010480930204909380
:108A0000030481E0089580E00895809192078150E9
:108A1000823070F4109292070E94EBD160930004B0
:108A200070930104809302049093030481E00895FD
:108A300080E008952091BD123091BE122635310597
:108A40003CF420913F0730914007263031051CF05F
:108A5000882331F092CF662319F0D7DF0C94C4C875
:108A600008959C0197FF26C0EE27FF27E81BF90B0E
:108A70002D398FEF38070CF05DC08DE28093A40292
:108A8000CF0164E670E00E94A1F1CB012AE030E062
:108A9000B9010E94A1F1805D8093A502CF01B901C7
:108AA0000E94A1F1CB01B9010E94A1F1805D8093E8
:108AB000A6022AC0283E83E03807B4F1C90168EE57
:108AC00073E00E94A1F1CB01EAE0F0E0BF010E9457
:108AD000A1F1805D8093A402C90164E670E00E9468
:108AE000A1F1CB01BF010E94A1F1805D8093A5029D
:108AF000C901BF010E94A1F1CB01BF010E94A1F1F8
:108B0000805D8093A602F901CF016AE070E00E94C7
:108B1000A1F1805D8093A70284EA92E008958DE23E
:108B200037FDC5CF80E2C3CFF90180E2243631059D
:108B30000CF0A4CF80E28093A4028093A502EA30D7
:108B4000F1056CF38DE237FF80E28093A502CF013F
:108B50006AE070E00E94A1F1605D6093A602D4CF4C
:108B60009C0197FD2DC080E2243631055CF0C901DF
:108B700064E670E00E94A1F1CB016AE070E00E941F
:108B8000A1F1805D8093A50280E22A3031055CF07E
:108B9000EAE0F0E0C901BF010E94A1F1CB01BF01F1
:108BA0000E94A1F1805D8093A602C9016AE070E095
:108BB0000E94A1F1805D8093A70285EA92E008956A
:108BC0003195219531098DE2DDCFCF92DF92EF9281
:108BD000FF92FC01C080D180E280F38020E030E091
:108BE000A901C701B6010E94E9EA87FD26C06DEB25
:108BF00077E386E095E3A70196010E9407F26B01F7
:108C00007C0120E030E0A9010E94E9EA20E030E0A8
:108C100040E05FE387FF04C020E030E040E05FEB2E
:108C2000C701B6010E9407F20E94E6F2CB0198DF6D
:108C3000FF90EF90DF90CF9008956DEB77E386E0A3
:108C400095EBD9CFA4E0B0E0E8E2F6E40C94DFF1D4
:108C50000E94EFEA69837A838B839C83CE0101961D
:108C6000B4DF2496E2E00C94FBF1FC016081718199
:108C7000828193810E94E6F2CB0172CFA4E0B0E042
:108C8000E4E4F6E40C94DFF10E94EFEA69837A836E
:108C90008B839C83CE010196E8DF2496E2E00C945E
:108CA000FBF18F929F92AF92BF92EF92FF920F9340
:108CB0001F93CF93DF93EC018B01E42EF22E809172
:108CC0007C1390917D138C179D07C9F123E6CB3758
:108CD000D20709F03FC08A509C4771F40E94EBD143
:108CE0006E517B4F8F4F9F4F6093E8037093E90362
:108CF0008093EA039093EB03D0937D13C0937C138E
:108D000030E020E0009375071093760720937707F3
:108D100030937807E0927007F0927107CA50DC47F1
:108D200021F41092A0021092E70382E080936F0179
:108D300081E08093720710929F021092F303DF91FB
:108D4000CF911F910F91FF90EF90BF90AF909F90A8
:108D50008F9008952CE7CA30D20771F68B5793464F
:108D6000D9F40E94EBD18090E8039090E903A090A1
:108D7000EA03B090EB03681979098A099B0997FF08
:108D80000BC0809182078770873031F40E9467237F
:108D9000C5E1D8E58111B0CFCAE0DCE7ADCF20E076
:108DA00040E070E060E086E593E27BCF0E94A1B7EF
:108DB000882339F020E040E070E060E087E397E549
:108DC00070CFEDCF21E02093A002FC018081918142
:108DD000A281B3818093080190930901A0930A01B5
:108DE000B0930B0120E040E070E060E080915F070D
:108DF0009091600756CFA4E0B0E0E1E0F7E40C9476
:108E0000DFF18DEC9CECACECBCE389839A83AB8303
:108E1000BC83CE010196D6DF2496E2E00C94FBF1F0
:108E2000A4E0B0E0E6E1F7E40C94DFF18DEC9CEC1B
:108E3000ACECBDE389839A83AB83BC83CE010196FE
:108E4000C1DF2496E2E00C94FBF1A4E0B0E0EBE299
:108E5000F7E40C94DFF180E090E0A0E8BFE38983C1
:108E60009A83AB83BC83CE010196ACDF2496E2E00B
:108E70000C94FBF1A4E0B0E0E0E4F7E40C94DFF143
:108E800080E090E0A0E2B1E489839A83AB83BC8365
:108E9000CE01019697DF2496E2E00C94FBF181E08D
:108EA0008093A002809182078770873051F01092E2
:108EB00082071092170485E096E09093F006809365
:108EC000EF068091B9028093F50380E00E94097A51
:108ED00020E040E070E060E08FE697E4E2CE809131
:108EE0006F01882331F041E062EA73E082E00E9482
:108EF00059CC809117048770873071F41092F40375
:108F000020E040E070E060E087EB97E5CADE81E0BA
:108F10008093F3030C949822089520E040E070E0E1
:108F200060E08AE09CE7BDCE1092B2070E9435282F
:108F3000F4CFB0E0A0E0EFE9F7E40C94D9F1CDB6BE
:108F4000DEB6E5E8F7E0DF010D900020E9F7CD019E
:108F50008D5797402DB73EB7281B390B0FB6F894A5
:108F60003EBF0FBE2DBF0DB71EB70F5F1F4FFF9344
:108F7000EF9388E695E09F938F931F930F930E9442
:108F800082EA780134E0E30EF11C0F900F900F900D
:108F90000F900F900F90D7018D917D01882349F09C
:108FA000082E000C990B0E94E8F3F701319780839B
:108FB000F2CF63E675E0C8010E941BEA4FE350E080
:108FC000B80181EF96E00E9440F40FB6F894DEBE3F
:108FD0000FBECDBEA2DF0E94C4C8E8E00C94F5F13C
:108FE0008093330720E040E070E060E085ED97E596
:108FF00058CEA1E8B0E0EFEFF7E40C94CFF1ADB6B6
:10900000BEB684E690E09093A9128093A8121092C5
:10901000CD121092CC1241E064E070E0CE0187588E
:109020009F4F0E94A8B643E050E0BE0167587F4FB3
:109030008BE292E00E9432F4892BF9F0ED968FAD2D
:10904000ED97882339F08FE3EA968FAFEA97EB9696
:109050001FAEEB9782E0C4DF81E0809324049091FF
:10906000240481E089270FB6F894BEBE0FBEADBEC2
:10907000CF57DF4FE2E10C94EBF141E062E070E0AA
:10908000CE0183589F4F0E94A8B6E9961CAE1DAE34
:109090001EAE1FAEE9971092CD121092CC12CE01E7
:1090A0008F579F4F0E9466226DB67EB6CF57DF4F17
:1090B000C880C158D040D12C23E0C20ED11CCC0CAA
:1090C000DD1CCC0CDD1C8DB79EB78C199D090FB62D
:1090D000F8949EBF0FBE8DBFEDB7FEB731964F011E
:1090E0008C199D090FB6F8949EBF0FBE8DBF0DB7AA
:1090F0001EB70F5F1F4FEDB7FEB7EC19FD090FB696
:10910000F894FEBF0FBEEDBF8DB79EB701967C01F0
:10911000B601C4010E946B224091920381E048276E
:1091200064E070E084E89DE00E94A8B6B601C80142
:109130000E946B22B601C7010E946B2280919203AC
:1091400081114BC0CF57DF4F8881C158D04090E08C
:109150000296A4E7BDE050E040E030E020E065E9A1
:109160007AE0E5E8CE2EEAE0DE2E821793070CF4D3
:10917000B2C0F401E40FF51F20803180428053809B
:109180002D923D924D925D92821793070CF4A9C0E7
:10919000F801E40FF51F2080318042805380509603
:1091A0002D923D924D925C925397821793070CF447
:1091B0009EC0F701E40FF51F20803180428053806C
:1091C00090962D923D924D925C9293972F5F3F4FD8
:1091D0004C5F5F4F2430310541F688EA9DE00E94E4
:1091E0003E228CEA9DE00E943E2280EB9DE00E94A0
:1091F0003E2284EB9DE00E943E2288EB9DE00E948F
:109200003E22CE018B589F4F0E943E22CE018B58AA
:109210009F4F0E943E22CE018B589F4F0E943E22BC
:10922000CE018B589F4F0E943E2286E997E00E9414
:109230003E220FB6F8947EBE0FBE6DBE8E010F5F4C
:109240001F4FC8010E945E22CE0183599F4F0E948A
:109250004622AE968FADAE9791E018160CF090E0D6
:1092600090933201181614F40E94716AC8010E948A
:109270003E22D0909203D1100CC089819A81AB819B
:10928000BC8180932E0190932F01A0933001B09365
:10929000310185E294E00E943E22CE018B589F4F1F
:1092A0000E943E22CE0183599F4F0E946622C80130
:1092B0000E946622AE96EFACAE978981E89E70015F
:1092C000112491E0E91AF108C8F0CE018B589F4FA4
:1092D0000E943E22F6CFFB01259035904590549098
:1092E0004FCFF601259035904590549058CFE5E743
:1092F000FAE0259035904590549062CF89E593E14E
:109300000E945E228AE0F82EFA94CE01FF2029F016
:109310008B589F4F0E943E22F7CF80589F4F0E944C
:109320006622CE0181589F4F0E946622C058DF4FAF
:109330008881C058D040873009F059C1C158DF4FEB
:109340008881CF57D040873009F051C1D11003C078
:1093500080E00E94097A8AE893E00E94562282E81F
:1093600093E00E9456224091920381E0482764ECEA
:1093700070E08EEB92E00E94A8B6C8010E944E22D7
:10938000CE0183599F4F0E94462240919203FF24B1
:10939000F3944F2564E070E0C8010E94A8B68EEEF9
:1093A00096E00E944E22409192034F256CE070E0BF
:1093B0008EE497E00E94A8B6409192034F2564E1A5
:1093C00070E0C8010E94A8B6F0909203F11030C07E
:1093D00089819A81AB81BC818093C0129093C11224
:1093E000A093C212B093C3122CEA35EC47E25EE3BD
:1093F0006D817E818F8198850E944EEB6093C412AF
:109400007093C5128093C6129093C71220E030E586
:1094100043EC50E469857A858B859C850E944EEBF0
:109420006093C8127093C9128093CA129093CB12A2
:1094300041E04F2562E070E0C8010E94A8B6C80173
:109440000E943622E0909203E11030C089819A8117
:10945000AB81BC818093420790934307A09344075C
:10946000B09345072CEA35EC47E25EE36D817E81DF
:109470008F8198850E944EEB609346077093470753
:10948000809348079093490720E030E543EC50E48F
:1094900069857A858B859C850E944EEB60934A078F
:1094A00070934B0780934C0790934D07C8010E941F
:1094B0003622C8010E944622C8010E944622C801E5
:1094C0000E94462285E0F80111928A95E9F7FF246F
:1094D000F3944E2D4F2565E070E0C8010E94A8B6B8
:1094E000C8010E944E22409192034F2560E270E035
:1094F000C8010E94A8B6CE0183599F4F0E944E22F8
:10950000409192034F2569E070E0C8010E94A8B61F
:10951000409192034F2562E170E0C8010E94A8B615
:10952000409192034F2564E270E0C8010E94A8B602
:10953000409192034F2560E170E0C8010E94A8B6F7
:10954000409192034F2569E070E0C8010E94A8B6DF
:10955000C8010E943E22409192034F256CE070E0CA
:10956000C8010E94A8B6409192034F256CE670E0B6
:10957000C8010E94A8B619821A821B821C821D8211
:109580001E821F82188619861A861B861C86C801B1
:109590000E943622409192034F2568E070E0C80196
:1095A0000E94A8B6C8010E945E22CE0181589F4F3A
:1095B0000E944622CE0183599F4F0E943E228091F5
:1095C000A8129091A9128037934089F51092240433
:1095D0002091CC123091CD12EF968EAD9FADEF97CA
:1095E0002817390741F1F092240480E023C0CE010E
:1095F00083599F4F0E945622C8010E945622C0588C
:10960000DF4FE880C058D040C158DF4F8881CF5726
:10961000D040E89E70011124F1E0EF1AF10808F43F
:10962000ACCECE018B589F4F0E943E22F5CFF092D8
:10963000240481E0D5DC80919203811110CD8091CA
:10964000240481110CCD0E948E4009CD81E08093CD
:109650009203CFDC10929203882309F0CACC0E94B7
:109660006B4180E00895F2CFCF93DF93C091E70381
:10967000CC23B1F0C150C093E70389E0C89FE0015B
:109680001124CF54DC4F6A817B812F814E818881E8
:10969000998107DB88858093A002DF91CF9108959F
:1096A0003CDCFBCFA4E0B0E0E8E5FBE40C94D2F1B5
:1096B0000E946DCDF09070076F2C85E0782E7F0CA6
:1096C00086E0E82EEF1885E0D82EDF18AA24AA94A9
:1096D000B12C84E0C82ECF1882E0982E9F1881E02C
:1096E000882E8F185F2C5194F1105AC08091730707
:1096F000882309F444C080916F01882359F081E0E8
:1097000090917307911180E024E046E956E0652DC1
:109710000E94B9CC8091B2078093330724E0F21203
:10972000F7C010927F0780917307843009F4DDC081
:1097300080916F018823E1F011E0809173078430FC
:1097400009F010E08091330724E6829FC0011124C4
:1097500081589F4FB5010E94A1F1862F0E941D1DC7
:1097600000E09C014BE756E06C2D812F0E94B27502
:10977000F394F710B9CF87E0809371070DC0809103
:109780005A0710925A07882309F4B5CF6DDF8091EC
:109790007207882309F4AFCF2496EFE00C94EEF122
:1097A00021E0F21243C080917307813041F1809132
:1097B0006F018823F9F011E080917307813009F07F
:1097C00010E06091100170911101072E000C880BC0
:1097D000990B0E94EFEA69837A838B839C83CE0185
:1097E000019643DA00E09C0140E956E0682D812FA4
:1097F0000E94B2758091B20780933307B9CF8091F0
:109800005A0710925A07882391F210E000E027EEE1
:1098100033E04AE050E060E171E080E996E00E94C8
:1098200032CE80917207882311F2B6CF82E0F8120F
:10983000D7C080917307823021F180916F01882316
:10984000C9F211E080917307823009F010E0609155
:10985000BD127091BE12072E000C880B990B0E944E
:10986000EFEA69837A838B839C83CE010196FDD9CD
:1098700000E09C0149E856E0692D812F0E94B275F5
:1098800049CF80915A0710925A078823B1F20E945B
:1098900061CD04E312E225EF30E050E040E06DEBF3
:1098A00072E189E896E00E9432CE809172078823A7
:1098B00021F272CF80915A0710925A07882309F437
:1098C00097C00E9461CD04E81AE623E730E050E03B
:1098D00040E06FE377E085E896E00E9432CE809129
:1098E0007207882309F484C057CF80915A071092D9
:1098F0005A07882309F41CCF0E9461CD8BE796E0BC
:109900000E94A7D080917207882309F411CF44CF19
:1099100085E0F8123DC080917307853011F1809188
:109920006F01882309F424CF11E0809173078530FB
:1099300009F010E060912C0170912D01072E000CB0
:10994000880B990B0E94EFEA69837A838B839C834F
:10995000CE0101968AD900E09C0146E756E06D2DC4
:1099600004CF80915A0710925A078823C1F20EE360
:109970001DE127EE33E04AE050E06CE271E086E75B
:1099800096E00E9432CE80917207882341F204CF84
:1099900026E0F212EDCE80917307863091F080912F
:1099A0006F01882309F4E4CE81E09091730796302B
:1099B00009F080E023E047E656E06E2D0E94B9CC26
:1099C000D7CE80915A0710925A07882341F385E138
:1099D00098E50E94C3CD80917207882301F3DCCE05
:1099E00083E0F81297CE80917307833009F462CF39
:1099F00080916F01882309F4FDCE11E080917307F7
:109A0000833009F010E060913F0770914007072E06
:109A1000000C880B990B0E94EFEA69837A838B8391
:109A20009C83CE01019621D963E0661900E09C0178
:109A300045E856E022CFA4E0B0E0E1E2FDE40C947A
:109A4000D0F1EE24E3948091BD129091BE12892B47
:109A500009F4E12C0E946DCDF09070074F2C95E039
:109A6000592E5F0C88248A94912C83E0B82EBF185D
:109A700082E0A82EAF1881E0782E7F183F2C319419
:109A800086E0682E6F18F11015C080917307882347
:109A900009F4D7C080916F01882309F475C181E072
:109AA00090917307911180E024E042E656E0632D27
:109AB0000E94B9CC8091BD129091BE129093340750
:109AC0008093330721E0F212E8C080917307813060
:109AD00009F4C8C080916F01882309F44DC011E0DA
:109AE00080917307813009F010E060913307709125
:109AF0003407072E000C880B990B0E94EFEA69834C
:109B00007A838B839C83CE010196AFD800E09C01C1
:109B10004BE556E0672D812F0E94B2758091B20708
:109B20008093330793E0F91227C010927F0780914A
:109B30007307833009F4F4C080916F018823E1F04A
:109B400011E080917307833009F010E080913307B2
:109B500024E6829FC001112481589F4FB4010E94C6
:109B6000A1F1862F0E941D1D00E09C014DE456E0EE
:109B70006B2D812F0E94B275D12CC12C14E00F2DBA
:109B80000419C0923307F1121FC0F601EE0FFF1F38
:109B9000EA5CF94F859194919093810780938007B7
:109BA000809173078F1509F4CEC080916F018823CF
:109BB00059F081E090917307911380E023E043E432
:109BC00056E0602F0E94B9CC812F9FEFC91AD90AA5
:109BD00015E08530B1F680913F0790914007892BC1
:109BE00019F4EE2009F4CEC026E0F21221C08091D3
:109BF0007307863009F4B8C080916F018823C1F0E3
:109C000084E997E49F938F938AE396E09F938F93E1
:109C10006F9281E090917307963009F080E08F9306
:109C20000E9422230F900F900F900F900F900F9093
:109C300087E0EE24E394F394F51025CF8093710729
:109C40000DC080915A0710925A07882309F422CF39
:109C50000BDD80917207882309F41CCF2496E1E183
:109C60000C94ECF180915A0710925A07882309F45A
:109C700031CF0E9461CD02E313E225EF30E050E0E6
:109C800040E063E377E08BE596E00E9432CE80917E
:109C90007207882309F41ECFE1CF82E0F8123ECF8D
:109CA00080917307823019F180916F01882309F444
:109CB00063CF11E080917307823009F010E060916A
:109CC0003F0770914007072E000C880B990B0E94EC
:109CD000EFEA69837A838B839C83CE0101960E948D
:109CE000354600E09C0147E556E06A2D14CF80918F
:109CF0005A0710925A078823B9F20E9461CD04E8EE
:109D00001AE623E730E050E040E06FE377E087E5D4
:109D100096E00E9432CE80917207882329F29ECF6E
:109D200080915A0710925A07882309F405CF0E94A0
:109D300061CD8DE496E00E94A7D0809172078823C0
:109D400009F4FACE8BCF80915A0710925A078823D4
:109D500009F42BCF8DEC9EE40E94C3CD8091720755
:109D6000882309F422CF7ACF80915A0710925A079C
:109D7000882309F441CFD8D880917207882309F449
:109D80003BCF6CCF86E057CF8091BD129091BE1231
:109D90009093340780933307C1CEB0E0A0E0E3EDA9
:109DA000FEE40C94D1F1009133070E946DCDC09177
:109DB000700710E0000F111F0A5C194F95E0592E33
:109DC0005C0E2EE0E22E26E0F22ED3E0DC1B32E425
:109DD000C32E33E2D32E4CE1A42E46E0B42E82E013
:109DE000782E7C1A53E4852E56E0952E81E0682E5D
:109DF0006C1A4C2E4194C1112AC08091730788239C
:109E0000B1F080916F01882359F081E09091730740
:109E1000911180E024E04AE256E0642D0E94B9CC22
:109E2000CF5FC511E8CF84E0809371070BC08091AC
:109E30005A0710925A07882321F316DC8091720783
:109E40008823F9F2CDB7DEB7E0E10C94EDF1C13033
:109E500059F5F8018591949190938107809380073B
:109E600080917307813081F080916F018823C1F266
:109E70001F929F928F926F9281E090917307913021
:109E800009F474C080E072C080915A0710925A079A
:109E9000882351F380913307682F0E9436D2809136
:109EA0007207882309F3CECFC23009F042C0F8010F
:109EB0008591949190938107809380078091730797
:109EC0008230D1F080916F01882309F4A9CFDF920D
:109ED000CF92BF92AF927F9281E0909173079230C0
:109EE00009F080E08F930E9422230F900F900F9033
:109EF0000F900F900F9094CF80915A0710925A07AD
:109F0000882301F30E944223809172078823D1F2B3
:109F100099CF80915A0710925A078823C1F0609117
:109F200033078FEF0E9436D280917207882379F031
:109F300089CFC33009F074CFF80185919491909343
:109F400081078093800780917307833011F380919C
:109F50006F01882309F464CF1F92FF92EF92DF9381
:109F600081E090917307933009F08CCF8F930E941A
:109F700022230F900F900F900F900F9051CFB0E0D1
:109F8000A0E0E5ECFFE40C94D6F10E946DCDC09109
:109F9000700785E0E82EEC0E9AEEC92E95E0D92EDA
:109FA000D4E0DC1B13E01C1B25E0A22E26E0B22E21
:109FB00002E00C1B81E0F82EFC1A9C2E9194C1113A
:109FC0002AC0809173078823B1F080916F018823A4
:109FD00059F081E090917307911180E024E049E00D
:109FE00056E0692D0E94B9CCCF5FEC12E8CF85E036
:109FF000809371070BC080915A0710925A078823EB
:10A0000021F332DB809172078823F9F2CDB7DEB7F6
:10A01000EBE00C94F2F1C13011F5809173078130BF
:10A0200079F080916F018823F9F281E090917307B4
:10A03000913009F080E023E047EB5DE26F2DD2CF55
:10A0400080915A0710925A07882359F38CE990E5BA
:10A050000E94C3CD80917207882319F3D7CFC230F5
:10A0600009F053C090917307923071F080916F01A5
:10A07000882309F4B9CF81E0923009F080E020E232
:10A080004BEF55E0602FAECF80915A0710925A07E0
:10A09000882361F3B092F006A092EF0680917207D8
:10A0A000882321F3B3CF80917307833081F08091AF
:10A0B0006F01882309F498CF81E090917307933062
:10A0C00009F080E023E04EEE55E0612F8BCF8091C8
:10A0D0005A0710925A07882351F387ED90E60E94A1
:10A0E000C3CD80917207882311F390CF80915A07D6
:10A0F00010925A07882391F0D092F006C092EF0692
:10A1000080917207882351F081CFC33061F2C4304F
:10A1100009F06ACF90917307943041F380916F01F9
:10A12000882309F461CF81E0943009F080E020E2D7
:10A1300049ED55E06D2F56CFB0E0A0E0E2EAF0E542
:10A140000C94DAF10E946DCDC091700785E0E82E85
:10A15000EC0ED4E0DC1B13E01C1B02E00C1B81E0C6
:10A16000F82EFC1ADC2ED194C1112AC080917307FD
:10A170008823B1F080916F01882359F081E090919C
:10A180007307911180E024E042ED55E06D2D0E94AF
:10A19000B9CCCF5FEC12E8CF85E0809371070BC09C
:10A1A00080915A0710925A07882321F35DDA809133
:10A1B00072078823F9F2CDB7DEB7E7E00C94F6F129
:10A1C000C13011F580917307813079F080916F0172
:10A1D0008823F9F281E090917307913009F080E0D3
:10A1E00023E04DED5DE26F2DD2CF80915A071092A2
:10A1F0005A07882359F381E593E20E94C3CD8091E9
:10A200007207882319F3D7CFC23009F055C0809167
:10A210007307823081F080916F01882309F4B9CFF0
:10A2200081E090917307923009F080E023E046EDE1
:10A230005DE2602FACCF80915A0710925A078823B5
:10A2400051F38CE493E20E94C3CD8091720788237E
:10A2500011F3B1CF80917307833081F080916F014A
:10A26000882309F496CF81E090917307933009F029
:10A2700080E023E04FEC5DE2612F89CF80915A07A7
:10A2800010925A07882351F387E493E20E94C3CDCA
:10A2900080917207882311F38ECF80915A07109214
:10A2A0005A07882391F086ED96E40E94C3CD8091F1
:10A2B0007207882351F07FCFC33061F2C43009F0B8
:10A2C00068CF80917307843041F380916F018823B8
:10A2D00009F45FCF81E090917307943009F080E03A
:10A2E00023E041EC5DE26D2F52CFACE0B0E0EBE754
:10A2F000F1E50C94D0F19C878B87362E80915A071C
:10A3000010925A07882339F01092A002ADD92C96EA
:10A31000E1E10C94ECF16091750770917607809102
:10A32000770790917807611571058105910509F40A
:10A330005CC020911201222309F4AEC020911301C8
:10A340002111AAC021E0321609F484C0E2E03E16D1
:10A3500009F491C0C0901401D0901501E09016014D
:10A36000F09017014090200150902101609022014F
:10A37000709023010E94EFEA2091080130910901B9
:10A3800040910A0150910B010E944EEB6F83788738
:10A3900089879A87F4E03F9E80011124C80186587E
:10A3A0009E4F9E838D83FC012081318142815381A8
:10A3B0006F81788589859A850E9407F24B015C013F
:10A3C000A3019201C701B6010E94E9EA811173C09D
:10A3D000F801E658FE4F80829182A282B382832DDB
:10A3E0000E946F6E81E080936F011092750710924A
:10A3F0007607109277071092780780916F01882373
:10A4000009F485CF24E0329EF0011124E658FE4F76
:10A41000C080D180E280F380C982DA82EB82FC8244
:10A420002DEC3CEC4CEC5DE360910801709109016E
:10A4300080910A0190910B010E946AF387FD65C02B
:10A44000CE0101960E946B1BBC018B859C850E94EE
:10A450004B755DCFC0901801D0901901E0901A01A2
:10A46000F0901B014090240150902501609026013E
:10A47000709027017FCFC0901C01D0901D01E0900B
:10A480001E01F0901F01409028015090290160901A
:10A490002A0170902B016ECF412C20E5522E23EC27
:10A4A000622E27E4722EC12C30E5D32E33ECE32E3E
:10A4B00037ECF32E5FCF20E030E0A9016F81788583
:10A4C00089859A850E94E9EA87FF0FC0A701960156
:10A4D000C501B4010E94E9EA87FF7ACFED81FE81D0
:10A4E000C082D182E282F3827ACFA3019201C501B8
:10A4F000B4010E946AF318160CF06ACFED81FE8158
:10A5000040825182628273826ACF20E030E44CE163
:10A5100056E4C701B6010E944EEB4B015C0120E0FE
:10A5200030E0A901C701B6010E94E9EA20E030E06D
:10A5300040EA50E487FF04C020E030E040EA50ECFD
:10A54000C501B4010E9407F22DEC3CEC4CEC5DE33C
:10A550000E944EEB0E94E6F26B017C01F7FC64C0A6
:10A5600020EA36E841E050E00E9439F1CA01B90121
:10A570002AE030E040E050E00E9439F1605D6093F5
:10A58000A102C701B60120E137E240E050E00E949D
:10A5900039F18AE0882E912CA12CB12CCA01B90185
:10A5A000A50194010E9439F1605D6093A202C70188
:10A5B000B60128EE33E040E050E00E9439F1CA01D4
:10A5C000B901A50194010E9439F1605D6093A30275
:10A5D0008EE28093A402C701B60124E630E040E099
:10A5E00050E00E9439F1CA01B901A50194010E940D
:10A5F00039F1605D6093A502C701B601A501940120
:10A600000E9439F16B017C01CA01B901A5019401D5
:10A610000E9439F1605D6093A60280E3C80EC0928B
:10A62000A70281EA92E010CFF094E094D094C09415
:10A63000C11CD11CE11CF11C6DE2A1CF62E08FECCA
:10A640009DE253CE61E086ED9DE24FCE60E08DED60
:10A650009DE24BCEA4E0B0E0E0E3F3E50C94DFF143
:10A6600080915A0710925A07882341F01092A00255
:10A670000E94344B2496E2E00C94FBF16091750744
:10A680007091760780917707909178076115710531
:10A690008105910561F10E94EFEA20910801309156
:10A6A000090140910A0150910B010E944EEB20914B
:10A6B00086013091870140918801509189010E9463
:10A6C00007F26093860170938701809388019093CD
:10A6D000890183E00E946F6E81E080936F01109288
:10A6E000750710927607109277071092780780917D
:10A6F0006F01882309F4BECF20915B0730915C077E
:10A7000040915D0750915E076091860170918701CD
:10A7100080918801909189010E9406F269837A8371
:10A720008B839C83CE0101960E946B1BBC0181EC44
:10A730009DE20E944B759ECFB0E0A0E0E2EAF3E517
:10A740000C94DAF10E946723082F0E946DCDC0910E
:10A750007007FC2E85E0E82EEC0E11E01C1BDC2EB1
:10A76000D194C11114C0809173078823F9F08091AE
:10A770006F01882309F474C081E0909173079111EF
:10A7800080E024E04CE753E06D2D0E94B9CC01112C
:10A790003AC0D2E0C130C1F5809173078130B9F081
:10A7A00080916F01811122C0D2E044C080915A078C
:10A7B00010925A078823D9F20E94344B8091720775
:10A7C0008823A9F2CDB7DEB7E7E00C94F6F18091CB
:10A7D0005A0710925A07882319F38BE795E50E94D0
:10A7E000C3CD809172078823D9F2ECCF81E090919C
:10A7F0007307913009F080E023E043E753E0612FD5
:10A800000E94B9CCD1CFD1E0DC1314C08091730782
:10A810008D17B9F080916F01882361F06C2F6F194B
:10A8200081E0909173079C1380E023E047E653E0BA
:10A830000E94B9CCCF5FCE1194CFDF5FD093710768
:10A84000C1CF80915A0710925A07882319F38EE9D5
:10A850009AE50E94C3CD809172078823D9F2B2CFC6
:10A86000D1E0002309F4A0CFE5CFB0E0A0E0EBE316
:10A87000F4E50C94D3F10E946DCDC09170076C2E5D
:10A8800085E0782E7C0E03E813E89AE2A92E94E086
:10A89000B92ED5E0DC1B25E5E22E23E8F22E84E07C
:10A8A000D82EDC1A83E0C82ECC1A82E0982E9C1A8F
:10A8B00081E0882E8C1AC1112CC0809173078823E7
:10A8C000B9F080916F01882361F0662D619581E078
:10A8D00090917307911180E024E04EE454E00E94CF
:10A8E000B9CCCF5FC711E7CF86E0809371070CC06A
:10A8F00080915A0710925A07882319F30E94344B0B
:10A90000809172078823E9F2CDB7DEB7EEE00C94B0
:10A91000EFF1C13049F5809173078130A1F080914A
:10A920006F018823F1F28AE993E89F938F9388E47B
:10A9300094E09F938F938F9281E090917307913071
:10A9400069F180E02BC080915A0710925A07882342
:10A9500031F38AE993E8892B11F00E949A83809160
:10A9600072078823E1F2D0CFC23009F08FC0809106
:10A9700073078230E9F080916F01882309F4B1CF29
:10A980008AE093E29F938F938EE394E09F938F935B
:10A990009F9281E090917307923099F68F930E9475
:10A9A00022230F900F900F900F900F900F9099CF40
:10A9B00080915A0710925A078823E9F20E940A23CD
:10A9C000809172078823B9F29FCF809173078330FB
:10A9D000A9F080916F01882309F483CF8CE693E876
:10A9E0009F938F9387E394E09F938F93CF9281E01F
:10A9F00090917307933009F0A4CFD0CF80915A077C
:10AA000010925A07882329F38CE693E8892B11F0DA
:10AA10000E946C83809172078823D9F275CF809150
:10AA20007307843099F080916F01882309F459CF1E
:10AA3000FF92EF9282E394E09F938F93DF9281E005
:10AA400090917307943009F07CCFA8CF80915A077A
:10AA500010925A07882339F3E114F10411F00E948F
:10AA60005583809172078823F1F24ECF80915A0767
:10AA700010925A078823B1F00115110511F00E94B8
:10AA8000838380917207882369F03ECFC33009F435
:10AA90009CCFC43021F2C53009F023CF80917307D9
:10AAA000853021F380916F01882309F41ACF1F9319
:10AAB0000F93BF92AF92DF9381E09091730795302F
:10AAC00009F03FCF6BCF80E090E0A0E8B0E4809346
:10AAD000820190938301A0938401B09385018FE15B
:10AAE00092E00E9490228091F5030E94097A1092D0
:10AAF000A0020C94344BB0E0A0E0E1E8F5E50C9442
:10AB0000D8F10E946DCDC091700785E0C82ECC0EA3
:10AB1000D4E0DC1B13E01C1B82E0F82EFC1A81E061
:10AB2000E82EEC1ABC2EB194C1112BC08091730792
:10AB30008823B1F080916F01882359F081E09091D2
:10AB40007307911180E024E045E553E06B2D0E94EE
:10AB5000B9CCCF5FCC12E8CF85E0809371070CC0F1
:10AB600080915A0710925A07882321F30E94344B90
:10AB7000809172078823F1F2CDB7DEB7E9E00C943B
:10AB8000F4F1C13089F5809173078130C1F0809173
:10AB90006F018823F1F2DD24D39480917307813013
:10ABA00009F0D12C88E89DE00E94511E00E09C0134
:10ABB0004AE453E06E2D8D2D0E94B275CACF80916C
:10ABC0005A0710925A07882311F30E9461CD42ED73
:10ABD0005CE268E87DE08AE493E00E94D2CD809157
:10ABE00072078823A1F2C8CFC23009F073C08091E8
:10ABF00073078230B1F080916F01882309F4A9CFE7
:10AC0000DD24D39480917307823009F0D12C8CE835
:10AC10009DE00E94511E00E09C014FE353E06F2D28
:10AC2000CACF80915A0710925A07882321F30E94B5
:10AC300061CD41ED5CE26CE87DE08FE393E00E9442
:10AC4000D2CD809172078823B1F296CF809173079D
:10AC50008330B1F080916F01882309F47ACFDD242D
:10AC6000D39480917307833009F0D12C80E99DE063
:10AC70000E94511E00E09C0144E353E0612F9BCFF2
:10AC800080915A0710925A07882321F30E9461CDC0
:10AC900040ED5CE260E97DE084E393E00E94D2CD88
:10ACA000809172078823B1F267CF80915A07109282
:10ACB0005A078823C9F00E9461CD4FEC5CE264E939
:10ACC0007DE089E293E00E94D2CD809172078823D3
:10ACD00059F052CFC33009F4B9CFC43009F039CF9D
:10ACE00080917307843009F380916F01882309F400
:10ACF00030CFDD24D39480917307843009F0D12CB8
:10AD000084E99DE00E94511E00E09C0149E253E06D
:10AD10006D2F51CFA3E0B0E0E0E9F6E50C94CFF160
:10AD20004C013B015A011901280181E08093A002E6
:10AD30004091750750917607609177077091780779
:10AD4000411551056105710571F0141615060CF0D9
:10AD500080E08093F30310927507109276071092AB
:10AD60007707109278071091F30380915A078B832D
:10AD700010925A07811105C080916F01882309F450
:10AD80006FC0C2010E94176F082F80E0C114D10468
:10AD900019F0C6010E94176F1A821982E114F1049A
:10ADA000B1F4402F50E0282F30E0CA01820F931FEA
:10ADB00046976CF485E190E0841B950B821B930B06
:10ADC00097FD0196959587958A8381E0898301E0B7
:10ADD00024E039E6A201BE016F5F7F4FCE010296EB
:10ADE0000E946F70E114F10491F08A81882321F0B0
:10ADF0001A8289818F5F898300E027E039E6A70105
:10AE0000BE016F5F7F4FCE0102960E946F70C1142A
:10AE1000D10459F000E024E039E6A601BE016F5FDD
:10AE20007F4FCE0102960E946F7041E04127B3012F
:10AE300081E00E9470D4C4010E94176F412FB401B9
:10AE400094E1981B892F0E9470D4EB81EE2341F08E
:10AE5000111101C05101A114B10431F0F50109959E
:10AE60002396E2E10C94EBF10E94344BF9CFCF92A0
:10AE7000DF92EF92FF920F931F9383EBC82E85E032
:10AE8000D82EF12CE12C05EB15E030E020E04FEC62
:10AE900056E465EC75E08AEC95E03CDF1F910F917C
:10AEA000FF90EF90DF90CF900895B0E0A0E0EBE549
:10AEB000F7E50C94D7F1ADB6BEB680912E1065E8DB
:10AEC00077E0882311F06EE270E1FB010190002031
:10AED000E9F7CF01861B970B01962DB73EB7281BCC
:10AEE000390B0FB6F8943EBF0FBE2DBF8DB79EB77E
:10AEF00001967C0180E2EDB7FEB78183C701019620
:10AF00000E942BF48FE6C82E85E0D82E01E715E0CD
:10AF100030E020E049E957E46DE775E084E895E02A
:10AF2000F9DE0FB6F894BEBE0FBEADBEEAE00C94DB
:10AF3000F3F1CF92DF92EF92FF920F931F938DEC7C
:10AF4000C82E84E0D82EF12CE12C00E415E030E08E
:10AF500020E047EC55E66FEC74E084ED94E0DADE37
:10AF60001F910F91FF90EF90DF90CF900895CF92B7
:10AF7000DF92EF92FF920F931F938AE8C82E83E02F
:10AF8000D82EF12CE12C0CE813E023E635E548E956
:10AF900052E268E973E08DE993E0BCDE1F910F9106
:10AFA000FF90EF90DF90CF900895B0E0A0E0EBED40
:10AFB000F7E50C94D7F1ADB6BEB683E392E00E94FC
:10AFC000176F90E001962DB73EB7281B390B0FB6CF
:10AFD000F8943EBF0FBE2DBF8DB79EB701967C0182
:10AFE00063E372E00E9431EA8091330700E012E0EF
:10AFF000813031F00BEE11E0823011F003E112E00C
:10B0000084E2C82E82E0D82E2DE837E449E453E6E6
:10B0100066E272E08DE292E07DDE0FB6F894BEBE8D
:10B020000FBEADBEEAE00C94F3F18F929F92AF9207
:10B03000BF92CF92DF92EF92FF920F9380915A07C7
:10B0400010925A07882371F01092A0020E94344B8C
:10B050000F91FF90EF90DF90CF90BF90AF909F90B7
:10B060008F90089581E08093A00280917507909160
:10B070007607A0917707B09178070097A105B105F1
:10B0800009F44AC05C01AA0CBB1CAA0CBB1C1092A0
:10B090007507109276071092770710927807B5011E
:10B0A0000B2C000C880B990B0E94EFEA2091BB0738
:10B0B0003091BC074091BD075091BE070E944EEBF6
:10B0C0002091611330916213409163135091641386
:10B0D0000E9407F26B017C0120E030E040EA51EC75
:10B0E0000E946AF387FD18C020E030E040EA51E496
:10B0F000C701B6010E94E9EA181674F0C5010E9462
:10B10000E7C8C0926113D0926213E0926313F09289
:10B11000641382E080936F0180916F01882309F4AA
:10B1200097CFC0906113D0906213E0906313F090BA
:10B13000641320E030E44CE156E4C701B6010E94FC
:10B140004EEB4B015C0120E030E0A901C701B601E4
:10B150000E94E9EA20E030E040EA50E487FF04C0C2
:10B1600020E030E040EA50ECC501B4010E9407F253
:10B170002DEC3CEC4CEC5DE30E944EEB0E94E6F2C1
:10B180006B017C018BE2F7FE09C0F094E094D0944F
:10B19000C094C11CD11CE11CF11C8DE28093A10262
:10B1A000C701B60120E137E240E050E00E9439F1EA
:10B1B0006AE0862E912CA12CB12CCA01B901A501FF
:10B1C00094010E9439F1605D6093A202C701B6014B
:10B1D00028EE33E040E050E00E9439F1CA01B901A5
:10B1E000A50194010E9439F1605D6093A3028EE293
:10B1F0008093A402C701B60124E630E040E050E0AD
:10B200000E9439F1CA01B901A50194010E9439F1E6
:10B21000605D6093A502C701B601A50194010E947B
:10B2200039F16B01CA01B901A50194010E9439F1FC
:10B23000605D6093A60260E36C0D6093A70261EA13
:10B2400072E084EF92E00E944B75C0906113D09041
:10B250006213E0906313F09064138090EF0390907A
:10B26000F003A090F103B090F203A5019401C7018F
:10B27000B6010E94E9EA8823E9F020E030E0A90164
:10B28000C701B6010E94E9EA882309F479C0A50143
:10B290009401C701B6010E94E9EA87FD73C081E00D
:10B2A0008093EE03C092EF03D092F003E092F1039B
:10B2B000F092F203D090EE038091B613813188F4BE
:10B2C0008091B813833068F044E04D195CEDE52EB1
:10B2D00052E0F52E0CE022E062E482E893E10E9465
:10B2E000ACD58091B613853180F48091B813843148
:10B2F00060F049EDE42E42E0F42E01E023E044E169
:10B300006CE382E893E10E94ACD58091B6138F3351
:10B3100008F09ECE8091B8138F3208F499CE40E3A6
:10B320004D198FEBE82E82E0F82E0DE022E06AE561
:10B3300082E893E10E94ACD541E34D1995EAE92EEC
:10B3400092E0F92E22E065E082E893E10E94ACD51C
:10B3500025E7E22E22E0F22E00E123E04FE262E157
:10B3600082E893E10E94ACD535E4E32E32E0F32E7F
:10B3700023E04FE267E682E893E10E94ACD568CE15
:10B3800080E08ECF8FEF8CCF0F931F93CF93DF93FF
:10B39000FC01EB018091750790917607A0917707EA
:10B3A000B0917807B7FF08C0109275071092760722
:10B3B0001092770710927807809164079091650743
:10B3C000A0916607B0916707409175075091760785
:10B3D000609177077091780784179507A607B707DC
:10B3E00044F48093750790937607A0937707B09302
:10B3F000780780916F018823E1F060917507709163
:10B4000076078091770790917807009168071091EF
:10B41000690720916A0730916B07600F711F821FC7
:10B42000931F0995BC0180916E0790916F070E9450
:10B430004B7580915A07811108C08091610788235C
:10B44000A9F180916F01882389F180916C07909117
:10B450006D070097B1F040917507509176076091A4
:10B46000770770917807009168071091690720911C
:10B470006A0730916B07400F511F621F731FFE0157
:10B480000995E0916207F0916307309741F0809150
:10B490006107811103C080915A078111099580913C
:10B4A0005A0710925A0781110E94344BDF91CF91B5
:10B4B0001F910F91089567E57DE180E79DE164CFDD
:10B4C00064ED7DE182E296E45FCF62EE7DE185E0AE
:10B4D0009FE15ACF66EF7DE18AE09EE155CF63E4BC
:10B4E0007EE18EE396E450CFE091E703E63028F565
:10B4F00081E08E0F8093E7034091750750917607A6
:10B50000609177077091780720917007909171078B
:10B510008091A00239E0E39FF0011124EF54FC4F29
:10B52000A0917C13B0917D13B183A0834283538398
:10B53000648375832683978380870895A7E0B0E0AE
:10B54000E4EAFAE50C94CFF10E946DCDF09070071B
:10B550002F2C85E08F0D8D833324339483E0E82EE8
:10B5600098EE892E93E0992EA12CB12C84E08F19AE
:10B570008E839E2D9F199F8382E0D82EDF18C32CC7
:10B58000CF18F1102CC0809173078823C1F08091EF
:10B590006F01882361F0622D619581E090917307BE
:10B5A000911180E024E045E553E00E94B9CCF3948A
:10B5B0009D81F912E6CF85E0809371070CC08091E0
:10B5C0005A0710925A07882311F30E94344B809136
:10B5D00072078823E1F22796E2E10C94EBF181E017
:10B5E000F8122DC0909173079130B9F080916F01DE
:10B5F0008823E9F281E0913009F080E09091A60380
:10B600002DE133E0911102C029E133E001E040E295
:10B6100053E06C2D0E94B275CACF80915A071092E8
:10B620005A07882319F38091A6038F258093A603D8
:10B63000E0926F01809172078823C1F2CCCF92E033
:10B64000F912D1C080917307823021F180916F018E
:10B65000882309F4ACCF11E080917307823009F0A0
:10B6600010E06091060170910701072E000C880B15
:10B67000990B0E94EFEA69837A838B839C83CE01C6
:10B6800001960E94354600E09C0142E153E06D2D99
:10B69000812FC0CF80915A0710925A078823B1F2A8
:10B6A00010E000E025EF30E050E040E066E071E0BF
:10B6B00082E193E00E9432CE80917207882331F2BA
:10B6C0008ACF80917307833019F180916F018823AD
:10B6D00009F46DCF11E080917307833009F010E019
:10B6E0006091040170910501072E000C880B990BE5
:10B6F0000E94EFEA69837A838B839C83CE01019653
:10B700000E94354600E09C014BE053E06F81C0CFC2
:10B7100080915A0710925A078823B9F210E000E08E
:10B7200025EF30E050E040E064E071E08BE093E032
:10B730000E9432CE80917207882339F24CCF8091DB
:10B740005A0710925A07882309F459C020E030E0C4
:10B7500048EC52E460910001709101018091020176
:10B76000909103010E944EEB0E94EBF22B0130926C
:10B770007207BADEE0926F0183E093E090936F0767
:10B7800080936E0780E091E090936D0780936C0743
:10B79000109268071092690710926A0710926B075F
:10B7A0008092640790926507A0926607B09267073F
:10B7B000712C612C40927507509276076092770742
:10B7C000709278078AE69AE590937D1380937C13B4
:10B7D00010926307109262071092610780917207BE
:10B7E000882369F0F8CE83E0F81609F46ACF94E074
:10B7F000F912DDCE80917307843009F4A0CF8091D7
:10B800006F01882309F4D3CE11E08091730784304F
:10B8100009F010E040900001509001016090020199
:10B820007090030120E030E0A901C301B2010E9441
:10B83000E9EA2DEB37E346E055EB87FD04C02DEB3D
:10B8400037E346E055E3C301B2010E9407F2698382
:10B850007A838B839C83CE0101960E94E11B00E0DA
:10B860009C0143E053E06E8113CFB0E0A0E0EBE336
:10B87000FCE50C94DFF18D8190919F10891778F091
:10B8800080939F109E01285F3F4F4E815F8164E54A
:10B8900070E08AE490E10E94B1EA10924910E2E07F
:10B8A0000C94FBF10F931F93CF93DF936F3F11F431
:10B8B00010929F1020919F1021111EC08C010E9498
:10B8C00038EA800F911FEC01C01BD10BC535D105A3
:10B8D0003CF00197FC012491207C2038D1F3F3CF78
:10B8E000DD27AE01B8018AE490E10E9459EAC65B07
:10B8F000DF4E188210924910DF91CF911F910F9166
:10B900000895A6E8B0E0E7E8FCE50C94DAF1C35846
:10B91000DF4F188219821A821B82CD57D040809146
:10B92000930290919402A0919502B0919602CF5704
:10B93000DF4F88839983AA83BB83C158D04084E6B4
:10B9400090E09093A9128093A8121092CD121092B9
:10B95000CC121092240464E070E0CE018F579F4F08
:10B960000E9495D18091A8129091A912029690936D
:10B97000A9128093A8121092CD121092CC1281E0DD
:10B98000CA57DF4F8883C658D040CE018A579F4F91
:10B990000E94752268E470E084E79DE00E9495D1E2
:10B9A00080E1E6E9F1E08E010F5F1F4FD8010190C1
:10B9B0000D928A95E1F760E170E0C8010E9495D18F
:10B9C00086E997E00E9481228CE0F80111928A9525
:10B9D000E9F7C8010E947D2282E391E00E9479226A
:10B9E0008EE291E00E9481228091BA029091BB0286
:10B9F000A091BC02B091BD0289839A83AB83BC83C2
:10BA0000C8010E948122C358DF4F188219821A820E
:10BA10001B82CD57D0407E01FDE6EF0EF11C83E086
:10BA2000F70180838983CE0183589F4F0E94812232
:10BA3000C7010E947522C8010E9475222AE0D22EF9
:10BA4000DA94DD2031F0CE0183589F4F0E9481228D
:10BA5000F7CF89E593E10E947D22C358DF4F18821A
:10BA600019821A821B82CD57D0409AE0D92EDA94DF
:10BA7000DD2031F0CE0183589F4F0E948122F7CF05
:10BA800087E08983F7018083C8010E947522C7017E
:10BA90000E94752268E070E08AE893E00E9495D1E8
:10BAA00068E070E082E893E00E9495D164EC70E079
:10BAB0008EEB92E00E9495D11982DD24DA94F70191
:10BAC000D082C8010E947922C7010E94752264E0D9
:10BAD00070E087E292E00E9495D18091EE06898322
:10BAE000C8010E9479226CE070E08EE497E00E9429
:10BAF00095D1198A1A8A1B8A1C8A80E090E0A0E8F6
:10BB0000BFE38D879E87AF87B88B8091C0129091DD
:10BB1000C112A091C212B091C31289839A83AB83E0
:10BB2000BC8320E030E543EC50E46091C412709196
:10BB3000C5128091C6129091C7120E944EEB6D8380
:10BB40007E838F8398872CEA35EC47E25EE3609131
:10BB5000C8127091C9128091CA129091CB120E94A2
:10BB60004EEB69877A878B879C8764E170E0C80118
:10BB70000E9495D184E190E09A83898362E070E02D
:10BB8000C8010E9495D18091420790914307A091EE
:10BB90004407B091450789839A83AB83BC8320E037
:10BBA00030E543EC50E4609146077091470780917F
:10BBB0004807909149070E944EEB6D837E838F83E7
:10BBC00098872CEA35EC47E25EE360914A07709172
:10BBD0004B0780914C0790914D070E944EEB69876F
:10BBE0007A878B879C87C8010E9471228CE0E6EAE5
:10BBF000F1E0D80101900D928A95E1F7C8010E9409
:10BC000071221982C8010E9475228FE78983C801B9
:10BC10000E947522D982C8010E94752285E0E2EB5C
:10BC2000F1E0D80101900D928A95E1F765E070E0AE
:10BC3000C8010E9495D11982C8010E94792280E230
:10BC4000E7EBF1E0D80101900D928A95E1F760E20F
:10BC500070E0C8010E9495D1F7011082C7010E94CF
:10BC600079221982C8010E94792280E090E0A0EE3A
:10BC7000BFE3C358DF4F88839983AA83BB83CD5723
:10BC8000D040CE0183589F4F0E948122C358DF4F7E
:10BC9000188219821A821B82CD57D040CE01835858
:10BCA0009F4F0E94812282E1F80111928A95E9F763
:10BCB00062E170E0C8010E9495D184E2E7EDF1E015
:10BCC000D80101900D928A95E1F764E270E0C80115
:10BCD0000E9495D180E1F80111928A95E9F760E11F
:10BCE00070E0C8010E9495D189E0F80111928A950F
:10BCF000E9F769E070E0C8010E9495D1C358DF4FB1
:10BD0000188219821A821B82CD57D040CE018358E7
:10BD10009F4F0E9481228CE0D82EF8018D2D119228
:10BD20008A95E9F76CE070E0C8010E9495D18CE635
:10BD3000F80111928A95E9F76CE670E0C8010E945B
:10BD400095D188E194E00E947122F701108211825E
:10BD500012821382148215821682178268E070E0C4
:10BD6000C7010E9495D1F7011192DA94E9F7CB57F8
:10BD7000DF4F1882C558D04080E090E0A0E4B0E4E6
:10BD8000ED968CAF9DAFAEAFBFAFED97C7010E94F0
:10BD90007D22CE018B579F4F0E947522CE0187587E
:10BDA0009F4F0E94812280912404811127C000911D
:10BDB000A8121091A9128091CC129091CD12F70186
:10BDC0009183808384E690E09093A9128093A812D7
:10BDD00064E070E08BE292E00E9495D162E070E056
:10BDE000C7010E9495D191E00037F3E01F0709F4E5
:10BDF00090E080912404892B809324048091240472
:10BE0000811104C060E089E59AE04CDD9091240442
:10BE100081E08927CA57DF4FE7E00C94F6F171CD36
:10BE2000A4E0B0E0E6E1FFE50C94CFF10E946723C7
:10BE3000782E0E946DCD209170072B83772009F416
:10BE4000CAC083E08C831B81212F2B5F298383E071
:10BE5000582E852D811B8A834424439421E7822E0A
:10BE60002AE6922E82E0682E611A342C311A212E95
:10BE700021943FE0E32E3FE5F32E4BE7C42E44E050
:10BE8000D42E5FE9A52E52E4B52E2B812111B8C026
:10BE900080917307882309F4A1C080916F018823E2
:10BEA00059F081E090917307911180E024E048EC13
:10BEB00054E0622D0E94B9CC7110BAC02B8123309E
:10BEC00009F0B6C080917307833009F4F7C0809100
:10BED0006F01811104C104E081E0800F9B8189130F
:10BEE0001FC080917307891709F435C180916F01D4
:10BEF0008823B1F0FF92EF92DF92CF928B81811B6A
:10BF00008F9381E0909173072B81921380E08F9340
:10BF10000E9422230F900F900F900F900F900F9080
:10BF200082E0800F71104EC09B81891323C08091E5
:10BF30007307891709F41DC180916F018823D1F01F
:10BF400083E39BE49F938F938DE694E09F938F937D
:10BF50008B81811B8F9381E0909173072B819213CA
:10BF600080E08F930E9422230F900F900F900F90EC
:10BF70000F900F9083E0800F9B81891321C08091E7
:10BF80007307891709F404C180916F018823C1F0F8
:10BF9000BF92AF928CE594E09F938F938B81811B2E
:10BFA0008F9381E0909173072B81921380E08F93A0
:10BFB0000E9422230F900F900F900F900F900F90E0
:10BFC00084E0800F9B819F5F9B83298129135DCF34
:10BFD0008093710711C094E09C8335CF80915A07FC
:10BFE00010925A07882309F458CF0E94344B80914D
:10BFF0007207882309F451CF2496E2E10C94EBF107
:10C000008B818130A1F580917307813009F1809196
:10C010006F01882309F450CF81E09091730791302C
:10C0200009F080E023E046EB54E0632D0E94B9CC98
:10C030008C819B8189130AC0809173072C818217A0
:10C0400009F45AC080916F0181116FC00C8144CFF7
:10C0500080915A0710925A078823C9F28CE993E518
:10C060000E94C3CD80917207882389F2C5CF9B813E
:10C07000923009F021CF80917307823081F0809156
:10C080006F01882309F418CF81E0909173079230F3
:10C0900009F080E023E047EA54E0662DC7CF8091A5
:10C0A0005A0710925A07882351F385E198E50E94B8
:10C0B000C3CD80917207882311F39ECF80915A07D8
:10C0C00010925A07882309F402CF85E394E50E9471
:10C0D000C3CD80917207882309F4F9CE8DCF81E01A
:10C0E00090917307933009F080E023E04FE954E02A
:10C0F0006A810E94B9CCEFCE80915A0710925A07FC
:10C10000882309F49FCF80913201842580933201E6
:10C1100050926F018114910411F00E94716A809114
:10C120007207882309F48ECF67CF6B81611B81E092
:10C13000909173072B81921380E0909132012EE849
:10C1400034E0911102C02AE834E001E041E954E012
:10C150000E94B2757BCF80915A0710925A078823AC
:10C1600009F4C4CECEDB80917207882309F4BECED9
:10C1700043CF80915A0710925A07882309F4DCCEE6
:10C180000E94264B80917207882309F4D5CE34CFC4
:10C1900080915A0710925A07882309F4F5CE0E941D
:10C1A0006B4180917207882309F4EECE25CFA7E07A
:10C1B000B0E0EDEDF0E60C94CFF18091820787704E
:10C1C000898380908A0390908B03A0908C03B09019
:10C1D0008D030E946DCD209170072E8339813730F9
:10C1E00009F075C085E194E09B838A831E81312F1D
:10C1F0003B5F3C8333243394812F81958D83232CA3
:10C20000211A84E6482E512C612C712C2E81222378
:10C2100009F462C03981373009F434C22E812130EB
:10C2200009F029C290917307913009F445C18091BA
:10C230006F01811154C182E0F82E81E08F0D8F8350
:10C240009981973009F063C020E030E0A901C50171
:10C25000B4010E94E9EA882309F459C03F818E8124
:10C26000381331C09091B9029F83809173072E815A
:10C27000821311C080915A0710925A07882359F0EF
:10C2800093259F8383E080936F010E948522809194
:10C29000720781110DC180916F018823A1F06E8119
:10C2A000611B81E0909173073E81931380E09F8131
:10C2B00026EF33E0911102C022EF33E001E049EFB5
:10C2C00053E00E94B275F394F394FF8220C020E102
:10C2D00034E03B832A838ACF80917307882309F453
:10C2E000D9C080916F01882309F494CF81E09091A7
:10C2F0007307911180E024E043E254E06D810E94D5
:10C30000B9CC8981873009F41DC193E09F83809166
:10C31000BA029091BB02A091BC02B091BD02809381
:10C32000330790933407A0933507B09336072F81D6
:10C330003E8123131EC080917307821709F407C141
:10C3400080916F018823A9F0EE80E11AFF24F39415
:10C35000809173073E818313F12C83E397E00E9461
:10C36000E54500E09C0146EE53E06E2D8F2D0E94C6
:10C37000B2758F818F5F9E81891316C0809173077C
:10C38000891709F439C180916F01882369F06E81A2
:10C39000611B81E0909173072E81921380E023E06E
:10C3A00047ED53E00E94B9CC8F818E5F3E818313AD
:10C3B00016C080917307831709F42FC180916F0114
:10C3C000882369F06E81611B81E0909173072E8153
:10C3D000921380E023E04AEC53E00E94B9CC8F81B5
:10C3E0008D5F3E81831323C080917307831709F407
:10C3F00025C180916F018823D1F083E39BE49F9353
:10C400008F938CEB93E09F938F938E81811B8F93FF
:10C4100081E0909173073E81931380E08F930E9497
:10C4200022230F900F900F900F900F900F908F81FD
:10C430008C5F9E81891323C080917307891709F44B
:10C440000CC180916F018823D1F08FE09FE59F930D
:10C450008F938DEA93E09F938F938E81811B8F93AF
:10C4600081E0909173072E81921380E08F930E9458
:10C4700022230F900F900F900F900F900F903E81FE
:10C480003F5F3E838C818313C1CE9F819B5F9093DE
:10C4900071070EC080915A0710925A07882309F439
:10C4A00020CF0E94344B80917207882309F419CF62
:10C4B0002796E2E10C94EBF180915A0710925A070B
:10C4C000882309F4B4CE25E036E03093F0062093BB
:10C4D000EF0680917207882309F4A9CEE9CF81E0A5
:10C4E000913009F080E020E249E154E0622D0E94A1
:10C4F000B9CCA1CE909173073E81931731F0809112
:10C500006F01811113C08E8197CE80915A071092CE
:10C510005A078823A1F32A813B813093F0062093A8
:10C52000EF0680917207882351F3C2CF6E81611BA1
:10C5300081E03E81931380E020E246E054E00E94D7
:10C54000B9CCE1CF22E02F83FF24F3947DCE8091FC
:10C550005A0710925A07882309F4F2CE0E9461CD3F
:10C5600060913307709134078091350790913607B9
:10C570000E94EBF26B01309272070E94745A83E0C2
:10C5800080936F0186EE93E090936F0780936E0720
:10C5900023E337E030936D0720936C071092680710
:10C5A0001092690710926A0710926B074092640715
:10C5B000509265076092660770926707F12CE12C34
:10C5C000C0927507D0927607E0927707F0927807CD
:10C5D00080E69AE590937D1380937C132BE832E2FA
:10C5E000309363072093620710926107809172076E
:10C5F000882309F4A5CE5CCF80915A0710925A0780
:10C60000882309F4C0CE85E198E50E94C3CD8091CE
:10C610007207882309F4B7CE4BCF80915A07109246
:10C620005A07882309F4CACE8FE497E40E94C3CD49
:10C6300080917207882309F4C1CE3ACF80915A07BE
:10C6400010925A07882309F4D4CE0E94264B809179
:10C650007207882309F4CDCE2BCF80915A07109210
:10C660005A07882309F4EDCE4CD9809172078823AC
:10C6700009F4E7CE1DCF2E81223009F43BCF33E001
:10C680003F8345CE8E81813009F434CF92E09F8381
:10C690005BCF0E946B4135D90C948D47CF9380912D
:10C6A000A903811109C08CED91E09093ED03809373
:10C6B000EC0381E08093A9030E94745A20E040E0DB
:10C6C00070E060E082E793E20E945146C1E0C093CF
:10C6D000A0020E94D32C0E94344BC093A00260E0C1
:10C6E0008BE29EE2DFD888ED91E09093F006809394
:10C6F000EF06CF910895A6E0B0E0E1E8F3E60C94F0
:10C70000CFF10E94E97B382E8091D41484FB6624FB
:10C7100060F8412C84FF03C00E94FC7B482E0E94DD
:10C720006DCD209170072D83522E2B5F298380E0E1
:10C730000EE215E091E0792E7518952D91959A836A
:10C740009EE4E92E93E6F92E2BE4C22E25E0D22EAC
:10C7500092E095199B8393E095199C833AEE832E82
:10C7600034E0932E4FEFA42E44E0B42E9D81298116
:10C77000921709F409C2992349F131106AC00E9445
:10C780003F82882309F47AC19D81913009F444C124
:10C7900022E02E832D818E8128135FC18091730743
:10C7A000281709F46EC180916F01882309F455C1DF
:10C7B0006D81651981E0909173072D81921380E05E
:10C7C00023E047E255E00E94B9CC47C1809173074E
:10C7D000882379F180916F01882379F281E090912B
:10C7E0007307911180E024E047E555E06A810E94DB
:10C7F000B9CC332021F224E02E839D812E81921327
:10C800004AC080917307981709F44CC180916F0159
:10C81000882309F440C06D81651981E09091730708
:10C820002D81921380E023E04BE155E00E94B9CCCA
:10C8300032C080915A0710925A07882359F20E94F9
:10C84000344B80917207882329F22696E2E10C94FA
:10C85000EBF18D81813009F47FC0823009F4A6C0EC
:10C860009D81933041F680917307833009F4C3C0F2
:10C8700080916F01882309F4BECF81E09091730706
:10C88000933009F080E023E04BE355E06C810E9497
:10C89000B9CC84E08E838E818F5F9D81981316C002
:10C8A00080917307981709F40EC180916F01882356
:10C8B00069F06D81651981E0909173072D81921364
:10C8C00080E023E04DE055E00E94B9CC8E818E5F80
:10C8D000662009F430C141103BC09D8198131BC0F4
:10C8E00020907307921509F4FFC080916F0188238F
:10C8F00091F01F92BF92AF928D8185198F9381E045
:10C900002D81221180E08F930E9422230F900F909F
:10C910000F900F900F908E818D5F9D81981316C0A0
:10C9200080917307981709F4F5C080916F018823EF
:10C9300069F06D81651981E0909173072D819213E3
:10C9400080E023E04EEE54E00E94B9CC8E818C5FF3
:10C950009D819F5F9D830ACF809173078130D1F0C5
:10C9600080916F01882309F446CFFF92EF92DF9206
:10C97000CF927F9281E090917307913009F080E02F
:10C980008F930E9422230F900F900F900F900F9083
:10C990000F9031CF80915A0710925A07882301F3E4
:10C9A0007DDE809172078823D9F24FCF8091730783
:10C9B000823091F080916F01882309F41CCF81E0CF
:10C9C00090917307923009F080E023E040E455E055
:10C9D0006B810E94B9CC0FCF80915A0710925A07F1
:10C9E000882341F389E997E50E94C3CD80917207BE
:10C9F000882301F32ACF80915A0710925A0788237F
:10CA000009F436CF82E59BE40E94C3CD8091720782
:10CA1000882309F42DCF19CF80917307813009F154
:10CA200080916F01882309F4B3CE8FED94E49F9336
:10CA30008F931F930F937F9281E0909173079130B2
:10CA400009F080E08F930E9422230F900F900F90A7
:10CA50000F900F900F9082E08E838E818F5F8E8378
:10CA6000CCCE80915A0710925A078823C9F20E94AF
:10CA7000DF4480917207882399F2E7CE91E09E838C
:10CA800089CE80915A0710925A07882309F48BCED9
:10CA90008FEB9FE40E94C3CD80917207882309F435
:10CAA00082CED3CE80915A0710925A07882309F478
:10CAB000ADCE8BE19DE40E94C3CD809172078823A7
:10CAC00009F4A4CEC2CE80915A0710925A07882347
:10CAD00009F4EBCE80E19FE50E94C3CD80917207FF
:10CAE000882309F4E2CEB1CE80915A0710925A07FA
:10CAF000882309F4FACE4FE350E069ED74E081EF4A
:10CB000096E00E9440F480917207882309F4EDCEEC
:10CB10008D811ECF80915A0710925A07882309F4FD
:10CB200004CF85E397E60E94C3CD809172078823E6
:10CB300009F4FBCEEDCF9D81981314C0909173073B
:10CB40002D81291791F080916F01882359F06D8113
:10CB5000651981E02D81291380E020E24DED54E03C
:10CB60000E94B9CC8E818D5FF3CE80915A071092CE
:10CB70005A07882341F39092F0068092EF06809145
:10CB80007207882301F3C4CF809371075ECE1092A1
:10CB90009E0210926E010E94FC7B9091D41480FB47
:10CBA00097F99093D41460E08AEC91E00E94525C73
:10CBB0000C948D470F931F930E94EBD100919A0222
:10CBC00010919B0220919C0230919D02601B710B81
:10CBD000820B930B97FD0CC089B183FB882780F9EA
:10CBE00091E089274A9B8260309B84608093990200
:10CBF0008091990281709091990291FD826090914B
:10CC0000A803981749F0813009F148F0823079F093
:10CC1000833091F08093A8031F910F910895913074
:10CC200079F09230B9F79091980291500CC0992305
:10CC300039F09330C1F3EECF9130A9F3923051F730
:10CC4000909198029F5F90939802E4CF992359F3B3
:10CC5000933001F7F5CF1F93CF93DF9380913A0183
:10CC60008F3708F475C08F579091BF129093A80426
:10CC7000992309F46BC05D9A909141079093A704A2
:10CC8000992309F46FC05C9A8F5F80933A01809179
:10CC9000A60491E089278093A60481118BDF8091FF
:10CCA000390191E0980F85300CF090E0823009F462
:10CCB000A8C00CF059C0882309F46EC0813009F473
:10CCC00095C090933901C0918307D0918407209734
:10CCD00009F42DC0F89413B1147082E00E94522C14
:10CCE00000C000C01C161D060CF0B9C02A9A00C076
:10CCF00000C02B9A00C0000082E090E00197F0F79E
:10CD00002B9800C000C0112309F4ABC02A9A00C0C0
:10CD100000C0789480918307909184071C161D06AB
:10CD20000CF0A1C0019790938407809383078091B2
:10CD3000BC0D9091BD0D009729F001979093BD0D0A
:10CD40008093BC0DDF91CF911F9108955D9894CF92
:10CD50009091A804891708F05D989091A70489170D
:10CD600008F492CF5C9890CF843009F461C00CF441
:10CD70005BC0853009F0A5CF2091A504211102C028
:10CD80008093A5048091A50481508093A5048823F5
:10CD900009F497CF95E095CF809138018F5F80316E
:10CDA0001CF4809338018DCF109238018091A70335
:10CDB000811113C02091B5123091B6123093B81280
:10CDC0002093B712209137073091380730933A07F4
:10CDD0002093390781E08093A7031092B612109236
:10CDE000B51210923807109237076BCF10927B0064
:10CDF00087E480937C0080917A00806480937A003D
:10CE000060CF80917A0086FD26C0409178005091D5
:10CE100079002091B5123091B612240F351F30934E
:10CE2000B6122093B5124DCF10927B0086E4E1CF6D
:10CE300080917A0086FD11C0409178005091790070
:10CE40002091370730913807240F351F309338076A
:10CE50002093370736CF92E034CF94E032CF2A9830
:10CE600046CF2A9854CF01965ECFACE3B0E0EBE317
:10CE7000F7E60C94CFF180917407882369F18091D3
:10CE8000D41410E000E084FF23C089EE92E10E94F8
:10CE9000FE248BE1E9EEF2E1DE01919601900D9224
:10CEA0008A95E1F710E000E0BE016F5F7F4FCE0191
:10CEB00081960E94FFDB18163CF4CE0101960E9479
:10CEC0000AD6080F111DF0CFCE0181960E94CE2602
:10CED0001093F7030093F6030E946DCD1091700735
:10CEE000312E85E0810F8CAF212E219485E9A82E6B
:10CEF0008DE1B82E90EA892E95E0992E01E0011B74
:10CF000025EA622E25E0722E111113C0809173075D
:10CF1000882391F180916F01882359F081E09091ED
:10CF20007307911180E024E04EEA55E0622D0E94E3
:10CF3000B9CC8091D41486FF3EC01130D9F48091D1
:10CF40007307813049F180916F01882309F43EC154
:10CF50001F927F926F920F9381E0909173079130AF
:10CF600009F080E08F930E9422230F900F900F9082
:10CF70000F900F9082E04FC080915A0710925A078D
:10CF8000882341F20E94344B80917207882311F26A
:10CF9000EC96E2E10C94EBF180915A0710925A075B
:10CFA000882389F2109270070E9416D88091720728
:10CFB000882349F2EDCF84FF2DC01130D9F680913E
:10CFC00073078130D1F080916F01882309F4FEC08E
:10CFD000BF92AF929F928F920F9381E090917307CF
:10CFE000913009F080E08F930E9422230F900F90E0
:10CFF0000F900F900F900F90BDCF80915A07109215
:10D000005A07882301F30E94951D80917207882397
:10D01000D1F2BECF81E090916F01992309F4D7C07E
:10D02000582ED12CC12C412E4318852DE090F603AB
:10D03000F090F703CE14DF0408F0C9C05112A5C068
:10D0400091E0E91AF108EC18FD0889EE92E10E94DE
:10D05000FE248BE1E9EEF2E1DE01919601900D9262
:10D060008A95E1F7F12CBE016F5F7F4FCE0181966B
:10D070000E94FFDB18167CF4CE0101960E940AD6AE
:10D08000882389F3EF106BC0BE016F5F7F4F85E887
:10D0900097E00E9425D6CE0181960E94CE268091EF
:10D0A000D4149091730785FF75C0911363C080916C
:10D0B0005A0710925A07882309F45CC019821C820F
:10D0C0008091EC1264E073E1882311F069EE72E163
:10D0D00021E045E857E0CE0101960E94D32688233F
:10D0E00009F43FC08BE1FE013196A9EEB2E1019057
:10D0F0000D928A95E1F78091D4148F7B8093D4149C
:10D10000A091CA14AA3080F481E08A0F8093CA14D7
:10D110008BE18A9FD0011124A454BC4EE9EEF2E1C8
:10D1200001900D928A95E1F7CE0101960E94CE26DC
:10D130001092700782E090E0A0E0B0E08093750765
:10D1400090937607A0937707B093780781E0809358
:10D15000720710929F0283E080936F0119CFF394BE
:10D1600082CF0E94018B65E877E08AE895E00E9413
:10D17000E5D5DACF80916F01882339F081E09113F2
:10D1800080E041E0642D0E94F7CC8FEFC81AD80AE6
:10D1900053944BCF911759F080916F018823A9F3D5
:10D1A00081E090917307911380E040E0EBCF809194
:10D1B0005A0710925A07882379F385E597E50E946C
:10D1C000C3CD80917207882339F3E2CE82E01F5FDE
:10D1D0009CAD911399CE80937107DACEFC01A081AA
:10D1E000B1811C92A281B3818C918F5F8C9302805C
:10D1F000F381E02D90818CE0989F800D1124EEE763
:10D20000F3E113AE84AF0895FC0184910895FC010D
:10D2100080810895009751F0FC0180E0919199235D
:10D2200031F0907C9038D1F38F5FF8CF80E0089593
:10D23000119800C087FD43C0419800C0119A00C0FA
:10D2400000C0119800C086FD46C0419800C0119AE8
:10D2500000C000C0119800C085FD3BC0419800C0CF
:10D26000119A00C000C0119800C084FD30C04198E0
:10D2700000C0119A00C000C0119800C083FD25C0F5
:10D28000419800C0119A00C000C0119800C082FDF2
:10D290001AC0419800C0119A00C000C0119800C087
:10D2A00081FD0FC0419800C0119A00C000C01198C4
:10D2B00000C0419800C0119A00C000C00895419A72
:10D2C000BCCF419AF0CF419AE5CF419ADACF419A4B
:10D2D000CFCF419AC4CF419AB9CF90E080E0089572
:10D2E000CF93DF93DB01F9019C919130C1F0943031
:10D2F00080F094509C938830D1F480819181009784
:10D3000071F0019791838083480F591FEA011882B9
:10D3100006C08C3539F49C5F9C93943041F4DF91C6
:10D32000CF9108958B3339F781E08C93F8CF20812A
:10D330003181B9016F5F7F4F71836083420F531F4B
:10D34000EA018883808191818F3591056CF7E7CF61
:10D350000F931F9381E00091D0141091D11420916C
:10D36000D2143091D3144091CC145091CD146091CB
:10D37000CE147091CF14041715072607370708F449
:10D3800080E01F910F91089590E080E00895209132
:10D390000D06833021F425FD0CC024FD0CC030E0C7
:10D3A000A90102C0559547958A95E2F7CA01817097
:10D3B000089581E0089580E008958091290684FD14
:10D3C0000BC080912B0687FD07C090912C069370AF
:10D3D00081E019F480E0089581E008952FEB280F93
:10D3E0002A3108F047C0E22FF0E0809129069091A1
:10D3F0002A06A0912B06B0912C0604C0B695A795DD
:10D40000979587952A95D2F780FD02C0817008957F
:10D41000E15FF94FE081EE2341F180919407909113
:10D420009507E80FF92FF11D808190ED980F9A3044
:10D4300030F08E3251F4818180538A3098F4F09329
:10D44000FE05E093FD0581E008958D3211F08B32E9
:10D4500049F4818190ED980F9A3088F38E3211F45F
:10D460008281EACFF0E0E0E0EACF1092FE05109270
:10D47000FD05E9CF80E00895CF93DF9385E4AEDF2B
:10D48000882309F188E04091290650912A0660918D
:10D490002B0670912C06972F9170C92F90E0D92FF1
:10D4A000CC0FDD1F71FB222720F930E0220F331F44
:10D4B000220F331FC22B67FB442740F9C42B8C2B50
:10D4C000DF91CF91089580E0DECF88DF882341F09F
:10D4D00081E02091FD053091FE05232B09F480E0C9
:10D4E00008951092C80580912E0190912F01A0916E
:10D4F0003001B09131018093980390939903A093E8
:10D500009A03B0939B030895CF93DF93C0913F0795
:10D51000D0914007209729F160913B0770913C071B
:10D5200080913D0790913E070E94E6F26E5F7F4F2B
:10D5300024976C177D07ACF47093A1036093A0034C
:10D540000E94EBD1605A75418F4F9F4F6093A203A9
:10D550007093A3038093A4039093A503DF91CF91CD
:10D5600008951092A2031092A3031092A4031092A4
:10D57000A503F4CFB0E0A0E0E0ECFAE60C94D8F11B
:10D580006B01E9014A3009F4D5C0453109F081C089
:10D59000DB011296ED91FC91F28096818781139ABE
:10D5A00000C00000E6E2F0E03197F0F7092F182FF5
:10D5B000EF2CE29420EFE22230E1B32EBF0CE80121
:10D5C00088EF36DE00C0000086E290E00197F0F7B9
:10D5D000BFE1BF1508F49BC08F2D8077806828DEDF
:10D5E0008E2D26DE00C0000086E290E00197F0F765
:10D5F00080E81EDE80E01CDE00C0000086E290E0D5
:10D600000197F0F78AEF14DE00C0000086E290E098
:10D610000197F0F7005F1F4F8881807F09DE8991B5
:10D620008295807F05DEC017D107B1F700C00000EA
:10D6300086E290E00197F0F7F394E0E1EE0EFB1044
:10D64000BECF1398D6011296ED91FC918081928104
:10D65000980F92832181921708F09FC194819F5F58
:10D6600094839381890F821710F08FEF820F838349
:10D67000458150E0440F551F70E060E0868197813E
:10D680000E9406F481E0CDB7DEB7E9E00C94F4F136
:10D69000DEC1FB0102811381423309F485C108F424
:10D6A0008DC1463409F475C1473409F482C14B3346
:10D6B00049F789812B81D80112967C911297139694
:10D6C0003C91213009F4BFC1233009F0A0C148EFDB
:10D6D000480F582F91E0341708F490E031E05417C8
:10D6E00008F030E0492F432B61E0571708F460E061
:10D6F000462311F4932331F2FA8030E0F901ED5B17
:10D70000FD4FD080215C3D4FF901E08099C180EE52
:10D710008F0D8068807F8CDD8F2D8295807F88DDE6
:10D7200000C0000086E290E00197F0F780E880DD1D
:10D7300080E861CF0B9A1398399A4198099A119A07
:10D74000139A00C0000086E290E00197F0F788E7A6
:10D7500090E0CEE9DFE0FE013197F1F70197D9F7CC
:10D7600088EF66DD00C0000086E290E00197F0F7E8
:10D7700080E25EDD80E05CDD00C0000086E290E0DB
:10D780000197F0F780E054DD80E852DD00C0000032
:10D7900086E290E00197F0F780E04ADD80E148DD25
:10D7A00000C0000086E290E00197F0F7CE010197FB
:10D7B000F1F7CE010197F1F7CE010197F1F7CE0114
:10D7C0000197F1F7CE010197F1F7CE010197F1F73B
:10D7D000CE010197F1F7CE010197F1F7CE01019744
:10D7E000F1F7CE010197F1F7CE010197F1F7CE01E4
:10D7F0000197F1F7CE010197F1F7CE010197F1F70B
:10D800002197F1F780E214DD80E412DD00C0000012
:10D8100086E290E00197F0F780E20ADD80E608DD1D
:10D8200000C0000086E290E00197F0F7D0E0C0E091
:10D830008C2F80778068FCDC8D2FFADC00C0000024
:10D8400086E290E00197F0F780E8F2DC80E0F0DC1F
:10D8500000C0000086E290E00197F0F78AEFE8DC74
:10D8600000C0000086E290E00197F0F780E2119896
:10D8700000C0419800C0119A00C000C0119800C0BB
:10D88000419800C0119A00C000C0119800C0419892
:10D8900000C0119A00C000C0119800C0419800C09B
:10D8A000119A00C000C0119800C0419800C0119AA0
:10D8B00000C000C0119800C0419800C0119A00C07B
:10D8C00000C0119800C0419800C0119A00C000C06B
:10D8D000119800C0419800C0119A00C000C0119872
:10D8E00000C0419800C0119A00C000C0119800C04B
:10D8F000419800C0119A00C000C0119800C0419822
:10D9000000C0119A00C000C0119800C0419800C02A
:10D91000119A00C000C0119800C0419800C0119A2F
:10D9200000C000C0119800C0419800C0119A00C00A
:10D9300000C0119800C0419800C0119A00C000C0FA
:10D94000119800C0419800C0119A00C000C000C0EA
:10D950000000E6E2F0E03197F0F7815009F087CF60
:10D9600088EF66DC00C0000086E290E00197F0F7E7
:10D97000CF5FD05FC03209F05BCF80E059DC80EC34
:10D9800057DC00C0000086E290E00197F0F71398A2
:10D9900079CEF8018581888375CE80E0CDB7DEB77A
:10D9A000E9E00C94F4F153C0B901C8010E94E9D236
:10D9B00069CED80111968C91888364CE443191F060
:10D9C000473109F05FCE1882D80112968C911297D8
:10D9D000898315968C91159781508A8313968C9123
:10D9E0008B8350CED80115964C91159750E0440F7B
:10D9F000551F70E060E016968D919C910E9406F490
:10DA0000F801128280818150838314823BCE3817C3
:10DA100008F438CE871708F435CEFA80E12CD12CE3
:10DA2000243070F46ACEBE01C8010E94E9D2898117
:10DA300098819D0D98838E0D8983FF0C09F422CE69
:10DA4000F7FEF6CFF0CF58E0580F482F43CEEF92B5
:10DA5000FF920F931F93CF93DF93EC018B017A0119
:10DA60008A859B858617970731F0888199810E9466
:10DA7000D6D41B870A87B701888199810E942FCD50
:10DA80002E813F81820F932F911D9F838E8390E083
:10DA900080E0CDB7DEB7E6E00C94F7F1B0E0A0E0AF
:10DAA000E4E5FDE60C94D7F1EC017B018A018A855F
:10DAB0009B858617970731F0888199810E94D6D47B
:10DAC000FB86EA8688859985019609F5CC80DA80FF
:10DAD0008E81D80EA880B980D5015596ED91FC9124
:10DAE000C5010995C80E780110E0F70121917F0169
:10DAF00021111FC08E819F81810F911D9F838E8375
:10DB000090E080E0CDB7DEB7EAE00C94F3F1EE8070
:10DB1000FF80B801888199810E942FCD8E0D9F2DA5
:10DB2000911D288539852817390780F681E090E016
:10DB3000E9CF4C2D6D2DC5010E942ED5D80E180FA2
:10DB4000D4CFB0E0A0E0E7EAFDE60C94DAF1EC0116
:10DB5000D62E1CAD0BAD7C0184E0E80EF11CE98DE6
:10DB6000FA8DC7010995412F480F2D2D602FC70150
:10DB70000E942ED59BAD890F8BAF81E090E0CDB791
:10DB8000DEB7E7E00C94F6F1682F70E090E080E0FB
:10DB90000C944CB48091FD059091FE05009731F0F6
:10DBA0004AE050E070E060E00C940AE960E070E068
:10DBB000CB0108958091FD059091FE05009731F00D
:10DBC0004AE050E070E060E00C94DDE760E070E077
:10DBD000CB010895EFDF97FD0AC0ECDF6F3F7105C1
:10DBE0008105910509F02CF4E5DF862F089580E08A
:10DBF00008958FEF0895CF93C62F67DC882311F027
:10DC0000E9DFC82F8C2FCF9108958091FD05909169
:10DC1000FE05892B39F0DEDF91E0811101C090E033
:10DC2000892F089591E0FCCFCF93DF93C82FD62F93
:10DC30004CDC882321F0E9DFDF91CF9108958C2F10
:10DC4000CDDB8111F9CF8D2FF7CFB4DFCB01089554
:10DC5000CF93DF93EB0139DC882311F0F6DFEC0181
:10DC6000CE01DF91CF9108950F931F93CF938091B1
:10DC7000FD059091FE050097D9F0FC018F01C1913F
:10DC80002C2F2F7D81F0C53411F0C536B9F7F8017E
:10DC9000108270E060E00E9487E6F801C083CF91B7
:10DCA0001F910F91089570E060E00E9487E6F7CF22
:10DCB00060E070E0CB01F3CFCF92DF92EF92FF9262
:10DCC0006A017B0102DC882319F0CEDF6B017C0145
:10DCD000C701B601FF90EF90DF90CF900895CF92EB
:10DCE000DF92EF92FF92CF93C82F0E94EBD16B018E
:10DCF0007C0124EA30E74DE75FE360910801709111
:10DD0000090180910A0190910B010E94E9EA87FDC7
:10DD100018C08AEF90E0A0E0B0E08C0D9D1DAE1D14
:10DD2000BF1D80936A0690936B06A0936C06B09318
:10DD30006D06C0936201CF91FF90EF90DF90CF907E
:10DD4000089580E090E0DC01E8CFCF938091390620
:10DD5000811154C01092B9131092BA131092BB13D0
:10DD600010928713109286131092891310928813C1
:10DD700010928B1381E080938A1382E280938C133C
:10DD80001092911310929013E5EAF3E123EB33E143
:10DD90008FEF81932E173F07E1F7C1E0C093A213E5
:10DDA00020E832EB3093981320939713C093991384
:10DDB00010929A1310929B1390E490939C131092DC
:10DDC0009D132FE732EB3093B4132093B3132AE55E
:10DDD00031E030938513209384139EE19093A9132F
:10DDE00091E19093AA139CE19093A7138093A613BB
:10DDF0008093A5130E9428D3C093390681E08093B5
:10DE0000380686EB92E29093AC128093AB1210929C
:10DE1000AE121092AD1253985B9A52985A9A389853
:10DE2000409A0E94DA6510929802CF910895FC0101
:10DE300080E0309749F09491992331F0907C9038AC
:10DE400009F08F5F3196F7CF0895B0E0A0E0EBE2E4
:10DE5000FFE60C94D7F1EC015B018A01FB01099507
:10DE600087FD10C0C82ED12CF12CE12C2196F80191
:10DE7000C082D182E282F382CE01CDB7DEB7EAE082
:10DE80000C94F3F1982F907E903CA9F48F7190E060
:10DE9000B0E0A0E06C017D0156E0CC0CDD1CEE1C76
:10DEA000FF1C5A95D1F7CE010196F50109958F73A4
:10DEB000C82A2296DCCF982F907F903E11F58F7064
:10DEC00090E0B0E0A0E06C017D0136E0CC0CDD1C00
:10DED000EE1CFF1C3A95D1F7CE010196F50109958C
:10DEE0008F73C82A46E0CC0CDD1CEE1CFF1C4A9543
:10DEF000D1F7CE010296F50109958F73C82A2396B2
:10DF0000B6CF982F987F903F79F5877090E0B0E07A
:10DF1000A0E06C017D0186E0CC0CDD1CEE1CFF1C3A
:10DF20008A95D1F7CE010196F50109958F73C82A1C
:10DF300096E0CC0CDD1CEE1CFF1C9A95D1F7CE01AF
:10DF40000296F50109958F73C82A26E0CC0CDD1CDA
:10DF5000EE1CFF1C2A95D1F7CE010396F501099519
:10DF60008F73C82A249683CF982F907C903841F4E1
:10DF7000807C803869F42196CE01F5010995F8CFAF
:10DF80008E7F8D3F28F02196CE01F5010995F8CFBF
:10DF9000C12CD12C76016BCF9CE0899F802D112460
:10DFA00091E0980F909337062CE0280F20937E077E
:10DFB00030E02E5F3F4F4091B6134217130619F021
:10DFC00014F080E008952091B8139217D0F76623DB
:10DFD00041F08E5F0E940DD480917E078E5F0E947B
:10DFE0000DD480917E079091B613891750F320913C
:10DFF000B81390913706291720F31092B913809324
:10E00000BA1381E0089520913606022E000C330BDE
:10E010008217130641F08093360661E274E282E8CB
:10E0200093E10C94D6D40895ACE0B0E0EAE1F0E7D7
:10E030000C94D9F16F3F71058105910509F070F4D9
:10E040008EE793E17EDDE0918613F09187133196A0
:10E05000849190E02C96E8E00C94F5F1F090B913DF
:10E06000E090BA132091380621110FC048E852E21F
:10E070006E2D8F2D0E9487D590E080E0F80EF092F3
:10E08000B913E092BA139927E5CFC0908613D090C8
:10E09000871322E833E13A8329832F2D30E03C8334
:10E0A0002B832E2D30E03E832D8318861F822FEF89
:10E0B0003FEF3A8729871C861B860EE41DE69E01EA
:10E0C0002F5F3F4FAB01BC01C6010E948EB3B6016A
:10E0D00082E893E10E94D6D48F819885CFCF4F926A
:10E0E0005F926F927F928F929F92BF92CF92DF92B8
:10E0F000EF92FF920F931F93CF93DF93CDB7DEB7CD
:10E1000028970FB6F894DEBF0FBECDBF7C016A0121
:10E110004901FB0190818CE0989F800D1124982F7C
:10E12000F7012081822F880F820F880F8093B91307
:10E130009093BA134115510559F1FA82E9827C8313
:10E140006B8301111EC0AE014B5F5F4FB401C6016E
:10E150007CDE6C016D817E818F81988561157105F2
:10E1600081059105A9F060DFF70180818F5F8083D1
:10E17000853148F3CE01019631D8E5CFB12C860127
:10E1800029C08A01B12C26C0452846284728B1F766
:10E1900028960FB6F894DEBF0FBECDBFDF91CF91AA
:10E1A0001F910F91FF90EF90DF90CF90BF909F90C5
:10E1B0008F907F906F905F904F900895B39407C0B9
:10E1C000B1102DC001151105C9F20F5F1F4F0115C8
:10E1D0001105A9F2AE014B5F5F4FB401C60135DEF8
:10E1E0006C014D805E806F8078844114510461041D
:10E1F0007104A9F0F0E24F1651046104710401F3B7
:10E20000D301C2018D97A109B1090297A105B105FA
:10E2100030F04BE2441651046104710479F6F701C1
:10E220008081482F4B0D5527551F4631510534F03D
:10E23000853020F0CE0101960E94EE6881E0411405
:10E2400051046104710409F480E0B80EF701808183
:10E250008B0D8083BB2009F497CFBA94AE014B5F3E
:10E260005F4FB401C801F1DD8C016D817E818F812A
:10E270009885DADEEFCFCF93DF93FC0125AD211136
:10E2800004C021E025AF0E9428D3C0918413D0910F
:10E290008513E091B313F091B41382E00995E091F6
:10E2A000B313F091B41381E0099530E020E044E12C
:10E2B000BE0182E893E10E9423D325EB33E147E1DD
:10E2C000BE0182E893E10E9423D3E091B313F09161
:10E2D000B41380E00995DF91CF9108954F925F923A
:10E2E0006F927F928F929F92AF92BF92CF92DF9266
:10E2F000EF92FF92CF93DF9300D000D0CDB7DEB77F
:10E300000E94EBD16B017C01809162018F3FC1F1D2
:10E310000E94EBD180906A0690906B06A0906C06EC
:10E32000B0906D06681979098A099B0997FD28C084
:10E3300080916A1390916B138F5F8F70891701F131
:10E34000E0916201E53008F0DCC024E0E29FF001DA
:10E350001124E95BFD4F80819181A281B381898382
:10E360009A83AB83BC8320E030E0A901BE016F5FDC
:10E370007F4F8AE791E00E94C2C78FEF80936201CE
:10E380000E94DA658091990282FFC4C0809179066B
:10E3900081111DC091E09093790680919E0289279A
:10E3A00080935A0710929E0283E080936F0110922F
:10E3B00099020E94EBD16C507E4F8F4F9F4F60931C
:10E3C0009A0270939B0280939C0290939D0280918D
:10E3D000750690917606A0917706B0917806A70110
:10E3E0009601281B390B4A0B5B0BDA01C901B7FFF9
:10E3F00005C080919F02882309F4C5C1D701C601D9
:10E400008C599F4FAF4FBF4F809375069093760600
:10E41000A0937706B093780660919802062E000CC0
:10E42000770B77FF03C07195619571099091980200
:10E4300080917406981371C0633008F06EC010921A
:10E4400098028091980280937406643008F075C039
:10E4500080915A078111F3C080917C1390917D13B4
:10E460008A509C4741F480916301882309F4F9C0E4
:10E470008150809363010E94A72F8090AE079090F7
:10E48000AF07A090B007B090B10781110E94B42FE0
:10E49000D501C4013AE0B695A795979587953A9529
:10E4A000D1F7009741E0A407B10520F08FEF9FEF6F
:10E4B000A0E0B0E09695879520916F012111E3C00F
:10E4C00030919F0231118BC180917C1390917D130B
:10E4D0008A509C4709F46AC18091A002811166C1EB
:10E4E0008091700690917106A0917206B0917306AA
:10E4F000C81AD90AEA0AFB0AF7FC66C10E948D47CE
:10E5000063C18091700190917101A0917201B091ED
:10E51000730125CF109279065ACF633009F091CF5D
:10E520008091980287FD07C081E0880F880F809353
:10E53000980264E086CF8FEFF8CF80917D0721E0CD
:10E5400030E040E050E0882309F456C0809079071D
:10E5500090907A07A0907B07B0907C07811491047B
:10E56000A104B104E9F170E090E080E00E94EDEADE
:10E5700020E030E040E85EE30E944EEB2B013C01DE
:10E58000C701B601681979098A099B090E94EDEA59
:10E590009B01AC01C301B2010E947EF220E030E099
:10E5A0004AE754E40E944EEB4B015C0120E030E06E
:10E5B00040EA52E40E946AF324E630E040E050E092
:10E5C00087FF12C020E030E040EF51E4C501B40104
:10E5D0000E946AF32AE030E040E050E087FF04C088
:10E5E00021E030E040E050E0C0927907D0927A0715
:10E5F000E0927B07F0927C07A09198020A2E000C13
:10E60000BB0B0E945FF124E030E040E050E00E944C
:10E6100039F18091750790917607A0917707B091B5
:10E620007807820F931FA41FB51F809375079093DF
:10E630007607A0937707B093780710929802D701D6
:10E64000C6018856954CAF4FBF4F8093700690938C
:10E650007106A0937206B093730681E080936F01F8
:10E66000FBCE8CE08093630180916E0690916F06E3
:10E67000009729F0019790936F0680936E0681E0D2
:10E6800080936F01F8CE009741F040916E06509153
:10E690006F064817590708F017CF80919F02811124
:10E6A00011C0223038F0243008F43FC0243011F477
:10E6B00010926F018EE793E1DEDD81E080937407B5
:10E6C00080939F0283E09FDC81E08093A213E0911E
:10E6D0007C13F0917D1309951092740780919F022D
:10E6E000811127C010925A0780917C1390917D135D
:10E6F0008A509C4709F0F0CE0E94EBD1DC01CB019F
:10E700008C199D09AE09BF0980906E0690906F0626
:10E71000B12CA12C88169906AA06BB0608F0D4CE07
:10E7200090936F0680936E06CFCE81E080936F0149
:10E73000C1CF82E893E10E94A6D491E0811101C08B
:10E7400090E090939F02882369F280917C139091CE
:10E750007D138A509C47B9F40E94EBD1DC01CB01B8
:10E760008C199D09AE09BF09C0906E06D0906F0646
:10E77000F12CE12CC816D906EA06FB0620F490938A
:10E780006F0680936E060F900F900F900F90DF91A1
:10E79000CF91FF90EF90DF90CF90BF90AF909F9080
:10E7A0008F907F906F905F904F90089548E9C40ECE
:10E7B0004AE3D41EE11CF11CC0927006D09271068F
:10E7C000E0927206F092730680919F028111DBCF76
:10E7D00080916F018130B9F610926F01D4CF00970C
:10E7E00009F470CF52CFACE0B0E0E9EFF3E70C945E
:10E7F000D9F1F090B913E090BA13209138062111A5
:10E8000012C048E652E26E2D8F2D0E9487D590E00F
:10E8100080E0F80EF092B913E092BA1399272C9683
:10E82000E8E00C94F5F1C0908613D090871322E8AD
:10E8300033E13A8329832F2D30E03C832B832E2D27
:10E8400030E03E832D8318861F827A8769871C8675
:10E850001B860EE41DE69E012F5F3F4F44E059E604
:10E86000BC01C6010E9423B4B60182E893E10E9474
:10E87000D6D48F819885CDCFA4E0B0E0E2E4F4E770
:10E880000C94D5F17C01062F5A01122F862F660FAA
:10E89000990B9C01255C3D4F690186E0882E912CE7
:10E8A00011160CF03DC0AE014F5F5F4F64E079E69A
:10E8B000C701CBDA7C0169817A818B819C816115EA
:10E8C00071058105910561F16D3371058105910532
:10E8D00009F450C06E3771058105910509F44AC0ED
:10E8E0006A3271058105910501F507FF11C08CEAB7
:10E8F00092E20E3F11F088EA92E236E01302B00194
:10E90000112471DF66E070E00E94A1F1161B60C067
:10E9100065E470E080E090E087DB115069F510E07D
:10E92000812F2496ECE00C94F1F16432710581059D
:10E93000910571F4A114B104D1F0E6E01E02B0011A
:10E940001124C50150DFB4010E94A1F1161BA8CF0C
:10E95000603471058105910551F41150F601608113
:10E96000062E000C770B880B990B5EDB99CF5CDBD6
:10E97000115096CF07FDBBCF61E089819A81AB81B1
:10E98000BC81CD97A105B10509F460E0600F6A3044
:10E99000A4F01150862F6AE00E9480F1092F682FA1
:10E9A000880F770B605D7F4F072E000C880B990B4B
:10E9B0003BDB112309F4B3CF602F062E000C770B3D
:10E9C000605D7F4F072E000C880B990B2DDB1150DB
:10E9D000112309F4A4CF86E01802B0011124C70165
:10E9E00002DF66E070E00E94A1F1161B99CFEEE70E
:10E9F000F3E183AF64AF6FEF7FEFCA01F4CEACE019
:10EA0000B0E0E5E0F5E70C94D9F1F090B913E090AF
:10EA1000BA1320913806211112C048E452E26E2D3B
:10EA20008F2D0E9487D590E080E0F80EF092B91308
:10EA3000E092BA1399272C96E8E00C94F5F1C09077
:10EA40008613D090871322E833E13A8329832F2D50
:10EA500030E03C832B832E2D30E03E832D831886BF
:10EA60001F827A8769871C861B860EE41DE69E013D
:10EA70002F5F3F4F47E059E6BC01C6010E9423B417
:10EA8000B60182E893E10E94D6D48F819885CDCFDC
:10EA90006FEF7FEFB4CFB0E0A0E0E1E5F5E70C94D5
:10EAA000D7F15C016B01C3D9E82EC6010E940A6947
:10EAB000F12C03E110E0081B1109C5E20E151F053A
:10EAC0000CF4CFE18C2F90E09C012E5F3F4F4091E2
:10EAD000B6134217130609F08CF509972091B81365
:10EAE000281719065CF140918007509181076091C9
:10EAF0007F071092B913C093BA1325E1C501BCDE9C
:10EB0000D1E0C114D104A9F06AE370E080E090E0A4
:10EB10008BDA0E151F05A4F4C45F8091B613C817D5
:10EB200040F02091B8134C2F4950550B241715066F
:10EB30004CF4CDB7DEB7EAE00C94F3F1D0E0E1CFCE
:10EB4000DD23B9F3802F880F080F000F0093B9134E
:10EB5000C093BA1360E270E080E090E065DAC6012D
:10EB600097DFE7CFACE0B0E0E8EBF5E70C94D5F148
:10EB7000982F862F6A017901B02E692F0DDA88232C
:10EB800009F487C010913806C701002371F14FD9ED
:10EB9000A82E8090861390908713111142C02FEFFA
:10EBA0003FEF122F23E12A194091800750918107EE
:10EBB00060917F07C60160DEAA2009F46AC0B6E052
:10EBC0008B9F600111246AE370E080E090E02CDA12
:10EBD00057E0C516D10408F442C060E270E080E05E
:10EBE00090E022DAC81AD90AF3CF0E940A69A82E47
:10EBF0008090861390908713112389F2FE0133963B
:10EC00008AE0DF011D928A95E9F782E893E19A8311
:10EC1000898307E21DE69E012F5F3F4F47E059E6DB
:10EC200012C0FE0133968AE0DF011D928A95E9F752
:10EC300082E893E19A83898307E21DE69E012F5FB4
:10EC40003F4F44E059E6B701C4010E9423B4B40128
:10EC500082E893E10E94D6D42F813885A2CF4091DB
:10EC60007E07212F30E0A6E0AA9EC00111242E5F6E
:10EC70003F4F281739070CF49C0180E8821B8093D2
:10EC8000B9134093BA13BB2041F06FEF7FEFC70178
:10EC9000AADD2C96ECE00C94F1F1C701F9DEF9CF76
:10ECA000EEE7F3E183AF64AFCA01F2CE0C94A9B4EE
:10ECB0004F925F926F927F928F929F92BF92CF926C
:10ECC000DF92EF92FF920F931F93CF93DF931092F7
:10ECD0002E0610922D062FE3209331061092300657
:10ECE00010922F061092290610922A0610922B06D7
:10ECF00010922C069C01F90190812F5F3F4F9032BA
:10ED0000D1F39E34C9F4818190ED980F9A3020F0B0
:10ED10008D3211F08B3281F432969F012F5F3F4F7D
:10ED2000808180538A3008F46DC09F012F5F3F4F70
:10ED30008081803209F468C0F0939507E0939407CE
:10ED40008F010F5F1F4FC0816AE270E0C8010E940F
:10ED500020F4009731F0FC01319780818032E1F39B
:10ED60001182CD3421F0C43511F0C734D9F5F80142
:10ED700080810F5F1F4F8032D1F380538A3090F52E
:10ED8000C093310690E080E06AE0AF014F5F5F4FD3
:10ED9000689F9001699F300D1124C901C09720819F
:10EDA000820F911D27FD9A95FA01208120532A3068
:10EDB00060F39093300680932F06DF0131962C91FB
:10EDC0002032D9F3CD3461F58E31910539F0F0F46C
:10EDD0008731910519F08C31910511F5B0932E060C
:10EDE000A0932D06DF91CF911F910F91FF90EF908F
:10EDF000DF90CF90BF909F908F907F906F905F90AB
:10EE00004F900895F90189CFF9018FCF853791058A
:10EE100038F08737910510F3803A13E09107F1F24B
:10EE2000809094079090950740E050E0BA0130E060
:10EE300020E0C12CD12C7601C394FD013196DC91E8
:10EE4000DD2309F484C0D132F1F4CD34E1F4803211
:10EE50009105C9F44093290650932A0660932B0626
:10EE600070932C06F0932E06E0932D0663E270E07B
:10EE7000CF010E9420F4009709F4B4CFFC01108266
:10EE8000B1CFDF01DACFD154DA3108F05BC0DF0156
:10EE90001D91103291F0A0EDA10FAA30E8F01E32C2
:10EEA00071F4A181A053AA30B8F02115310519F4ED
:10EEB0009F0121503109B12C13C0FD01E8CF1D3253
:10EEC00011F01B3291F7A181B0EDBA0FBA3020F0EA
:10EED000AE3259F7A281E6CFBE2EB818309759F35B
:10EEE000AD2FB0E02601370104C0440C551C661C50
:10EEF000771CDA95D2F74429552966297729A15F2D
:10EF0000B94FBC92A081A154AA3108F4BACFDF0155
:10EF1000D191DD2309F491CF00EDB02EBD0E19E0A3
:10EF20001B15A8F713EDB12EBD0E11E01B1578F7D8
:10EF3000DB3269F3FD013196DC91D03209F07DCFEF
:10EF4000DF01F8CF21153105E9F69D01DBCF3093C4
:10EF50002E0620932D064093290650932A0660938F
:10EF60002B0670932C063ECFFC016591759185911F
:10EF7000949108958F929F92AF92BF92CF92DF9219
:10EF8000EF92FF92CF93DF93EC018090BA029090C2
:10EF9000BB02A090BC02B090BD0220E030E0A9010D
:10EFA000C501B4010E94E9EA882309F452C0C8806F
:10EFB000D980EA80FB80A7019601C501B4010E94B7
:10EFC000E9EA18160CF04AC02091F9053091FA05CB
:10EFD0004091FB055091FC05C701B6010E94E9EA8A
:10EFE000882321F1C092F905D092FA05E092FB0541
:10EFF000F092FC052091F5053091F6054091F7055A
:10F000005091F805C701B6010E944EEB9B01AC017F
:10F0100060E070E080E89FE30E9406F260934F0199
:10F0200070935001809351019093520160914F0170
:10F03000709150018091510190915201DF91CF91D7
:10F04000FF90EF90DF90CF90BF90AF909F908F9008
:10F05000089560E070E080E89FE3F0CF60E070E04A
:10F06000CB01ECCFB0E0A0E0E8E3F8E70C94D1F1FD
:10F07000EC012091820330918303409184035091ED
:10F080008503688179818A819B810E9406F24B0108
:10F090005C01209186033091870340918803509151
:10F0A00089036C817D818E819F810E9406F26B01B4
:10F0B0007C01A50194016091470170914801809104
:10F0C000490190914A010E94E9EA882309F454C059
:10F0D0008092470190924801A0924901B0924A0162
:10F0E0002091ED053091EE054091EF055091F0052E
:10F0F000C501B4010E944EEB2B013C010E9417F3A5
:10F100004B015C0120E030E040EA50E40E94E9EA73
:10F11000181634F4812C912CC0EAAC2EC0E4BC2E1D
:10F1200020E030E0A901C501B4010E946AF387FF25
:10F1300003C0812C912C5401A5019401C301B2019B
:10F140000E9406F26093E5057093E6058093E7055B
:10F150009093E805C501B4010E94E6F26093E305CF
:10F16000062E000C770B6F5F7F4F6630710514F031
:10F1700066E070E06093E105D09145011091E305F0
:10F18000A701960160914B0170914C0180914D0156
:10F1900090914E010E94E9EA811123C0D11375C0FC
:10F1A0002091C9053091CA054091CB055091CC05FD
:10F1B0006091E5057091E6058091E7059091E8057D
:10F1C0000E944EEB2091CD053091CE054091CF05A8
:10F1D0005091D0050E9407F2CDB7DEB7E0E10C9464
:10F1E000EDF1C0924B01D0924C01E0924D01F092B2
:10F1F0004E012091F1053091F2054091F3055091B7
:10F20000F405C701B6010E944EEB4B015C010E9460
:10F2100017F36B017C0120E030E040EA50E40E94EB
:10F22000E9EA181634F4C12CD12CB0EAEB2EB0E484
:10F23000FB2E20E030E0A901C701B6010E946AF36D
:10F2400087FF03C0C12CD12C7601A7019601C5010F
:10F25000B4010E9406F26093E9057093EA05809379
:10F26000EB059093EC05C701B6010E94E6F26093AE
:10F27000E405062E000C770B6F5F7F4F663071053B
:10F2800014F066E070E06093E205C091E405D113EC
:10F2900005C0809146018C1709F470C08091E30588
:10F2A0009091E40590934601809345010C2E000C4B
:10F2B000DD0B27E01203C0011124FC01EC0FFD1F40
:10F2C000EE0FFF1FEE0FFF1FE254FD4F2081318133
:10F2D000428153812093DD053093DE054093DF05A5
:10F2E0005093E0050091E205002E000C110BFC018B
:10F2F000E00FF11FEE0FFF1FEE0FFF1FE254FD4F57
:10F3000060817181828193810E9406F26093D905A8
:10F310007093DA058093DB059093DC052091E1057D
:10F3200037E02303F0011124CE0FDF1FCC0FDD1FC8
:10F33000CC0FDD1FC254DD4F288139814A815B81AA
:10F340002093D5053093D6054093D7055093D80523
:10F35000E00FF11FEE0FFF1FEE0FFF1FE254FD4FF6
:10F3600060817181828193810E9406F26093D10550
:10F370007093D2058093D3059093D4058090E905CE
:10F380009090EA05A090EB05B090EC052091D9058E
:10F390003091DA054091DB055091DC05C501B401DF
:10F3A0000E944EEB2091DD053091DE054091DF0596
:10F3B0005091E0050E9407F26B017C01C092CD05DF
:10F3C000D092CE05E092CF05F092D0052091D105E4
:10F3D0003091D2054091D3055091D405C501B401B7
:10F3E0000E944EEB2091D5053091D6054091D7056E
:10F3F0005091D8050E9407F2A70196010E9406F2DB
:10F400006093C9057093CA058093CB059093CC0592
:10F41000C7CEACE0B0E0EFE0FAE70C94DEF1182FD5
:10F42000882379F020E030E0A90160918A0370918F
:10F430008B0380918C0390918D030E94E9EA8823CD
:10F44000F1F08091B9028117D1F00E94D32C8CE0A9
:10F45000EFE2F2E0DE01119601900D928A95E1F75C
:10F46000CE010196FFDD8091B902882361F08AE721
:10F4700091E00E94292D1092B9020E9422402C9600
:10F48000E3E00C94FAF181E08093B9028AE791E01D
:10F490000E94F52CF2CFCF92DF92EF92FF9280E0A4
:10F4A000B8DF10928603109287031092880310929F
:10F4B00089031092820310928303109284031092A6
:10F4C000850310928E0310928F0310929003109276
:10F4D000910310928A0310928B0310928C03109266
:10F4E0008D034EEB52E027E0C12CD12C60ECE62ED0
:10F4F0006FE7F62E90E080E0FC01EE0FFF1FEE0FAD
:10F50000FF1FE40FF51FC082D182E282F3820196D1
:10F510008730910589F72150445E5F4F2111EACF72
:10F52000FF90EF90DF90CF9008954F925F926F928F
:10F530007F928F929F92AF92BF92CF92DF92EF9283
:10F54000FF921F93CF93DF93EC01162F2091BA0205
:10F550003091BB024091BC025091BD02688179811B
:10F560008A819B810E94E9EA882309F497C0B090C0
:10F57000B90280E04EDFC880D980EA80FB8020E0BD
:10F5800030E0A901C701B6010E946AF387FF03C0FA
:10F59000C12CD12C7601C092BA02D092BB02E0926B
:10F5A000BC02F092BD022DEB37E346E855EBC701F4
:10F5B000B6010E94E9EA87FD0BC02DEB37E346E870
:10F5C00055E3C701B6010E946AF318160CF076C025
:10F5D000A701960160E070E080E89FE30E947EF260
:10F5E0006093F5057093F6058093F7059093F80501
:10F5F00080EF9FEFA9E7B4EC8093F9059093FA05AB
:10F60000A093FB05B093FC05BB2009F447C04090D4
:10F610007A0150907B0160907C0170907D01809018
:10F620007E0190907F01A0908001B0908101C090F8
:10F630008201D0908301E0908401F090850181E007
:10F64000E8DE112359F1A301920160917A017091D2
:10F650007B0180917C0190917D010E94E9EA8111FA
:10F660001BC0A501940160917E0170917F01809182
:10F670008001909181010E94E9EA81110DC02091E1
:10F680008201309183014091840150918501C7012D
:10F69000B6010E94E9EA81110E947040DF91CF918A
:10F6A0001F91FF90EF90DF90CF90BF90AF909F9011
:10F6B0008F907F906F905F904F90089560E070E022
:10F6C000CB018ECF8F929F92AF92BF92CF92DF925B
:10F6D000EF92FF92C0908A03D0908B03E0908C034E
:10F6E000F0908D0320E030E0A901C701B6010E942F
:10F6F000E9EA8823E1F1A701960160E070E080E883
:10F700009FE30E947EF26B017C0180908E039090BB
:10F710008F03A0909003B090910320E030E0A90106
:10F72000C501B4010E94E9EA882329F1A5019401E9
:10F7300060E070E080E89FE30E947EF2C092ED05F9
:10F74000D092EE05E092EF05F092F0056093F1059E
:10F750007093F2058093F3059093F405FF90EF907A
:10F76000DF90CF90BF90AF909F908F900895C12C65
:10F77000D12C7601CACF60E070E0CB01DFCFCF9211
:10F78000DF92EF92FF926B017C0183E3C816D104F4
:10F79000E104F10470F082E3C81AD108E108F1082D
:10F7A00062E370E080E090E00E9462D10E94152A3E
:10F7B000ECCFC701B6010E9462D10E94152AFF90CA
:10F7C000EF90DF90CF900895BC0190E080E00C9422
:10F7D0004CB480919207813069F09091D41492FBDF
:10F7E000882780F992FF07C097FB882780F991E06E
:10F7F0008927089581E008959091D41494FB882777
:10F8000080F994FF06C081E09091D112911101C05E
:10F8100080E00895A4E0B0E0E0E1FCE70C94D1F1D1
:10F8200010927D0780915A0710925A07882361F041
:10F8300020E040E070E060E08BE793E60E945146F4
:10F840002496E0E10C94EDF120911001309111012A
:10F850004091750750917607CA01820F931F243695
:10F86000310509F01DC44730510544F006978A3030
:10F8700091050CF024C48AE090E02BC406964A3F20
:10F880005F4FACF380917407882309F4C8C160917D
:10F89000BD127091BE12072E000C880B990B0E94AE
:10F8A000EFEAB1E0B9832091B9123091BA124091D8
:10F8B000BB125091BC120E946AF318160CF0198208
:10F8C00060913F0770914007072E000C880B990B41
:10F8D0000E94EFEA20913B0730913C0740913D07A1
:10F8E00050913E070E946AF318161CF4E981E26009
:10F8F000E983C980C0926906C0907A01D0907B01EB
:10F90000E0907C01F0907D0180917E0190917F01DB
:10F91000A0918001B091810189839A83AB83BC83DC
:10F920008090820190908301A0908401B090850125
:10F9300020E030E04AE754E4C501B4010E944EEBF8
:10F940002B013C0120E030E0A901C501B4010E9477
:10F95000E9EA20E030E040EA50EC87FD04C020E016
:10F9600030E040EA50E4C301B2010E9407F22DECFE
:10F970003CEC4CEC5DE30E944EEB0E94E6F24B0146
:10F980005C0180E2B7FE09C0B094A094909480948A
:10F99000811C911CA11CB11C8DE28093A10260E22C
:10F9A00090E1891697E29906A104B1048CF0C50193
:10F9B000B40120E137E240E050E00E9439F1CA0191
:10F9C000B9012AE030E040E050E00E9439F1605D8A
:10F9D0006093A20260E2A8EE8A16A3E09A06A10450
:10F9E000B1048CF0C501B40128EE33E040E050E0F2
:10F9F0000E9439F1CA01B9012AE030E040E050E04C
:10FA00000E9439F1605D6093A302C501B40124E650
:10FA100030E040E050E00E9439F16AE0462E512C7F
:10FA2000612C712CCA01B901A30192010E9439F124
:10FA3000605D6093A402C501B401A30192010E941C
:10FA400039F14B01CA01B901A30192010E9439F1B8
:10FA5000882009F44EC32EE22093A502605D6093D6
:10FA6000A602B0E38B0E8092A70261EA72E081E603
:10FA700096E00E942BF420E030E0A901C701B60116
:10FA80000E94E9EA20E030E040E05FEB87FD04C03F
:10FA900020E030E040E05FE3C701B6010E9407F2DA
:10FAA0000E94E6F2CB010E943145BC018CE596E054
:10FAB0000E942BF420E030E0A90169817A818B81DA
:10FAC0009C810E94E9EA20E030E040E05FEB87FDA6
:10FAD00004C020E030E040E05FE369817A818B81FF
:10FAE0009C810E9407F20E94E6F2CB010E94314500
:10FAF000BC0187E596E00E942BF48091D41483FD2D
:10FB00000AC37ADE882309F409C38091CC1490914A
:10FB1000CD14A091CE14B091CF140097A105B105DA
:10FB200009F4FCC2BC01CD016D597F4F8F4F9F4F2F
:10FB300024E630E040E050E00E9417F16091D014DC
:10FB40007091D1148091D2149091D3140E9417F126
:10FB500029830E9470444B015C01162F8091610142
:10FB6000C9808C15C1F0C092610128E4C29EB00129
:10FB7000112490E080E00E94EDEA2AE037ED43E2B4
:10FB80005CE30E944EEB0E94EBF260935606C110BC
:10FB9000C7C21092510680916001181709F43FC046
:10FBA00080926001C501B40120E13EE040E050E0F8
:10FBB0000E9417F1690189019CE3492E512C612CA7
:10FBC000712CC501B401A30192010E9417F14B01F0
:10FBD0005C01CA01B901A30192010E9417F1C1148D
:10FBE000D10409F0C4C29F928F927F936F938CECE3
:10FBF00092E29F938F9381E496E09F938F930E946C
:10FC000082EA0FB6F894DEBF0FBECDBF85E0982F15
:10FC1000990F990F891B880F8058809340060E9486
:10FC2000EBD100913B0610913C0620913D063091AE
:10FC30003E066B017C01C01AD10AE20AF30A970161
:10FC4000860137FD11C020913A06209520933A068F
:10FC50006A547C4F8F4F9F4F60933B0670933C06D6
:10FC600080933D0690933E06D0903A06D98281E07B
:10FC70000E9403708091B613873180F48091B8138D
:10FC8000843060F08FEAE82E83E2F82E03E126E06C
:10FC900044E064E082E893E10E94ACD5809169067B
:10FCA000982F927048E00CE081FD02C042E102E032
:10FCB0008091B613843180F48091B813841760F07A
:10FCC000992309F473C28BE893E27C0123E060E599
:10FCD00082E893E10E94ACD58091B6138431C0F4E0
:10FCE0008091B8138230A0F0C980CC2009F461C2A1
:10FCF0008091B207882309F45CC28FE493E27C010F
:10FD000002E123E042E068E682E893E10E94ACD59C
:10FD10008091B6138C3108F09DC08090B9129090FC
:10FD2000BA12A090BB12B090BC12C090BD12D0907D
:10FD3000BE12843198F48091B813883078F08091A5
:10FD4000690680FF39C281E093E27C010CE022E089
:10FD500048E069E382E893E10E94ACD58091B61354
:10FD6000883040F4D7FE2BC245EE52E267E087E3CD
:10FD70000E94F7748091B6138C31B0F48091B8135F
:10FD8000843190F020E030E040E05FE3C501B40151
:10FD90000E9407F20E94E6F277FF34C245EE52E27B
:10FDA0006CE187E30E94F774C0903B07D0903C075A
:10FDB000E0903D07F0903E078091B613883060F4E4
:10FDC00080913F079091400797FF3FC245EE52E276
:10FDD00067E081E50E94F7748091B6138C31B0F42E
:10FDE0008091B813843190F020E030E040E05FE390
:10FDF000C701B6010E9407F20E94E6F277FF47C2F0
:10FE000045EE52E26CE181E50E94F7748091B613F1
:10FE10008C3100F58091B8138431E0F08091B20705
:10FE20008823C1F024E6829FC001112481589F4F8E
:10FE30006FEF70E00E94A1F1CB010E94B045AC01D0
:10FE40006CE187E60E94507665E270E080E090E029
:10FE50000E941470D1DC882379F18091B613843329
:10FE600058F58091B8138A3238F107E028E04AE269
:10FE70006AE282E893E10E9453D405E022E04CE27A
:10FE800062E382E893E10E9453D424E04AE061E314
:10FE90008AE20E9423D4609184137091851382E3D7
:10FEA00080939E138BE280939F132EE933E142E30C
:10FEB00082E893E10E9423D38091B613853350F4F6
:10FEC0008091B813813330F024E04AE461E386E3A3
:10FED0000E9423D48091B613843368F48091B813C0
:10FEE000823348F002E02091560642E367E382E85D
:10FEF00093E10E9453D48091B6138033D8F480915B
:10FF0000B8138832B8F080915106882361F041E53A
:10FF100056E060E387E30E94507665E270E080E09F
:10FF200090E00E94147041E456E060E38091400646
:10FF30000E9450768091B613883208F060C080919C
:10FF4000B8138D3108F45BC02BE040E86DE180E030
:10FF50000E9423D48091B613873208F050C080915C
:10FF6000B8138F3108F44BC083E08093B91316E2C5
:10FF70001093BA1368E570E080E090E00E9414707E
:10FF80008BE08093B9131093BA13C980CC2009F485
:10FF9000A1C18CE596E00E94487588E28093B91370
:10FFA00016E21093BA1369E570E080E090E00E94D9
:10FFB000147080E38093B9131093BA13C980CC20D6
:10FFC00009F4ABC187E596E00E9448758DE4809303
:10FFD000B91316E21093BA136AE570E080E090E07E
:10FFE0000E94147085E58093B9131093BA13C980E9
:10FFF000CC2009F4B5C181E696E00E944875809155
:020000021000EC
:10000000B613833338F58091B8138B3218F183E03F
:100010000E94037083E08093B91383E38093BA1343
:1000200066E070E080E090E00E94147081E00E9441
:10003000037080911001909111010E94B045AC01B4
:1000400063E38CE00E94507665E270E080E090E02F
:100050000E9414708091B613813408F0F1CB809126
:10006000B813863308F4ECCB1092B9138EE3809367
:10007000BA138AE490E10E940A69182F863108F0C9
:1000800092C18AE490E10E944875153109F4D8CBF9
:1000900060E270E080E090E00E9414701F5FF5CF96
:1000A000243631054CF48536910504F58A309105E6
:1000B00034F48AE090E009C084369105BCF0883EB3
:1000C000A3E09A0714F087EE93E02817390709F4A4
:1000D000D9CB909311018093100110927507109263
:1000E00076071092770710927807CCCB84E690E0E1
:1000F000F0CF662351F02EE22093A502605D60935D
:10010000A60280E28093A702B0CC80E28093A60290
:100110008093A502F6CFE4E6E9831BCD198219CDC1
:10012000498180E2443628F0842F64E60E9474F10D
:10013000805D8093A502698190E26A3040F02AE0F8
:10014000862F622F0E9474F10E9474F1905D90934B
:10015000A60289816AE00E9474F1905D9093A702E3
:1001600065EA72E081E596E00E942BF414CD043636
:10017000110538F47F936F93DF92CF9280EC92E277
:1001800038CD7F936F93DF92CF9286EB92E29F936D
:100190008F9381E496E09F938F930E9482EA0FB63B
:1001A000F894DEBF0FBECDBF86E031CD85E893E287
:1001B0008CCD89E193E2A3CD89EE92E2C6CDC60152
:1001C0000E94B045FC01808193E0803229F4818156
:1001D00092E0803209F491E043E050E0491B51097C
:1001E0004E0F5F1F892F880F880F981B892F67E09C
:1001F000805C0E94507669E070E080E090E00E94B0
:100200001470B8CDCB010E94B045FC01808193E011
:10021000803229F4818192E0803209F491E043E058
:1002200050E0491B51094E0F5F1F892F880F880F1F
:10023000981B892F6CE1805C0E94507669E070E029
:1002400080E090E00E941470AFCD0E94B045FC01A8
:10025000808193E0803229F4818192E0803209F438
:1002600091E043E050E0491B51094E0F5F1F892F79
:10027000880F880F981B892F67E0865A0E94507656
:1002800069E070E080E090E00E941470A5CDCB01A1
:100290000E94B045FC01808193E0803229F4818185
:1002A00092E0803209F491E043E050E0491B5109AB
:1002B0004E0F5F1F892F880F880F981B892F6CE1C5
:1002C000865A0E94507669E070E080E090E00E94DB
:1002D00014709CCD87E00E94CF3B80FF13C00CE5DB
:1002E00016E0D8016D918D01662309F456CE6F3268
:1002F0000CF06FE3062E000C770B880B990B0E9415
:100300001470EFCF8091820780FD43CE6FEF7FEFB7
:1003100080EE92E20E94F37340CE87E00E94CF3BD2
:1003200081FF13C007E516E0D8016D918D016623AA
:1003300009F44CCE6F320CF06FE3062E000C770BF5
:10034000880B990B0E941470EFCF8091820781FD7A
:1003500039CE6FEF7FEF80EE92E20E94F37336CEDC
:1003600087E00E94CF3B82FF13C001E616E0D80170
:100370006D918D01662309F442CE6F320CF06FE36C
:10038000062E000C770B880B990B0E941470EFCF90
:100390008091820782FD2FCE6FEF7FEF88ED92E292
:1003A0000E94F3732CCE81E0C980C11001C080E0AF
:1003B00090913F068917C9F0D0904910D982809357
:1003C0003F068AE490E10E940A69D81608F054C0FA
:1003D00029812F5F2983E22FF0E0E65BFF4E8081C9
:1003E000807C8038A9F3209349100091491010E0D7
:1003F000065B1F4EC8010E940A69898360E870E0AD
:10040000C8010E94FF744981453108F019CA60E2B1
:1004100070E080E090E00E9414706981643109F41A
:100420000FCA60E270E080E090E00E941470898161
:10043000833109F405CA60E270E080E090E00E9438
:1004400014709981923109F4FBC9292F30E02E5F95
:100450003F4F4AEF4203B001439F700D1124605893
:100460007F4F8AE490E10E94FF7460E270E080E0D8
:1004700090E00E941470E4C910924910B6CF8091A8
:100480009207823059F0B8D9882349F08091D4146A
:1004900082FB882780F991E08927089581E00895FB
:1004A00081E00895DC01EC918E2F90E0FC01EE0FCD
:1004B000FF1FE80FF91FEF5CFC4E80818F77808370
:1004C0000895892B79F41092900082E08093910036
:1004D0001092950010929400C19A809171008260F0
:1004E000809371000895B0E0A0E0E9E7F2E80C9491
:1004F000D4F1EC017B0188818C3008F0A4C090E03D
:10050000FC01EE0FFF1FE80FF91FEF5CFC4E80812E
:100510008F770E94D4B619821A8288812CE0622FCC
:100520000E9474F1829FB001112430E020E0AB0101
:10053000420F531FFA01EE0FFF1FE40FF51FEF5C90
:10054000FC4E908197FD07C02F5F3F4F2C30310547
:1005500071F790E0B6DF7880072D10E06801CC0CD1
:10056000DD1CF601E00FF11FEF5CFC4E808180681E
:10057000808377FC68C080E2E81682E0F8060CF021
:100580003FC08A8128E532E0281B310987FD339579
:10059000220F331F220F331F032E000C440B550B69
:1005A000898178E8872E912C881A910887FD939489
:1005B000880C991C880C991C092C000CAA08BB08F3
:1005C00060E070E0CB01F7FC0AC0B701653B710544
:1005D00014F064EB70E0072E000C880B990B2819BF
:1005E00039094A095B090E9408F124EB30E040E038
:1005F00050E00E9439F1820E931EA41EB51E7401B4
:100600008BE08715D8F0298188E890E0821B91095A
:1006100027FD9395880F991F880F991FE816F906F3
:10062000BCF402972FB7F894E601C00FD11FCF5C3E
:10063000DC4E880F991F9A8389832FBF62E370E095
:1006400080E090E09CD8CDB7DEB7EDE00C94F0F1FF
:100650002A8188E592E0821B910927FD9395880FF6
:10066000991F880F991FE816F906DCF6C701D9CF44
:10067000CF93DF93EB01682F70E086E593E133DFE2
:10068000688179818A819B81643F21E072078105BD
:10069000910520F464EF71E080E090E070D886B1BD
:1006A00082958170DF91CF910895A4E0B0E0EBE5F1
:1006B000F3E80C94DFF18EEE92E0A0E0B0E08983E5
:1006C0009A83AB83BC83BE016F5F7F4F8AE5D0DF27
:1006D0002496E2E00C94FBF1A4E0B0E0E2E7F3E85A
:1006E0000C94DFF18EEE92E0A0E0B0E089839A8373
:1006F000AB83BC83BE016F5F7F4F8AE0B9DF249676
:10070000E2E00C94FBF1A4E0B0E0E9E8F3E80C943B
:10071000DFF184EF91E0A0E0B0E089839A83AB83BE
:10072000BC83BE016F5F7F4F8CE3A2DF2496E2E0C3
:100730000C94FBF1A4E0B0E0E0EAF3E80C94DFF104
:1007400084EF91E0A0E0B0E089839A83AB83BC831F
:10075000BE016F5F7F4F80EA8BDF2496E2E00C944E
:10076000FBF11F920F920FB60F9211240BB60F924E
:100770002F933F934F935F936F937F938F939F93A9
:10078000AF93BF93EF93FF938091B90587FF27C085
:1007900010929500109294008091B9058F5F80931C
:1007A000B9058091B905082E000C990B20915513BD
:1007B0002817190629F024F08091B9058C30DCF156
:1007C0008091940090919500049680349C4908F49F
:1007D0007DC08091940090919500049679C080919D
:1007E000B905082E000C990B2091551328171906EE
:1007F00099F294F2E091B9058E2FEE0F990BFC015E
:10080000EE0FFF1FE80FF91FEF5CFC4E808187FFA2
:10081000C3CFE091B9058E2FEE0F990BFC01EE0FBF
:10082000FF1FE80FF91FEF5CFC4E808160E08F77BF
:100830000E9406D1B1CF2091940030919500E091B3
:10084000B9058E2FEE0F990BFC01EE0FFF1FE80F7D
:10085000F91FEF5CFC4E81819281820F931F909370
:10086000990080939800E091B9058E2FEE0F990BB7
:10087000FC01EE0FFF1FE80FF91FEF5CFC4E8081BB
:1008800087FF11C0E091B9058E2FEE0F990BFC0187
:10089000EE0FFF1FE80FF91FEF5CFC4E808161E057
:1008A0008F770E9406D1FF91EF91BF91AF919F91F9
:1008B0008F917F916F915F914F913F912F910F9009
:1008C0000BBE0F900FBE0F901F90189580E49CE90F
:1008D00090939900809398008FEF8093B905E3CFB0
:1008E0009091C00095FFFCCF8093C6000895CF93F0
:1008F000DF93EC018991882311F0F2DFFBCFDF91C8
:10090000CF910895CF93DF93EC018991882311F063
:10091000E7DFFBCF8DE0E4DF8AE0E2DFDF91CF911C
:100920000895CF93DF93EC01FE01849121968823F3
:1009300011F0D6DFF9CFDF91CF9108950F931F9378
:10094000CF938C01C62F8AE290E2EBDFC801E9DF8A
:100950008AE3C6DF80E38C0FC3DF8AE0C1DFCF917B
:100960001F910F910895CF92DF92EF92FF926A014B
:100970007B01D7DF42E0C701B6010E94F3B6FF90CA
:10098000EF90DF90CF900895CF93DF9361E470E212
:100990000E9440C8C0916513D09166134881598167
:1009A0006A817B8188E390E2DEDF4C815D816E812C
:1009B0007F818EE39EE2D7DF4091611350916213F5
:1009C00060916313709164138BE39EE2CCDF85E347
:1009D00090E2A7DF8FE290E2A4DF8AE081DFDF917F
:1009E000CF910895C0DF8AE07BCFADE5B0E0EBEFBB
:1009F000F4E80C94CFF170E060E085E40E94286E8A
:100A00007C01182F8F3FB1F1882341F084E292E2FC
:100A100088DFC35ADF4FE2E10C94EBF16EEB70E03C
:100A200083E50E94286E5C0165E070E083E40E942B
:100A3000286E6C0160E085E50E94146E2C968FAFE5
:100A40002C9760E087E192E20E94525C0E94EBD119
:100A500069877A878B879C871F3F09F067C434E7D3
:100A6000A316B1040CF489C18CEE91E25ADF0E9406
:100A7000C4C8CFCF6CE370E0D3CF20E030E040E0DB
:100A80005EE32BAF3CAF4DAF5EAFABC12AE939E9B6
:100A900049E15FE323962CAF3DAF4EAF5FAF2397A5
:100AA000ADC14090B9125090BA126090BB127090D4
:100AB000BC1251C22B96EEADFFAD2B974083A4C262
:100AC0004BEEC42ED12CE12CF12C22C384E190E01A
:100AD000A0E0B0E08D879E87AF87B88B34E1C32E4E
:100AE000D12CE12CF12C24C3CD86DE86EF86F88A4A
:100AF0001FC32B96EEADFFAD2B978083E9C3D501C5
:100B0000C4012EA53FA548A959A9821B930BA40B8C
:100B1000B50BB7FD47C02D968FAD2D970E948C2742
:100B20008AE0DEDED501C4018053984FAF4FBF4F3E
:100B30008EA79FA7A8ABB9AB9AA991116FC02BA99B
:100B40003CA94DA95EA9C301B2010E946AF318161F
:100B50000CF050C020E030E040E050E4C301B201AE
:100B60000E9407F26BAB7CAB8DAB9EAB2AA53BA57D
:100B70004CA55DA5280D391D4A1D5B1D2FAB38AF57
:100B800049AF5AAF6D966CAD7DAD8EAD9FAD6D9793
:100B90000E94EFEAA30192010E94E9EA881F8827D8
:100BA000881F8AAB89859A85AB85BC85898F9A8F8A
:100BB000AB8FBC8F29893A894B895C892817390703
:100BC0004A075B0720F4298F3A8F4B8F5C8F898D02
:100BD0009A8DAB8DBC8D881A990AAA0ABB0A91E836
:100BE00089169FE4990692E1A906B10460F180E1BB
:100BF00091E22DC2D501C4012FA938AD49AD5AAD3E
:100C0000821B930BA40BB50B4DE053E16CE173E138
:100C1000B7FDC8CF812F0E94D328C4CF69966CAD91
:100C20007DAD8EAD9FAD69970E94EFEA9B01AC014F
:100C3000C301B2010E94E9EA87FFB4CF4AE453E15D
:100C40006AE573E1E7CF2996AEADBFAD2997A2154E
:100C5000B3050CF08FC0B3E02B1631040CF48AC03E
:100C600083EB90E25EDE1F3F09F066C0E3EAF0E24C
:100C7000FE83ED8382E990E254DE8D819E8151DE18
:100C800049815A816B817C818FEA90E2ABDE82E9F7
:100C900090E247DE8D819E8144DE4D8D5E8D6F8DAD
:100CA00078A18BEA90E29EDE82E990E23ADE8D81C5
:100CB0009E8137DE49A15AA16BA17CA187EA90E20F
:100CC00091DE2C963FAD2C97332309F4D0CE2CEA3D
:100CD00035EC47E25EE36D8D7E8D8F8D98A10E948D
:100CE0004EEB6B017C0120E030E543EC50E469A160
:100CF0007AA18BA19CA10E944EEB29813A814B8164
:100D00005C811F3FF1F420934207309343074093E7
:100D1000440750934507C0924607D0924707E09298
:100D20004807F092490760934A0770934B078093F6
:100D30004C0790934D079BCE2EE83DE23E832D83DA
:100D400099CF2093C0123093C1124093C212509396
:100D5000C312C092C412D092C512E092C612F09291
:100D6000C7126093C8127093C9128093CA129093ED
:100D7000CB127DCE0E946E71CEC088ED91E2D1DDA6
:100D80000E9435288FE7809341072CE330E0C9A605
:100D9000A8EEB3E00E9465F16AA77BA78CA79DA788
:100DA00029853A854B855C85260F371F481F591FBB
:100DB0002FAB38AF49AF5AAF81E080936E0160E04E
:100DC00084EC91E20E94525C02E00E0D023008F0C9
:100DD00054CE8BEA9AEAAAEABEE38BAF9CAFADAFE2
:100DE000BEAF023008F052CE8DEC9CECACE4BEE31A
:100DF00023968CAF9DAFAEAFBFAF2397023008F400
:100E0000E12C2D96EFAE2D9789859A85AB85BC8513
:100E1000898B9A8BAB8BBC8B8EA79FA7A8ABB9ABEA
:100E200019A21AA21BA21CA21D8E1E8E1F8E18A212
:100E300019821A821B821C822FE730E040E050E0CA
:100E40002D873E874F87588B80E090E4ACE1B6E475
:100E50008D839E83AF83B8871D8A1E8A1F8A188E52
:100E6000FFE7CF2ED12CE12CF12C1AAA1BAA1CAA29
:100E70001DAA1EAA1DA21EA21FA218A691E02496BA
:100E80009FAF2497312C212C412C512C32019501FC
:100E90000B2C000C440B550B61962CAF3DAF4EAFA5
:100EA0005FAF619749A5042E000C550B29965FAFE3
:100EB0004EAF299757E11502C0011124DC01A1545E
:100EC000BD4E2B96BFAFAEAF2B97C5014E969C0182
:100ED000092E000C440B550B65962CAF3DAF4EAF61
:100EE0005FAF6597CC979C01990F440B550B6996A2
:100EF0002CAF3DAF4EAF5FAF699736E0A31AB10894
:100F0000C5010B2C000CAA0BBB0B6D968CAF9DAFD3
:100F1000AEAFBFAF6D9780916E01882309F498C082
:100F20000E94EBD14B015C019091A7036E969FAF9D
:100F30006E97992309F47BC00E94AE291092A703F3
:100F40001F3F09F0AECD40903B0750903C076090AA
:100F50003D0770903E07A30192016D897E898F89BC
:100F6000988D0E946AF387FF04C04D8A5E8A6F8A5B
:100F7000788EA30192016D817E818F8198850E9478
:100F8000E9EA181624F44D825E826F8278866196B3
:100F90006CAD7DAD8EAD9FAD61970E94EFEA698F1C
:100FA0007A8F8B8F9C8F2496AFAD2497AA2309F458
:100FB00054C09B01AC01C301B2010E946AF3181630
:100FC000B4F5D501C40129893A894B895C89821B12
:100FD000930BA40BB50BAC01BD01485853416109FB
:100FE000710977FD24C04D855E856F8578894C1920
:100FF0005D096E097F0975956795579547951F3F60
:1010000009F058CD409341078DA39EA3AFA3B8A785
:10101000298D3A8D4B8D5C8D2D8B3E8B4F8B588F50
:1010200089869A86AB86BC8624961FAE24976596E1
:101030006CAD7DAD8EAD9FAD65970E94EFEAA301CB
:1010400092010E94E9EA87FF5ACD8EE291E269DCC3
:1010500010926E010E9435280ACD298D3A8D4B8D54
:101060005C8DC301B2010E94E9EA87FFE0CFD501A0
:10107000C40129853A854B855C85821B930BA40BA3
:10108000B50BAC01BD01485853416109710977FDA9
:10109000CECF2114310409F40AC12DA13EA14FA1E4
:1010A00058A5280F391F4A1F5B1F298B3A8B4B8B82
:1010B0005C8B2DA13EA14FA158A5281B390B4A0BD3
:1010C0005B0BC701B6010E9408F129893A894B8957
:1010D0005C890E9439F1CD84DE84EF84F888C20EE9
:1010E000D31EE41EF51E34E1C316D104E104F1045D
:1010F0000CF4ECCC4CEEC416D104E104F1040CF079
:10110000DFCC50E8C516D104E104F1040CF4ECCCBA
:10111000CD86DE86EF86F88A8EEF90E0A0E0B0E024
:101120009C01AD012C193D094E095F0969017A0145
:101130008CEB91E2F6DB6D857E858F8598890E9428
:10114000567687EB91E2EDDBC701B6010E94567639
:101150004D815E816F81788580EB91E204DC4D8961
:101160005E896F89788D89EA91E2FDDB93E029162B
:1011700031040CF49CC0C701B6010E94EFEA20E0E4
:1011800030E040E850E40E944EEB69837A838B8321
:101190009C832D813E814F8158856D897E898F8901
:1011A000988D0E9406F22BED3FE049EC5FE30E9430
:1011B0004EEB9B01AC0169817A818B819C810E94FD
:1011C0007EF227966CAF7DAF8EAF9FAF2797698970
:1011D0007A898B899C890E94EFEA2FE632E143E805
:1011E0005AE30E944EEB6D837E838F83988723960C
:1011F0002CAD3DAD4EAD5FAD239727966CAD7DAD6B
:101200008EAD9FAD27970E944EEB69837A838B83C7
:101210009C839B01AC010E9407F22D813E814F818E
:1012200058850E947EF26D8F7E8F8F8F98A32BAD95
:101230003CAD4DAD5EAD6D817E818F8198850E9404
:101240004EEB29813A814B815C810E944EEB69A370
:101250007AA38BA39CA327964CAD5DAD6EAD7FADFD
:10126000279783EA91E27FDB4D815E816F817885EC
:101270008DE991E2B7DB8EE891E2023010F08FE762
:1012800091E24FDB49815A816B817C8189E791E250
:101290006ADB4D8D5E8D6F8D78A183E791E263DB14
:1012A00049A15AA16BA17CA18DE691E29BDB8D85C2
:1012B0009E85AF85B8898C0D9D1DAE1DBF1DB59552
:1012C000A795979587951F3F09F013CC8093410709
:1012D0002996FFAD2997FF9329A52F933F922F922F
:1012E00089E591E29F938F9384E691E29F938F9398
:1012F0001F920E94355C3FEF231A330A0FB6F89411
:10130000DEBF0FBECDBF898D9A8DAB8DBC8D8D8319
:101310009E83AF83B887898A9A8AAB8ABC8A6E9685
:101320009FAD6E9724969FAF249781CE8E2C0E2C66
:10133000000C9908F40183E0EE0FFF1F8A95E1F796
:10134000EA59FE4F868197810F978A159B050CF409
:101350008BCB88ED91E2E5DA0E94352887E1889D04
:10136000F001899DF00D1124EB54FD4E8FE782872B
:1013700024E130E00CCDCF93DF936DE279E10E9460
:1013800040C8C7E3D7E04B855C856D857E8584E2E8
:1013900099E1E9DA20E030E543EC50E46F857889A3
:1013A00089899A890E944EEBAB01BC0181E299E1E7
:1013B000DADA2CEA35EC47E25EE36B897C898D89C9
:1013C0009E890E944EEBAB01BC018EE199E10ADBE4
:1013D000DF91CF9108956FEA78E10E9440C8609153
:1013E000840D7091850D8091860D9091870D0E94DE
:1013F000EDEAAB01BC0186EA98E1B5DA4091B40DA3
:101400005091B50D6091B60D7091B70D83EA98E1DA
:10141000AADA4091B80D5091B90D6091BA0D709152
:10142000BB0D80EA98E19FDA4091960750919707AB
:1014300060919807709199078DE998E1D3CACF938D
:10144000DF9363E578E10E9440C8C4E7DDE04CA982
:101450005DA96EA97FA98AE498E185DA48AD59AD06
:101460006AAD7BAD87E498E17EDA4CAD5DAD6EADE3
:101470007FAD80EA98E1B6DADF91CF910895CF93FE
:10148000DF936FE278E10E9440C8C4E7DDE04CA141
:101490005DA16EA17FA186E298E165DA48A559A514
:1014A0006AA57BA58EE39EE25EDA4CA55DA56EA5DE
:1014B0007FA58BE39EE257DA48A959A96AA97BA9BF
:1014C00088E39EE28FDADF91CF910895CF93DF9387
:1014D0006AE078E10E9440C8C4E7DDE06881798174
:1014E0008A819B810E94EDEAAB01BC0181E098E119
:1014F0003ADA6C817D818E819F810E94EDEAAB0199
:10150000BC018EE39EE22FDA688579858A859B850A
:101510000E94EDEAAB01BC018BE39EE224DA6C850C
:101520007D858E859F850E94EDEAAB01BC0188E335
:101530009EE258DADF91CF9108958F929F92AF92F9
:10154000BF92EF92FF920F931F93CF93DF938AE6A0
:1015500096E1E7D9C0E0D7E0D15019F080E2C0D9D8
:10156000FBCF8C2F0E94C46DCF5FC730A1F78AE0FC
:10157000B7D90EEB12E0C0E080E2B2D98C2F0E9406
:10158000C46D7801D7E080E2ABD9F701808091800B
:10159000A280B38020E030E0A901C501B4010E941F
:1015A0006AF387FD02C08BE29BD943E0C501B40119
:1015B0000E94F3B6D150FCE1EF0EF11CD111E3CF44
:1015C0008AE08ED9CF5F0C5F1F4FC730A9F68AE043
:1015D00087D9DF91CF911F910F91FF90EF90BF902E
:1015E000AF909F908F900895811105C08CE39FE18B
:1015F00098D98AE075C980E49FE1FACF83E696E145
:1016000090C98DE596E18DC9CF9384E50E94656A06
:10161000C0E08823D9F00E94EA6DC82F1816B4F4F0
:10162000F0DF8DE45DD980912F06909130060E9405
:10163000E47B87E29AE175D96C2FCC0F770B880B8E
:10164000990B0E94A9B48AE04BD9CFEF8C2FCF9190
:101650000895CF93C82F63E179E10E9429C8C11191
:1016600001C0CFDF4091C0125091C1126091C212EF
:101670007091C3128AE099E176D920E030E543EC1D
:1016800050E46091C4127091C5128091C61290917D
:10169000C7120E944EEBAB01BC0187E099E163D910
:1016A0002CEA35EC47E25EE36091C8127091C912F2
:1016B0008091CA129091CB120E944EEBAB01BC01FB
:1016C00084E099E150D98AE00BD9CF910895B0E038
:1016D000A0E0EDE6FBE80C94D9F161E083E50E941F
:1016E000146EC1E0C8276AE17AE18C2F0E9429C8F4
:1016F000C11101C086DF82E19AE113D98FE290E245
:1017000010D98AE0EDD860E07AE18C2F0E9429C8D8
:10171000C11101C076DF83EE99E103D98C2F0E94BD
:1017200049C88C2FACDE8C2FD1DE8C2F88DE8C2F1D
:1017300052DE69E679E18C2F0E9440C8D091B9024F
:1017400080E699E1EED86D2F70E090E080E00E9495
:10175000A9B44091BA025091BB026091BC02709151
:10176000BD028BE39EE2FFD883E599E1DAD8809150
:10177000B9023ADF20E030E0A90160918A0370915C
:101780008B0380918C0390918D030E94E9EA88235A
:1017900079F18EEBE82E82E0F82E10E0670100E090
:1017A000C11101C02EDF89ED99E1BBD8802F0E94C5
:1017B000C46D86ED99E1B5D8812F0E94C46D8BE38D
:1017C0009EE2AFD8F601608171818281938145E00C
:1017D0000E94F3B68AE084D80F5FFCE1CF0ED11CE3
:1017E0000730F1F61F5F84E0E80EF11C1730B1F608
:1017F0006DE879E18C2F0E9429C80EE417E0D0E053
:10180000C11101C0FEDE84E899E18BD88D2F0E94C2
:10181000C46DF80160817181072E000C880B990B53
:101820000E94EFEAAB01BC0181E899E19CD8F80184
:1018300062817381072E000C880B990B0E94EFEADE
:10184000AB01BC018EE799E18ED8F801E480F58008
:101850008BE799E166D8C7010E94E47B8AE040D813
:101860000A5F1F4FD13061F58C2FF3DE8C2F83DDA3
:101870008C2F8AD86FEB79E18C2F0E9440C8C091E1
:10188000320186EB99E14DD86C2F70E090E080E05A
:101890000E94A9B440912E0150912F016091300116
:1018A0007091310183EB99E15ED888EA99E139D8EA
:1018B0008091320199DECDB7DEB7E8E00C94F5F106
:1018C000D1E09ECFACE1B0E0E8E6FCE80C94CFF1CB
:1018D00083E50E94EE69182F882309F41CC10E9439
:1018E000056E8D8380917A0190917B01A0917C019E
:1018F000B0917D01898F9A8FAB8FBC8F20917E0133
:1019000030917F0140918001509181012D8B3E8B60
:101910004F8B588F8091820190918301A091840117
:10192000B09185018D879E87AF87B88B112331F0E9
:101930009D81911103C080E00E94097A809129065F
:1019400090912A06A0912B06B0912C0635E1B69510
:10195000A795979587953A95D1F79C01AD01217090
:1019600033274427552729873A874B875C8720E010
:1019700030E0A90160918A0370918B0380918C0300
:1019800090918D030E94E9EA882309F4C8C083E49A
:101990000E94EE69882309F493C00E94346E698B1B
:1019A0007A8B8B8B9C8B4EEB52E05F834E838A014C
:1019B00057E05887412C512C98EC692E92EC792EE7
:1019C000812C912C28ECA22E22E4B22E312C212C39
:1019D000F101EE0FFF1FEE0FFF1FE00FF11FC080A0
:1019E000D180E280F380A7019601C501B4010E9475
:1019F000E9EA181614F446015701A7019601C3013C
:101A0000B2010E946AF387FF02C0260137018FEFFF
:101A1000281A380A97E029163104D1F6A885A15072
:101A2000A887045E1F4FA111D1CFA3019201C50168
:101A3000B4010E9407F220E030E040E05FE30E9442
:101A40004EEB29893A894B895C890E9407F24B0148
:101A50005C012DEB37E346E855EB0E94E9EA87FD90
:101A60000AC02DEB37E346E855E3C501B4010E94F7
:101A70006AF318162CF580E00E94097A17E0EE80D0
:101A8000FF8007E0F70161917191819191917F0150
:101A90006F01F4E0CF1AD108A50194010E9406F26B
:101AA000D6016D937D938D939C931397015051F7BD
:101AB0001150EE81FF817C96FF83EE831111DFCF01
:101AC00089859A85AB85BC85892B8A2B8B2B79F0F0
:101AD00020E030E0A90160918A0370918B0380912E
:101AE0008C0390918D030E94E9EA811126DD8AE53D
:101AF0000E94EE69882359F00E94346E69837A83CC
:101B00008B839C8360E0CE0101960E94957A8D8143
:101B10000E94097A14C02091B9022D83E3CEFD8181
:101B2000F11108C029853A854B855C85232B242B30
:101B3000252BE9F266DD8CE397E10E9491849D817B
:101B4000992349F08091B902811105C057DD8DE1DB
:101B500097E10E94918455DD8FE097E10E94918486
:101B60008091B90241DD4DDD82E097E10E949184D0
:101B7000C090BA02D090BB02E090BC02F090BD02CF
:101B800020E030E0A901C701B6010E946AF31816EF
:101B90000CF040C042E0C701B6010E94F3B68DE0F0
:101BA0000E9470848AE00E947084298D3A8D4B8D4A
:101BB0005C8D60917A0170917B0180917C019091A4
:101BC0007D010E94E9EA81111FC02D893E894F895C
:101BD000588D60917E0170917F018091800190917C
:101BE00081010E94E9EA81110FC0209182013091A8
:101BF000830140918401509185016D857E858F859B
:101C000098890E94E9EA81110E9470406C96E2E195
